:020000024000BC
:100000006FE0E20600000000001801180028012837
:100010000228032800290129022903290429052986
:10002000062907290829002A012A022A032A042A64
:10003000052AA62A90E80600343404004204002071
:10004000BC040020CA0300209C03002032030020CF
:10005000D635040016360400B4370400343A0400E0
:10006000183B040094320400463204008C02002045
:1000700036020020D23F0400D0070020AC35040037
:10008000DA3C04007A8406005C860600C886060016
:100090007A390600B2390600146A0500885D050049
:1000A000D87E06000A3D0400C24106007AF0040032
:1000B0000AF1040064F10400FA470400384804001F
:1000C000B8460400A2B20400BEAD0400480A0020F5
:1000D000F6BE04005CC20400DEA0040080A00400A0
:1000E00042A404002AA104005EA00400D6A00400DB
:1000F00014A00400A4A10400FCA10400ACA104000D
:10010000B0A1040046A2040004A2040034A204002A
:10011000F4A60400F8A60400A0A10400A8A104000D
:1001200044A20400F6A60400F2A2040052A80400AF
:10013000BACF04002ED0040068D00400EEB404004E
:1001400004B504003CB5040086950400AC97040097
:10015000889804009E650400346004009A8B0400B3
:10016000B0600400E2860400C2C5060012BE0600AC
:10017000FEC2060020DA0600ECD806004ADD0600C2
:1001800006DD060042DD060096DE0600EEAC060047
:1001900026DE06007CD00600A2D00600C2D00600F3
:1001A00006DF0600F2D6060090D6060076DF0600CF
:1001B00072AF060006B0060026B00600D8AF0600F3
:1001C00094610600984C0600EE4F0600D64D0600DE
:1001D000B0570600307F0600727E060022AD060092
:1001E00056410400C2390600A24106009A420600A8
:1001F0003A750600C675060048770600C8B80400C0
:100200007E60060044580600744A0600025B060041
:10021000484C0600BA0900202E3A060070DD0600A0
:100220000ADD06003EDD06003ADD0600BE390400A8
:1002300032B6040078DD060080630600E464060040
:100240005065060064C3060074DD0600BEDD0600CE
:10025000145D0500C2DD060068250020802E002008
:1002600044C30600E2C40600C6DD06001ADE06002E
:100270001EDE06007CDD0600B6DD0600BADD0600E7
:1002800022DE0600406106000000000000000000C1
:10029000000000000000000000000000000000005E
:1002A000000000000000000000000000000000004E
:1002B000000000000000000000000000000000003E
:1002C0006373B60082801C419105110523AEF5FED3
:1002D000C5BFB737002037370020938787F413074F
:1002E00047666373F700828023A007009107D5BF9C
:1002F000411122C4B747024006C603A4C72023A663
:1003000007200F10000011C199E5B747024023A64E
:100310008720014545A093073500C207C183F19BA3
:10032000C207C183130740036366F7023737002013
:100330000325471E373700208326C71D6391A60279
:10034000373700200327072769D3C207DD8D05450E
:10035000029765BF373700200325071EE1BF7A21CA
:1003600031EF5A21636CF704B73600203306F740AB
:1003700021489386C61E6375C8028328050003D8EA
:100380006600138687001D8F2A9661175AA22320C4
:1003900016012313060010C15EA1130788FFFAA2FD
:1003A0006EA1EE222105B387F540FEA2B7470240B9
:1003B00023A68720B2402244410182800841BDBF6C
:1003C000B747024003A8C72023A607200F1000004C
:1003D00001E523A607218280B737002003AE471E20
:1003E000B737002003A3C71D8146F28763FE670865
:1003F00083A80700636DF50863EBA80813878700DF
:100400006364E508F223216705076319E6003736C0
:100410000020034746FF0507230AE6FE3736002083
:100420001305C61ECE237A21239307001306C61E8A
:100430002E97420741837AA16383C7033735002093
:100440000325051E630DF500EA2211E9DE2223A033
:1004500016012107BE95A105CEA27AA2B6879843C0
:1004600063046702B736002083A6061E630ED7001A
:10047000762399EAD6234E231843A106AE96D6A337
:1004800098C37E22A1077EA2B747024099B7BE86D5
:10049000C687A9BFB7370020B736002083A7471EFD
:1004A00003A6C61D2A87B305B5406314F6003A8536
:1004B00029A8938687009C43E369D7FEE377F7FE7C
:1004C0002E85E3E4D5FEE3F2F5FE828023AC05FE43
:1004D0001C4181E70CC18280BA8703A787FF6DFFAB
:1004E00023ACB7FE8280411126C24AC0B744024005
:1004F00006C622C403A9C42023A604200F100000AE
:1005000009E923A62421B240224492440249410130
:1005100082802A842105BD654205C18D4181C93B88
:1005200011C9FD572320050042A17CA123A6242147
:100530002105D1BF23A624210145F1B701114AC8E5
:100540004EC6B747024006CE22CC26CA83A9C72092
:100550002A8923A607200F10000037350020032426
:10056000851E8144014609E889ECA1654A859730DA
:1005700004E0E780607725A08347E4FF639D2703BD
:10058000A1C0A6851305851E973004E0E78000F51D
:1005900069DCA1654A85973004E0E780002FF240CE
:1005A0006244B747024023A6372126854249D244F8
:1005B000B2490561828091E02286032484FF65B7F9
:1005C000A284E5BFB737002083A7872399E33E8540
:1005D0008280BA236315B7009823E30AA7FEDC479D
:1005E000F5B7B747024003A7C72023A607200F107F
:1005F000000001C599C1814711E6B747024023A613
:10060000E7208280B386F50003C80600B306F50034
:10061000850723800601E317F6FEC5B7374702407A
:100620008327C720232607200F10000019C191C17E
:1006300011E6374702402326F7208280910503A761
:10064000C5FF11057D16232EE5FEDDB737470240B5
:100650008327C720232607200F10000001C533077A
:10066000C50011E6374702402326F72082800505A2
:10067000A30FB5FEE31DE5FEF5B7B747024083A61D
:10068000C72023A607200F10000081473307F5007D
:100690000307070019E7374702402326D7203E8586
:1006A00082808507E5B7011126CA4AC8B7470240CC
:1006B00006CE22CC83A4C7202A892E8623A6072013
:1006C0000F100000131506019305F004418132C696
:1006D00005312A8401C53246CA8521372285F24078
:1006E0006244B747024023A697204249D24405619D
:1006F0008280B747024003A7C72023A607200F1018
:10070000000001C599C1814711EAB747024023A6FD
:10071000E720054582808507E309F6FE3308F500EA
:10072000B386F500034808009422E306D8FEB747D5
:10073000024023A6E72001458280B747024003A775
:10074000C72023A607200F1000009307F6FFBE95D1
:100750002A966317C500B747024023A6E720828088
:10076000FD159C310505A30FF5FEE5B7374702409F
:100770008327C720232607200F10000001C5330759
:10078000C50019E6374702402326F720014582803D
:1007900005058346F5FFE397B6FEE31BE5FE374705
:1007A00002402326F72005458280797126D2B7348E
:1007B000002022D403A4842306D64AD04ECE52CCA5
:1007C00056CA5AC85EC662C455C4373A0020373983
:1007D0000020B7390020814BB73A002037CBC90140
:1007E000130ACA231309C91E938949283E2099EF89
:1007F0005C44639A0B0023ACF422032CC4002285D2
:10080000C1366284A9A823A6FB00C5BF83A70A231B
:1008100082971C443307F5406376F50003A749002F
:100820001D8F2A979306FB3763EAE6062328090003
:100830002E200820973004E0E78020055C405844D3
:10084000B1C70C4403A64900AE97BE8663E4B70067
:1008500063E4C700B386C74014C4A28B3A8459F43A
:10086000B73700209387C71E984B854663FCE60484
:100870007D1798CBB250225492540259F249624AE1
:10088000D24A424BB24B224C4561828063950B00A9
:1008900023ACE4229DB723A6EB0085B703278A0289
:1008A00019CB63EDA7003385A74083270901637443
:1008B000F5002328A900A28B404455B703A749009F
:1008C000BA97D5B723A8070075B701114EC6B74729
:1008D000024006CE22CC26CA4AC852C483A9C720E9
:1008E00023A607200F100000373400209307442868
:1008F000C843DC2713044428B9CFB73700209387B7
:10090000874003D7470B21CB83A4070B6385A4043F
:10091000B73700201387C71E184B138AC71E630FF3
:10092000A70E3739002083270923829763E5A40E99
:1009300083270923898C829703270A0163F3E40044
:100940002687B307A7003E85544063E4E70063E4CD
:10095000D7003385D740B747024023A637215C40F4
:10096000639DA702B73400209384C41E9848B7370C
:10097000002083A707236315A70A82975440B7472F
:1009800036FE938707C8B6973387A7003A85636416
:10099000F7006364D7003305D740B734002093874E
:1009A0004456DC539384445699CBB737002083A632
:1009B000075E3707CDFF7D179C46F98F9CC611E176
:1009C00048408547DCC4B737002083A74726829775
:1009D00005E1DC5089CFDC4499CB974006E0E78005
:1009E000E0CC973006E0E780202A23A60400753B80
:1009F000DC5091CBB737002003A7075EB706330062
:100A00001C47D58F1CC7F2406244D2444249B249C8
:100A1000224A056182805C40BE9419BF268525BFAD
:100A2000829794485840B387A6003E8563E4D70078
:100A3000E3E5E7F63385E7408DB7B737002023A419
:100A4000A7F411C5B737002005472386E7F4828055
:100A5000B737002003A787F4411122C406C61384C8
:100A600087F411C30297B737002083C7C7F493F701
:100A7000F70F99E323200400B24022444101828011
:100A8000011126CAB734002022CC4AC893874428D3
:100A900006CE4EC652C456C2DC2737390020938496
:100AA00044281304892195E3B737002093874756DC
:100AB000D833058B19CBF8339946639BE60AA3829A
:100AC0000700EF10B0645C4482971C4491C3829786
:100AD00037340020B73900209307C41E03A74923E9
:100AE0009033130AC41E8347C41E93961700BA9608
:100AF0009622C9CA8347C41E63EEC7082306041E94
:100B000037340020930744569C37130444566391AE
:100B10000710B737002083A70723F5C3DC4023283D
:100B2000FA006131B737002083A74726E9CB7C3034
:100B300011476366F70CB73700209387075BDC2704
:100B4000918BD5EFB737002083C7C7F493F7F70F22
:100B5000DDE783461A0003A6492363C7D70C624426
:100B6000F240D2444249B249224A924A0561B1BB9D
:100B7000F8339D46E39BE6F4A3820700EF1010597B
:100B80001C4899B7850793F7F70F2306F41EE3EC8B
:100B9000C7F48DB786073E970E2323100700034541
:100BA000C41EB737002083A7472113172500B73A83
:100BB0000020BA979C4323960A22829783D7CA22A1
:100BC0000347C41E93C7F7FF7D8D9317170003A734
:100BD00049233E971E235D8D0AA38347C41E81C708
:100BE00085072306F41E8327892181C78297232C3A
:100BF00009200347C41E83471A00E371F7F0F2404F
:100C00006244D2444249B249224A924A05618280F2
:100C10007C3093F7F70FE39E07EEA30404009730B0
:100C200006E0E780C054F5B51397170032971A23F2
:100C300079F785071DB7374702408326C720F1772C
:100C4000FD17F58F2326F72001000100B73700209C
:100C50009387C71EC84F832787262326D7206A0578
:100C600093C7F7FF99835D8D8280B737002083C7D4
:100C7000F71E89CFB737002083C7072991CBB73735
:100C8000002003A3472963070300028305458280F0
:100C9000094582801305F00F8280B737002003C614
:100CA0004740B737002003A747FC81476315F6008C
:100CB000814636858280BA8613078702835587FD71
:100CC000E389A5FE850793F7F70FCDB7B737002067
:100CD00003C75740B737002083A707FE2A860507BA
:100CE00081463E859E236388C7008506930765007D
:100CF000E3E9E6FE01458280B737002003A787FDC0
:100D000019E3014615A81C4703D8A700636B05012A
:100D100083584700B38608016355D5008146639424
:100D200016011843F1BF3E86C10703D3A7FF63171F
:100D3000A30099C123900501328582808506C206F1
:100D4000C182F1BFB737002003C64740B737002044
:100D500003A7473A81476315F600814636858280AE
:100D6000BA861307C703835567FCE389A5FE850789
:100D700093F7F70FCDB7032785116DCB411122C42F
:100D800006C65C258345E5042A8493F7C70F5CA556
:100D90001437522713958601618563F7C5066351A1
:100DA0000506082793F6F60714B7054693E62700CD
:100DB0006314C50093E6170054A45C4389075CC321
:100DC0004CB8032504112E864C430905EFF07F81B2
:100DD000832784115038D443DA27B296118FD4C3B5
:100DE000DAA789473CBCB73700200347640383C7B1
:100DF000E7246371F7045C2493E707015CA41DA852
:100E000093E717005CA46DBF9376F60F6359050254
:100E10000827854513E627006314B50013E617007D
:100E200050A454B8A304070085473CBC8327841111
:100E30009C43D5FBB240224401454101828093E7A7
:100E400017005CA454B8A3040700032504114C4305
:100E50000905EFF00FF9832784115038D443DA27BE
:100E6000B296118FD4C3DAA78D47C1B705458280EA
:100E7000B737002083A74753411122C406C6858B8C
:100E80002A84D5E34165130525F5977005E0E780D1
:100E900080DC51C93C253EA583270412ADE3232005
:100EA000A4122322A41285472311F4042320050051
:100EB0007C2854415EA5583418A5054718B5373726
:100EC0000020032787581385170215811C437D15C1
:100ED0001375F50F9CC25C43DCC21C479CC65C4783
:100EE000DCC61C4B9CCA5C4BDCCA1C4F9CCE5C4FC6
:100EF000DCCE19CD9386060213070702C1BF8327F4
:100F0000441288C3835724042322A412850769BF8F
:100F1000B7370020938787409A2705079AA7B240E2
:100F20002244410182805C2423090400054593C7C3
:100F300047005CA4EDB71C2D93F7E70FC5EB1C3DF4
:100F4000D5E73029542509CA373700208345650382
:100F50000347F72463E7E50013F7060149CB014790
:100F600009C6C18A0357251E81C68356651E36975A
:100F70003DCFB737002003D5C7281307C712374620
:100F80000F00B335A702411113060624814622C47F
:100F900026C206C67D543305A70297D006E0E78037
:100FA0000042B737002083C73725B384A700B7377F
:100FB000002003A7474A8327070963F387003E847D
:100FC000184375FBB737002083A707238297814713
:100FD0006364A400B307A440B2402244B3B79700AF
:100FE00093C7170092443E854101828081473E8528
:100FF0008280B737002003A7C7587C53FDFF82804B
:1010000001114EC6B73900209387894022CC03A432
:10101000470A26CAB7340020938744289E274AC827
:10102000035964080325040906CE3309F902B747BA
:101030000F001387F7239387072452C456C25AC060
:1010400093898940938444283A993359F902636D0E
:101050002503373A002083270A2333092541829745
:101060006367A9023309A940634609028357040450
:10107000A30F040085072310F4048347041463942A
:1010800007102285CD2D11A2DC403E95D9B7DC405A
:101090003E99C9BF83270A23829703278408636F79
:1010A000E508198D7E3C9A248E07B387E702130763
:1010B000003293870719B3D7E70263E5A708B74A59
:1010C0000F00138BFA23938A0A248357040485079D
:1010D0002310F4048347041499E32285692D2285A3
:1010E000976005E0E78020C8631D05248326040976
:1010F0008327C408D840B6973E8563E4D70063E4ED
:10110000E7003385E7407C3C035964082328A408A2
:1011100085077CBC9E243309F9025A993359590337
:10112000636C25053309254183270A238297636968
:10113000A9043305A940E34A05F80DBFDC40998FA7
:101140003E958DB7A1452285976005E0E780E0B91F
:10115000A305A402B737002003A307276303031ED8
:101160006244F240D2444249B249224A924A024B76
:101170008945154505610283330927412A996DB7D1
:10118000DC403E997DB72285512D2285976005E090
:10119000E78060BD6317051A8A2483576408B74641
:1011A0000F001386F623B387A7029386062403272E
:1011B0000409230B040283AA4400B297B3D7D702D1
:1011C000636BF718B307F7408326C4082324F40899
:1011D000014BB387E6003E8963E4D70063E457011F
:1011E000338957411E3023282409A1CB8356040498
:1011F0005A3037460F0056B03387E640B387E702D0
:101200003A301306062481468145BA97C207C18346
:101210003385A7023EB097D006E0E780401A11CD93
:101220004A95333925012E99AA8763142B016364EB
:101230005501B30755412328F40883270A238297D1
:101240002A8983270A238297E30D25FF83270A2310
:101250000329840882976365A9103305A9406302B6
:10126000051283DA84008357640837490F00130797
:10127000F923B387570313090924BA97B3D7270370
:101280003737002003473725BA9763ECA70EB335ED
:101290002503035A2402568681463305250397D039
:1012A00006E0E780C011330BAA0033055A03374626
:1012B0000F00130606248146814597D006E0E7809B
:1012C00000100DC1B337250356868146B305B90218
:1012D0003305A902BE9597D006E0E780400E33059E
:1012E000AA402AB03545973006E0E780E0F823A20F
:1012F000890A383485476318F706930700FD7CA4F4
:10130000B737002003A5C754DC24B5C7EFF0EFF2D0
:10131000B736002003A6C658B73700209387475634
:101320001547F8B35846F977FD17F98F5CC60F10CB
:10133000000083A7C6588966060B94C723A26707D7
:10134000D8C7F2406244D2444249B249224A924A42
:10135000024B05618280B3065701B387F640ADB5F5
:10136000DC403E99DDBD930710FC7CA4B73700201C
:1013700003A5475451BF8145973004E0E780C0AED4
:1013800041BFDC2423A2090A85C3B737002003A587
:10139000C753973004E0E780C0E7B7E700E03707BE
:1013A000000223A2E72071BF83479402854562446F
:1013B000F240D2444249B249224A924A024BB39582
:1013C000F500C205C18101450561172304E06700EE
:1013D000C34B011122CC4AC84EC606CE26CA52C4FF
:1013E00056C25AC0383585472A842E898329050973
:1013F0006315F71E83570508035BC503373A0020C2
:1014000093064A2883DA8600130A4A2863FF67197D
:101410001429639CE618032785116318071803270E
:10142000450A6314071874351D476390E6182A3D72
:10143000330BFB409307204E330565038324440997
:1014400037460F001306062481463305F502B737E9
:10145000002083C72725B3549502B3B5AA02BE94D2
:10146000C204C180231394083385AA0297D006E0F2
:10147000E780E0F4AA9933B5A9002E954E8783271B
:101480004A0019E163E4F9003387F940B384540357
:10149000B7460F009387F623938606242320E9009E
:1014A000BE94B3D4D40293171B00A6976369F70EBA
:1014B0001D8F2320E900B739002083A70923832447
:1014C0000900829763EEA4103385A440635D050A8A
:1014D00083A70923373B0020130B4B288297032750
:1014E00009006365E510198D7E3C03578B008E075C
:1014F000B387E7021307003293870719B3D7E702D0
:1015000063EBA70E374A0F00930AFA23130A0A2443
:101510008357040485072310F4048347041499E3D4
:101520002285912C2285976005E0E780C0836DE1DC
:10153000832604098327C40803274B00B6973E85FA
:1015400063E4D70063E4E7003385E7407C3C8354E1
:1015500064082328A40885077CBC83578B00B384C8
:10156000F402D694B3D444036363950CB30495405A
:1015700083A7092323209900829763EEA40A338569
:10158000A440E34705F8B737002083C7372563E257
:10159000A708B737002023A6874A01459DA88326C0
:1015A0004A00B387F6403E9729B783576408374708
:1015B0000F00B38457039307F723A69793040724D8
:1015C000B3D4970263E79900B3849940232099002C
:1015D000DDB583274A00BE99C5BF23A03501E1BD13
:1015E000B737002083A78728BE94F9BD83274B0017
:1015F000998F3E95D5BDA1452285975005E0E7809E
:10160000C06EA305A402B737002083A7072781EF88
:101610007D55F2406244D2444249B249224A924A3C
:10162000024B05618280894515458297D5B7B30481
:101630009740AA9435BF83274B00BE9489B721CD2C
:1016400001116C0022CC06CE2A84613339C1FD57CA
:101650006307F502B73600209386C623FC3A9456FA
:10166000324791C285836360F702B307F7403EC6F5
:10167000B24503459402972004E0E780E036F2404B
:10168000624405618280B736002083A6862836979B
:10169000E9BFBD32EDB78280B7370020797113877B
:1016A00087404AD00329C70906D622D426D24ECE77
:1016B00052CC56CA094763000906B7340020938A02
:1016C000874093874456FC339546938444560D4790
:1016D0006383F604DC442A8A99CB973006E0E780DE
:1016E000E0FC972006E0E780205A23A60400FD597D
:1016F0006C004A85F93915E937150020130505D521
:10170000EFF0AFB3A147DCA0B737002083A7C758DD
:101710000947F8D30D47B250225492540259F24966
:10172000624AD24A3A854561828063743501324407
:10173000AA8903290900E31D09FAFD571307F00FD1
:10174000E38BF9FC914763F187029307B4FF2320F1
:10175000FA0023A8FA0A0147DDFFB737002083A764
:1017600087282320FA0045BFB737002083A78728A2
:10177000ED17A297E9BF797126D206D622D44AD0B6
:101780004ECE52CC56CA5AC85EC683475503034450
:101790007513AA843E941374F40F9307400263F602
:1017A00087001304B4FD1374F40F03AA841383AAEF
:1017B000C413A38B841222865285D68597D006E067
:1017C000E78060BA058915E503CBD4120149814948
:1017D000337B6403930B50024A865285D68597D09B
:1017E00006E0E78040B8058915C563916903137465
:1017F000F90F238B8412B250225492540259F249A9
:10180000624AD24A424BB24B456182808509E20965
:1018100093D989410509E31179FDE1BF8327850942
:1018200003560504797193D60701BD8EC206C182A5
:10183000358E1357764093575640898B058B5D8FB5
:1018400093573640918B5D8F93571640A18B5D8FD8
:1018500093171600C18B5D8F9317360093F707021D
:101860005D8F931756009355860093F707041E0665
:101870005D8F1376F60F518F93D7554013D63540B1
:10188000118A898BD18F13D67540D18F13D615400D
:10189000218AD18F13961500418AD18F1396350076
:1018A00013760602D18F13965500137606049E0513
:1018B000D18F93F5F50FCD8FA20745465D8F330786
:1018C000C70222D42A8426D252CC56CA032A8413B1
:1018D000832AC4135AC806D63697420741839357C2
:1018E0007740135557400989858BC98F1355374069
:1018F0001189C98F135517402189C98F13151700F6
:101900004189C98F1315370013750502C98F131547
:10191000570093558700137505041E07C98F137769
:10192000F70FD98F13D5354013D755401189098B3F
:10193000498F13D57540498F13D515402189498F9B
:10194000139515004189498F1395350013750502CC
:10195000498F13955500137505049E05498F93F51E
:10196000F50F4D8F2207D98FB387C7024AD04ECECD
:101970005EC662C4B697C207C18313D7774013D53A
:1019800057400989058B498F13D537401189498FF5
:1019900013D517402189498F139517004189498F25
:1019A0001395370013750502498F1395570093D58A
:1019B0008700137505049E07498F93F7F70FD98F9A
:1019C00013D5354013D755401189098B498F13D54D
:1019D0007540498F13D515402189498F13951500FE
:1019E0004189498F1395350013750502498F139569
:1019F0005500137505049E05498F93F5F50F4D8F1E
:101A00002207D98FB387C702130650025285D685A5
:101A1000B697BD8E93940601C18033F6C402137B42
:101A2000F60F97D006E0E780009405890DED834717
:101A3000D41201498149B3849702130C5002C1802A
:101A40004A865285D68597D006E0E780C091058901
:101A5000937BF90F11C563863403850993F9F90F58
:101A60000509E31F89FD230B6413B25022549254DD
:101A70000259F249624AD24A424BB24B224C45616A
:101A800082805E8BCDB78327C508035685087971A0
:101A900093D60701BD8EC206C182358E135776409C
:101AA00093575640898B058B5D8F93573640918BAA
:101AB0005D8F93571640A18B5D8F93171600C18BD6
:101AC0005D8F9317360093F707025D8F93175600CB
:101AD0009355860093F707041E065D8F1376F60F65
:101AE000518F93D7554013D63540118A898BD18FAA
:101AF00013D67540D18F13D61540218AD18F1396F6
:101B00001500418AD18F1396350013760602D18FC6
:101B100013965500137606049E05D18F93F5F50FA5
:101B2000CD8FA20745465D8F3307C70222D42A8492
:101B300026D252CC56CA032A040A832A440A5AC817
:101B400006D636974207418393577740135557403F
:101B50000989858BC98F135537401189C98F135552
:101B600017402189C98F131517004189C98F131593
:101B7000370013750502C98F131557009355870059
:101B8000137505041E07C98F1377F70FD98F13D567
:101B9000354013D755401189098B498F13D57540AE
:101BA000498F13D515402189498F13951500418917
:101BB000498F1395350013750502498F139555000C
:101BC000137505049E05498F93F5F50F4D8F220778
:101BD000D98FB387C7024AD04ECE5EC662C4B697CD
:101BE000C207C18313D7774013D557400989058BA6
:101BF000498F13D537401189498F13D51740218953
:101C0000498F139517004189498F13953700137534
:101C10000502498F1395570093D587001375050466
:101C20009E07498F93F7F70FD98F13D5354013D7F8
:101C300055401189098B498F13D57540498F13D5AC
:101C400015402189498F139515004189498F1395B6
:101C5000350013750502498F13955500137505045A
:101C60009E05498F93F5F50F4D8F2207D98FB387C6
:101C7000C702130650025285D685B697BD8E93943F
:101C80000601C18033F6C402137BF60F97C006E04D
:101C9000E780606D05890DED83471408014981498E
:101CA000B3849702130C5002C1804A865285D685B0
:101CB00097C006E0E780206B0589937BF90F11C57B
:101CC00063863403850993F9F90F0509E31F89FD3C
:101CD000230F6407B250225492540259F249624AC7
:101CE000D24A424BB24B224C456182805E8BCDB7CB
:101CF0008327450903568508797193D60701BD8E60
:101D0000C206C182358E1357764093575640898B51
:101D1000058B5D8F93573640918B5D8F935716409F
:101D2000A18B5D8F93171600C18B5D8F93173600C3
:101D300093F707025D8F931756009355860093F72C
:101D400007041E065D8F1376F60F518F93D755400B
:101D500013D63540118A898BD18F13D67540D18F18
:101D600013D61540218AD18F13961500418AD18F41
:101D70001396350013760602D18F1396550013760D
:101D800006049E05D18F93F5F50FCD8FA20745462A
:101D90005D8F3307C70222D42A8426D252CC56CA7A
:101DA000032A040B832A440B5AC806D636974207E7
:101DB000418393577740135557400989858BC98FC5
:101DC000135537401189C98F135517402189C98F81
:101DD000131517004189C98F1315370013750502B4
:101DE000C98F1315570093558700137505041E07F7
:101DF000C98F1377F70FD98F13D5354013D75540B7
:101E00001189098B498F13D57540498F13D515401A
:101E10002189498F139515004189498F1395350004
:101E200013750502498F13955500137505049E051A
:101E3000498F93F5F50F4D8F2207D98FB387C702CE
:101E40004AD04ECE5EC662C4B697C207C18313D7CE
:101E5000774013D557400989058B498F13D53740F3
:101E60001189498F13D517402189498F1395170080
:101E70004189498F1395370013750502498F1395D2
:101E8000570093D58700137505049E07498F93F774
:101E9000F70FD98F13D5354013D755401189098BCA
:101EA000498F13D57540498F13D515402189498F26
:101EB000139515004189498F139535001375050257
:101EC000498F13955500137505049E05498F93F5A9
:101ED000F50F4D8F2207D98FB387C7021306500223
:101EE0005285D685B697BD8E93940601C18033F690
:101EF000C402137BF60F97C006E0E780C046058951
:101F00000DED8347F40801498149B3849702130C0E
:101F10005002C1804A865285D68597C006E0E78088
:101F200080440589937BF90F11C5638634038509C5
:101F300093F9F90F0509E31F89FD230F6407B250D8
:101F4000225492540259F249624AD24A424BB24B4D
:101F5000224C456182805E8BCDB74111B73700209E
:101F600026C283A4074606C622C44AC08547C1C408
:101F700003A4C40A854741C03C241307700A639335
:101F8000E70858301C34B736002013864628B3873C
:101F9000E7021A265042B387E702130700329387FD
:101FA0000719B3D7E70203A74409938446283E974D
:101FB0003A896364F7006364C7003309C740B737E1
:101FC000002083A70723232025018297B307A94078
:101FD0006374A900D840BA9781E79307F00F21A84E
:101FE00058309306204E3307D702E3F8E7FE9307F5
:101FF00080FA3CA48147B2402244924402493E8583
:10200000410182801307800AE399E7FCB73700207B
:1020100083A7072382972A893545972006E0E78022
:10202000A025B7370020938747562D47F8B358307F
:102030001C34B736002093864628B387E7029A26D9
:10204000D442B387E7021307003293870719B3D747
:10205000E70203A744093E973A866364F700636486
:10206000D7003306D740E31AC9F637D50500130564
:10207000C5AFEFE09F9CB737002083A7C75809473B
:10208000F8D7A1BF397122DC3734002093074456BA
:102090009C4F06DE26DA4AD84ED652D456D25AD0B3
:1020A0005ECE62CC66CA6AC86EC613970701635DCE
:1020B000071EB737002083A4074683A9C40A83C735
:1020C000990003A7C9009207330CF70003452C00C1
:1020D000314705053305E50203574C003A954205A3
:1020E0004181EFE04FC0AA8B630B051C130DC500A7
:1020F0002324A50103462C00B145F97A3306B60224
:102100001304445623130C000149373A0020373B8F
:102110000020B73C0020930D9005FD1A6A962326F7
:10212000CC0003C679009307D0070325CA583306AD
:10213000F60285671CC5B7073300060630D10326B3
:102140008B550C4293F5F5E70CC20C4293F5F5E77D
:1021500093E505100CC203A80C5E83258800DD8D75
:102160002324B80083A509002328B5050CC6835590
:102170006C000326CC002E962324CD0003461C00C1
:10218000930550024A96A301CD0003C504080146F9
:10219000A3000400972006E0E780A0E50326CA58C4
:1021A0004846B37555014CC60F1000000326CA58A7
:1021B000896503288B550CC6930500F84CA0832530
:1021C0000800B1818D89E1E1930560196CD248C6A0
:1021D000A30204008545A30004000CC2052F97202C
:1021E00006E0E78040011030058A5DCAEA85268551
:1021F00097C005E0E78040BB0DED03465D004DC292
:1022000083556C0003554C00B29563DBA508AC28E0
:10221000A848918D8905AA9503258D00EFE06FBC34
:1022200023020D0083455D0003566C002E96231398
:10223000CC008325CA58310DB0517DFE03462C00D9
:1022400005091379F90FE36EC9EC98245E85A38123
:10225000EB0083470C00A3820B002383CB00238277
:10226000FB006254F250D2544259B259225A925A47
:10227000025BF24B624CD24C424DB24D21611713BE
:1022800005E0670083EB832508000948B1818D894B
:10229000639505019305E04315BF9305E01B3DB72A
:1022A0007D562302CD0071B7B737002083A7C758EA
:1022B000FC5791C7B737002005472386E7F4F25053
:1022C0006254D2544259B259225A925A025BF24B8A
:1022D000624CD24C424DB24D21618280797122D440
:1022E00006D6BC312E8423160100DC87DC211008C1
:1022F00002C05C87DC318A8502C2DC8602C402C867
:1023000002CA02CC02CE552C0347F1011C20014524
:10231000631EF7000347E1011C3001456318F70015
:102320000345D1013C201D8D13351500B2502254B8
:10233000456182800111B737002022CC03A4474DAC
:1023400026CA4AC84EC606CEAA8413092500854966
:1023500005C09C303830858B6304F700405CCDBFEE
:102360001946930544004A85EFE0AFB8E31835FFFE
:102370002285F2406244D2444249B24905618280DA
:102380004111B737002022C403A4474D26C24AC0DA
:1023900006C693042500054901E82285B24022447F
:1023A0009244024941018280A6851305A4023D376B
:1023B000E30525FF405CCDB74111B737002022C4AB
:1023C00003A4474D26C24AC006C69304250005490A
:1023D00001E82285B24022449244024941018280B0
:1023E000A6851305A401DD3DE30525FF405CCDB7BF
:1023F000011122CC604126CA4AC84EC652C406CE3C
:10240000AA841D4A130965058549BC446364F40028
:10241000054591A0D8345C206317470503C78402A3
:102420006304F7000040D5B7583083C75405E31B59
:10243000F7FE1946CA8513056400EFE08FABE3137E
:1024400035FF582483C79402E31EF7FC7A24BE3478
:10245000E31AF7FC0145F2406244D2444249B249D2
:10246000224A05618280E31FF7FA583083C754057A
:10247000E31AF7FA1946CA8513056400EFE06FA75F
:10248000E31235FBC1BF4111B737002022C403A4BA
:10249000874806C626C24AC079C88347840B1307FB
:1024A000700A6393E70A0347140E8347A40BB736F9
:1024B000002013864628B387E7021A26938446280D
:1024C0005042B387E7021307003293870719B3D747
:1024D000E7020327440A3E973A896364F70063647E
:1024E000C7003309C740B737002083A7072323203D
:1024F00025018297B307A9406374A900D840BA9711
:102500008DC70347140E9306204E3307D70263FE90
:10251000E700930780FA230CF40A01442285B240B5
:102520002244924402494101828037350600130556
:10253000E5A0EFE08FD0B737002083A7C758094741
:102540001304F00FF8D7D9BF1307800A1304F00F54
:10255000E396E7FC373506001305E5A0EFE0EFCD85
:10256000B737002083A7C7580947F8D745BF0544A8
:1025700075B70111B737002022CC03A4C74C26CA77
:1025800006CE2AC42EC6854419E40145F2406244B1
:10259000D244056182809C841830858B6304F700E7
:1025A0000044DDB719469305A10013052400EFE0B0
:1025B0004F94E31795FE0545D1BFB736002083A79A
:1025C00046551307001098C323A00700183103488D
:1025D0002500220742084297034805004297034816
:1025E00035006208429798D75831034865002207A2
:1025F0004208429703484500429703487500620825
:102600004297D8D718350348A500220742084297B9
:102610000348850042970348B5006208429798DB5B
:1026200058350348E5002207420842970348C50091
:102630006835429762052A97D8DB9831A82122078E
:1026400042052A9788212A97A83162052A9798CFB0
:10265000D831E821220742052A97C8212A97E83174
:1026600062052A97D8CF9835A825220742052A97D0
:1026700088252A97A83562052A9798D3D835E82562
:10268000220742052A97C825EC352A97E2052E979E
:10269000D8D3D843759BD8C3D84313671700D8C382
:1026A00098431367170098C303A746555C43858B6F
:1026B000BDE71C4F01451CA283A746559C4FA18333
:1026C0001CB283A746559C4FC1833CA283A74655A5
:1026D0009C4FE1833CB283A74655D84F58A2D84FB0
:1026E000218358B2D84F418378A2D84F618378B202
:1026F000985318A69853218318B69853418338A647
:102700009853618338B6D85358A6D853218358B606
:10271000D853418378A6DC53E1837CB682800100E4
:1027200061B7B737002003A7C7581605136505081A
:102730003C4B93E707083CCBB737002083A74755AE
:1027400003A7450E88C398CB03A7850E0145D8CBB8
:1027500003A7C50B98CF03A7050CD8CF03A7450C3B
:1027600098D303A7850CD8D303A7C50C98D703A784
:10277000050DD8D703A7450D98DB03A7850DD8DB3A
:1027800003A7C50D98C703A7050ED8C798431367BD
:10279000070498C38280B737002003A7C7581605DF
:1027A000136505083C4B93E707083CCBB73700207F
:1027B00083A7475503A7C50E88C398CB03A7050F6A
:1027C0000145D8CB03A7C50B98CF03A7050CD8CFDD
:1027D00003A7450C98D303A7850CD8D303A7C50C32
:1027E00098D703A7050DD8D703A7450D98DB03A7F6
:1027F000850DD8DB03A7C50D98C703A7050ED8C75D
:1028000098431367070498C3B73700209387475648
:10281000130700F8F8A38280B736002003A7865577
:1028200041114AC01C5F06C622C4998326C2858B0B
:102830003689B5CF93070006373400201CDF834765
:1028400044569304445693F7070489CFB7370020C2
:1028500083A707238297C8CC8347445693F7F70B87
:102860002302F4568347445693F7070285C38347F0
:102870004456373700200327C75893F7F70D230234
:10288000F456DC48A16614C786077CD7DC2093F792
:10289000070491EF8547DCB0B737002083A7C758FE
:1028A000096798C7130700FCD8A09848F8D30327F6
:1028B00089551C5F9183858B89CBC1471CDFB73756
:1028C0000020938747568546D4A31C5F9D83858B44
:1028D00091CB930700081CDFB7370020938747563A
:1028E0000547D8A3B737002083A74755D8430583AA
:1028F000058B19C7D843759BD8C3D843799BD8C3D8
:10290000B24022449244024941018280B7370020FC
:10291000B736002003A6C7589387465603C74656C6
:10292000058B19E79833058B01E7785265FBD8339F
:10293000A3820700828037380020032788551C5F58
:102940009583858BBDE701C61C5BBD831CA29DC61C
:1029500083278855985B460793576701635607009E
:1029600093E707C0C207C18303970600C207C18768
:1029700009C7BA970947B3C7E7029EA285C11C31B0
:1029800091CF3E951C350547194593F6F70663939D
:10299000E602E207E187394563CE070083278855C1
:1029A0003737002001459C5FED838D8BA307F756D9
:1029B000828005458280411122C406C6373400203A
:1029C00026C20327C4583DE5AE877453FDFEB734D5
:1029D0000020938444563E85B285238104009710DD
:1029E00006E0E780A04CB737002083A78755B706DD
:1029F00080009843558F98C3D857719BD8D78327A9
:102A0000C458A3820400A3800400094798C3832606
:102A1000C458B737002093874756B823058B11E772
:102A2000B833058B19E3F8526DFBB240224492444F
:102A3000410182808D47631FF500B737002083A7CF
:102A40008755B70680009843558F98C3D857719B18
:102A5000D8D775BF8547E31CF5FA5447F977FD17BA
:102A6000F58F5CC70F1000008327C4580967130651
:102A700000F898C7373700201307475650A3373759
:102A8000002003268755184231830D8B11E7130769
:102A90006019F8D3D4C7A5BF1842094631830D8BFE
:102AA0006315C7001307E043EDB71307E01BD5B765
:102AB0005D7152DC373A002003278A5586C6A2C4CE
:102AC000A6C2CAC04EDE1C43B739002037390020E9
:102AD00093F7F7E793E707081CC383A6095E370758
:102AE000CEFF7D179C46130680022A84F98F9CC670
:102AF0008327C9582800AE8423A80704930510082B
:102B0000EFD0DFB43545971006E0E780E076832705
:102B10008A559376F41F3706330023A40700984B99
:102B2000370FFCFF4E881367F70398CBF84FCA881E
:102B3000130510F8137707E0558FF8CF9843F57613
:102B4000FD16758F98C3373700208326C9581307A1
:102B50004756A3020700A3000700054798C2984301
:102B6000D285B70204001377F7E798C3984393031D
:102B7000802511491377F7E71367071098C303A758
:102B8000095E7D1F85491C47930F8002D18F1CC7AA
:102B900093079005BCCA01473400135337002693AE
:102BA0008347030013767700B3D7C740858BE1C313
:102BB00083A78555832E085E239C07042390070670
:102BC00003AECE02137EDEFF23A6CE0383AE070044
:102BD000137EF70793FE0EF833EECE0123A0C70154
:102BE00003AE4702336E5E0023A2C70383AEC8580C
:102BF000014E23A27E0603DA070663074E0303AEE7
:102C00000703038A0600135EFE00620E135E8E4108
:102C10006358CA0103AE0703135EFE002380C6019A
:102C200003DE0706137EFE0F03AA4E0663060A00A4
:102C300003DA8705E37F49FB03AE4702337EEE01EB
:102C400023A2C70383870600635CF400034E0300DE
:102C50003396C9001346F6FF3376C6012300C3003E
:102C60003E8663D3A7002A86131586016185050772
:102C70001377F70F8506E312F7F3B6402644964420
:102C80000649F259625A61618280B737002083A7F2
:102C9000C758D8479316170163D206029847931670
:102CA000170163DD06007D57B8D7373700201307BB
:102CB000C71E544F850654CF116798C798470D8398
:102CC000058B11CF3737002013074756342393E67F
:102CD000160034A3930600F854A3214798C79847D9
:102CE000058B19CB3737002013074756143393E66B
:102CF000160014B3054798C798470983058B09E761
:102D000098470583058B31CB37370020130647568C
:102D1000A30206009447B735002083A58555898214
:102D2000858AE5C69441B1828D8AE9EEA84B54525A
:102D30001376050294324DC2F9E29306D005D4CF42
:102D40008346475693E616002302D756114798C785
:102D5000D855719B13671700D8D59847931637013C
:102D600063D40602373700209306874003C6C607A0
:102D700013078740418A45C203C7C6071367070286
:102D8000238EE606056798C798479316270163DFE9
:102D9000060037370020130747565423E206E18622
:102DA00063D40600854654A3096798C798479316CD
:102DB000070163D206023737002013078740834696
:102DC000D707858AADCA8346D70793E62600A30EA8
:102DD000D706216798C78280ADD205466395C600A5
:102DE00093061006A9BF09466395C60093065006D0
:102DF000B9B70D466395C6009306900689B793064A
:102E0000B00635BF9306C0061DBF383213671700E2
:102E100038B209472DBF8346C7070946BD8A638874
:102E2000C6008346C7070D46BD8AE39DC6F491469A
:102E3000230ED70681BF8346D707918AD9DA834606
:102E4000D70793E6860061B7B737002083A7C75836
:102E5000B736002013874656904710CF90470D8213
:102E6000058A11CA30231366160030A3130600F832
:102E700050A3214690C79047058A19C610331366A0
:102E8000160010B3054690C790470982058A09E6E7
:102E900090470582058A31C6A30207009047B735DF
:102EA000002083A585550982058A59CA904131823F
:102EB0000D8A41E6A84B505313750502103221C903
:102EC00035EA1306D005D0CF03C646561366160062
:102ED0002382C656914694C7D455F19A93E61600BC
:102EE000D4D5944713962601635B06005423E2066B
:102EF000E18663D40600854654A3096798C79847BE
:102F00009316070163D40600216798C7828055DABB
:102F100005456315A6001306100675B70945631528
:102F2000A6001306500645B70D456315A600130607
:102F3000900651BF1306B00679B71306C00661B7F5
:102F4000343393E6160034B3894671B7373700201F
:102F5000B7360020138606591307075B5C372C3EF3
:102F6000484AAE97FD8BB355F5001CB25CB7858916
:102F70008DE9183B814613080002B3F7E7020147C9
:102F8000B355E50085899378F70F89C96395D70014
:102F9000A30016018280850693F6F60F0507E3115C
:102FA00007FF8280B737002093874756DC3393F7BB
:102FB000F70FD1EBB737002083A70723411122C4B5
:102FC0004AC006C626C28297373900209307095B9C
:102FD00080471309095B6302A40663688504018DB9
:102FE000B734002093870459BC2F135455009384A1
:102FF00004596364F40485676371F404813FBC2C55
:10300000032789009396570036971D8C2324E900E7
:10301000E376F4FE22448830B2409244024981456E
:103020004101171306E06700236CB737002083A720
:10303000872833848740229565B7B2402244924462
:103040000249410182808280B737002083A707238D
:10305000011122CC26CA52C406CE4AC84EC6829757
:10306000B73400209387045B8047014A6300A406BD
:103070009384045B63658506018D373700209307D1
:103080000759BC2F13545500137AF501130907593A
:10309000636BF402B739002093894928453D834684
:1030A000A90103A8840083A54900139756004297FD
:1030B000158C3A86636407016364B7003306B74032
:1030C00090C4E37DD4FC1604336A4401F2406244A8
:1030D0005285D2444249B249224A05618280B737BB
:1030E000002083A7872833848740229579B7B73794
:1030F000002003A7C7588567938707777CD3B73726
:10310000002083A7075E83A607091396560063581D
:10311000060083A6070913966600634406007453ED
:10312000FDF28280EFD0DF9273000000000000000B
:10313000970200009382C20C0383020023800200E6
:10314000630F0300F32510342EC09705000093850C
:10315000A5FD73901534EFF03FCF7300203086DC6F
:0C316000EFF0BFB2E650828000000000DB
:10316C00B73700203737002083A7471E0327C71D1A
:10317C0001456313F7008280F62399E2D623369536
:10318C009C43C5BFB737002083A5C7233737002022
:10319C009387C723138605222322C71EDA2393871E
:1031AC0085FFB73600204111BA97056523AEF61C92
:1031BC0006C61D05935637006374E5009306002080
:1031CC003307D600373500202320E51E23A0E52247
:1031DC00E11656A2231306001CC3998FE1175EA3B8
:1031EC0023130700B53FB240B73700202399A71E21
:1031FC0041018280B73700203737002083A7471E54
:10320C008326C71D01456393F6008280FA2309E7E4
:10321C00DA236373E5003A859C43F5B7184183A71D
:10322C0085FF6319B7001CC1FD5723AC05FE238F26
:10323C00F5FE8280232CF6FEC5BF411122C426C2A6
:10324C003744024006C68324C420232604200F10D2
:10325C00000009E9232694201545B24022449244EB
:10326C00410182800347E5FF9307F00F6306F700E7
:10327C00232694201145D5B797D0FB1FE780C0E8D3
:10328C00014523269420D1BF411126C24AC0B74420
:10329C00024006C622C403A9C42023A604200F1092
:1032AC00000089E523A62421154515A0B737002079
:1032BC0083C7D71E2A842E856375F400894763EE75
:1032CC008700A53FB747024023A627210D45B240F2
:1032DC002244924402494101828083A785FF99E7E9
:1032EC0003C7E5FF9307F00F6308F700B937B7473B
:1032FC00024023A627214DBF37350020238F85FEA2
:10330C001305851E97D0FB1FE780C0F0A1652285B1
:10331C006D2C014523A624215DBFB737002023A4C3
:10332C00071E8280BDCD797122D406D626D24AD012
:10333C004ECE01444147B3D78540858BB1CF1205A2
:10334C00314722953305E502B737002003A9C7277B
:10335C008544B3948400C204C180BE892A99032792
:10336C00090011C7032549002EC60297B245314703
:10337C003304E40283A7C9273E941C4489E7232025
:10338C00090023220900B2502254A58D02599254EF
:10339C00F2492E85456182800504E31EE4F88144E0
:1033AC00DDB72E85828041111397050122C406C614
:1033BC0026C24AC041872E846351070297D0FB1F57
:1033CC00E78040EC11C1953DA1673D8C2285B24050
:1033DC0022449244024941018280EDD9AA870147D7
:1033EC004146B356E440858A9DCA9207BA97B146C6
:1033FC00B387D702B736002003A9C6278544B394F8
:10340C00E400C204C1803E998327090003254900CA
:10341C0082972320090023220900258C45BF05072C
:10342C00E311C7FC8144D5BF411126C2B747024006
:10343C0006C622C483A4C72023A607200F100000B1
:10344C00B737002083A7072637340020130484F1F4
:10345C0091C782971C403E9508C031A0B737002019
:10346C0083A70723FDF71C40374703001307D73FFB
:10347C00B387E70237A72600130737ECB240BA9799
:10348C001CC0B747024023A6972008402244924410
:10349C0041018280797126D2B747024006D622D4E8
:1034AC004AD04ECE52CC56CA5AC85EC662C483A409
:1034BC00C72023A607200F10000005E123A69720A4
:1034CC000945B250225492540259F249624AD24AE6
:1034DC00424BB24B224C45618280B737002083A708
:1034EC000723BA8A368AB28B2E8BAA898297B73772
:1034FC00002003A7C7273E890144B146C147330CBE
:10350C00D40233068701104259E2C165938505F058
:10351C00414597D0FB1FE78020B219EDB73700204B
:10352C0083A7072781C7814511458297B74702407A
:10353C0023A697202D4571B7B737002003A7872303
:10354C0039E323ACA722230005008327C9270547AD
:10355C003317870023260500232475013AA1232263
:10356C005501E29723A0370123A2670123A4570139
:10357C0063040A0023008A00B747024023A6972061
:10358C00014581B73E875C47F5FF48C76DBF050411
:10359C00E317F4F6B747024023A69720214515B749
:1035AC00B737002083A70728411122C406C6373439
:1035BC0000201304C41E89C782975C483E9548C8F6
:1035CC004848B240224441018280B747024083A65A
:1035DC00C72023A607200F10000037370020034711
:1035EC00D71E6370E502373600201317150003252C
:1035FC0046233A951A21D98D0EA123A6D720014531
:10360C00828023A6D7200D458280B747024083A62F
:10361C00C72023A607200F100000373700200347D0
:10362C00D71E6372E50237360020131715000325E9
:10363C00462393C5F5FF3A951A21F98D0EA123A6C1
:10364C00D7200145828023A6D7200D458280011109
:10365C004AC83747024006CE22CC26CA4EC652C4B0
:10366C000329C720232607200F100000130705FF8E
:10367C001377F70FFD4763E3E70AB146B306D502AC
:10368C00B737002003A7C72736971C43C1CB9354E9
:10369C00450005443D893315A400131405014180F0
:1036AC00AE892685A28597D0FB1FE78020C62A8A83
:1036BC0029C9A2852685913FB737002083A7072308
:1036CC00B73400209384442882979E242A84814610
:1036DC00B385370313060064B3B73703138505327C
:1036EC00B335B500BE95EFA09221B30785003E8798
:1036FC00D44063E4A70063E4D7003387D740232486
:10370C00EA00B747024023A627210145F240624454
:10371C00D2444249B249224A05618280B7470240ED
:10372C0023A627210945DDB701114AC8B747024036
:10373C0006CE22CC26CA4EC603A9C72023A6072034
:10374C000F100000BD4763EBA70431473307E502B8
:10375C00B737002083A7C727BA979C43A1C305445A
:10376C003314A40042044180AE840145A28597D055
:10377C00FB1FE780A0B9AA8911C5A2850145713547
:10378C0023A49900B747024023A627210145F24004
:10379C006244D2444249B24905618280B747024033
:1037AC0023A627210945E5B7797126D252CCB74417
:1037BC00024006D622D44AD04ECE56CA5AC85EC64D
:1037CC0003AAC42023A604200F100000B737002042
:1037DC0083C7D71E6378F500B737002083AB072368
:1037EC0063970B00B747024023A6472199A03739AE
:1037FC00002013094928AE8A032B49008355890000
:10380C00B74736FE938707C83E9BB387C5022A8409
:10381C00B2898146B3B5C50213850732B337F500BB
:10382C0013060064BE95EFA0920D6370AB0223A645
:10383C0044210145B250225492540259F249624A31
:10384C00D24A424BB24B45618280829B83558900A0
:10385C00AA8413060064B38735038146B3B53503D8
:10386C0013850732B337F500BE95EFA05209B307A5
:10387C009500BE840327490063E4A70063E4E700D6
:10388C00B384E740D685228597D0FB1FE78000A83C
:10389C0001C904C5B747024023A64721054559BFB6
:1038AC00936504F0C205C181414597C0FB1FE780B9
:1038BC00A07811E9B737002083A7072785D7A28501
:1038CC001145829705B7373700208327872399EF57
:1038DC00232CA72285472326050004C52311550157
:1038EC0000A11CB12322050075B7BA87D84775FF14
:1038FC00C8C7CDB779714ECEB747024006D622D491
:10390C0026D24AD052CC56CA5AC85EC662C466C2C7
:10391C006AC083A9C72023A607200F10000025C169
:10392C0041443689B28A2E8AAA84B14C373B002096
:10393C00054D130C0003B30B94030327CB275E97A1
:10394C001C43B9EF9375F400B315BD0013554440F7
:10395C00C2055686C1811375F50FB93531C1832760
:10396C00CB27DE9784C323A24701630409002300FD
:10397C008900B747024023A63721014521A023A681
:10398C0037210945B250225492540259F249624AE5
:10399C00D24A424BB24B224C924C024D4561828032
:1039AC000504E31A84F9B747024023A637212145C1
:1039BC00D1BF011122CC26CA4AC84EC6B747024015
:1039CC0006CE03A9C7202A84AE89B28423A6072079
:1039DC000F100000D13B2285CE8597D0FB1FE780CE
:1039EC00E0922A8405C5B737002083D5C728130673
:1039FC0000648146B3879502B3B5950213850732EF
:103A0C00B337F500BE95EFA0826F48C01335140094
:103A1C00F2406244B747024023A62721D2444249D0
:103A2C00B2490E0505618280011122CC4AC84EC6EE
:103A3C00B747024006CE26CA83A9C7202A892E84FE
:103A4C0023A607200F10000097D0FB1FE780008CE7
:103A5C00AA8419C123110500A2854A857D36B73782
:103A6C00002083C7C71E63992701B737002003D7EF
:103A7C00C722598C23968722B747024023A63721A9
:103A8C00014591E01945F2406244D2444249B249A1
:103A9C0005618280011126CA4AC8B744024006CE8D
:103AAC0022CC4EC603A9C42023A604200F1000006C
:103ABC009307F00263E6A704B1473304F502B73964
:103ACC00002083A7C927A2979C439DCB9377F50031
:103ADC008545B395F500C205C1811181B13783A726
:103AEC00C9270145A29723A0070023A2070023A6FC
:103AFC002421F2406244D2444249B2490561828099
:103B0C00B747024023A627210945E5B7411126C234
:103B1C0006C622C4B747024083A4C72023A60720A9
:103B2C000F10000097C0FB1FE780407E19E901458C
:103B3C00B2402244B747024023A697209244410149
:103B4C008280B737002083A7072300458297B737B9
:103B5C000020938747286367A402D843B74636FEF4
:103B6C00938606C83305A4403697E372E5FC130729
:103B7C000064B335E502922781463305E502EFA0D8
:103B8C0002587DB7D8433A94C9BF4111B7370020CA
:103B9C0006C623A0A7280295B240B737002023A25F
:103BAC00A720014541018280914763E9B700B737EF
:103BBC0000208A0593878721BE9588C18280B737FC
:103BCC00002023AC072237350020B73700204111E5
:103BDC0023A007285146B7370020814513058521BE
:103BEC0006C623A8072222C426C23734002097C059
:103BFC00FB1FE780207A1305C41E13068002814543
:103C0C0097C0FB1FE7800079EFF0CFD7B7370020C4
:103C1C0083C717251304C41E854513D527008D8B28
:103C2C003E958D473305F5029947B7340020390589
:103C3C001375F50F28A03305F5021305052497C05D
:103C4C00FB1FE780603F23AEA4262DCD3020994783
:103C5C0081453306F6021306062497C0FB1FE78046
:103C6C00607383A7C4273820B734002093870724B8
:103C7C000A0723AAF420BA9737370020232AF72201
:103C8C00EFF0AFE91D211C3083A644213736040028
:103C9C001397270036971306063310C313871700A4
:103CAC001377F70F0A073736040036971306263BAF
:103CBC0010C313873700890793F7F70F8A0718B0DB
:103CCC00B69790C3B2402244924441018280373768
:103CDC0000201307C71E1C33342363FFD700B736ED
:103CEC00002083A646211386170010B313972700D4
:103CFC00369708C33E8582809307F00FE5BF1C41C1
:103D0C00F1CF41777D8FB706002089476319D70C17
:103D1C005A2171C7411126C21946AA849305F00F86
:103D2C00610506C622C497C0FB1FE780A078054733
:103D3C008D47630FE5089C4491C7985C994749CB24
:103D4C00D85C59C73734002013060004814513058D
:103D5C00C42397C0FB1FE780E06313060004A6850D
:103D6C001305C42397C0FB1FE780205C9307C42373
:103D7C00DA2701E713070010DAA7F82719E305473C
:103D8C00F8A79A2B19E36D479AABF83719E3154747
:103D9C00F8B7B82B19E30547B8ABB83B19E3F837BC
:103DAC00B8BBD82B19E32547D8ABF82801E7130784
:103DBC00C003F8ABDC5791C78297B7370020239A22
:103DCC00A71EB73700207D57A382E764CD3B814700
:103DDC00B240224492443E854101828089473E850F
:103DEC00828001114AC8373900208327492806CE22
:103DFC0022CC26CA52C456C24EC68297130A0064FD
:103E0C00B335450313094928835A890081465686E0
:103E1C0033054503EFA0A22EB73700201387C71E2A
:103E2C00004FAA840145630694029389C71E33850B
:103E3C008440636E94000325490056868146B33551
:103E4C00AA023305AA02EFA0822B018D269523AC82
:103E5C009900F2406244D2444249B249224A924A01
:103E6C0005618280011122CC2E84B7E506000A85FB
:103E7C0041469385055506CEEFA0826118080604CD
:103E8C003A94B7370020035504FF83D7E728F24054
:103E9C006244AA9737450F00130505243355F502E4
:103EAC0005618280B737002083D7E72851471D452D
:103EBC00637CF702794719456378F70213072003EF
:103ECC0015456373F7021307B0041145637EF700C1
:103EDC00130740060D456379F70013076009094580
:103EEC006374F70013B5B70F8280011122CC06CE94
:103EFC002A842EC6EFF04FD3B245F240818D33A504
:103F0C00A502229562441375F50F0561828001119B
:103F1C0022CC06CE2A842EC6EFF00FD1B245F24049
:103F2C00818D33A5A502229562444205418105612C
:103F3C008280011122CC06CE2A842EC6EFF0CFCE81
:103F4C00B245F240818D33B5A502229562440561DC
:103F5C008280B737002023AAA7288280B737002099
:103F6C001387C723585739CF411122C426C24AC0E0
:103F7C0006C61389C7230297B73700201387C71EBD
:103F8C001A272A849384C71E05CBBA876373A700AC
:103F9C00AA87C207C183BA866373E400A286C206ED
:103FAC00C182958F51476359F7008327090391C349
:103FBC008297EF00C22D82A4B2402244924402495F
:103FCC004101828082800111B737002022CC373426
:103FDC00002023AA07289307C4239C5B06CEAA853E
:103FEC001304C42381C72AC68297B245C9C19C4118
:103FFC000545B5CBDC41A5CB9E25B5C7BE25A5C7D0
:10400C00DC2589CB5C3813F737008983BA970947CD
:10401C00634BF7043735002041461305452897C0FC
:10402C00FB1FE7808030B737002083A6472837373F
:10403C0000202328D72278380DE3938747288A2736
:10404C009307805737460F003305F50213060624F5
:10405C0081468145EFA0A20A68B8374504001305D4
:10406C00E5DE25360145F240624405618280B737B2
:10407C0000209387C71E3717002023AE07001307B5
:10408C006798B737002023A2E72837873200938739
:10409C004728FD56130727A1D4C398C723860700CA
:1040AC00B747024023A4D726BDBF011122CC373419
:1040BC0000209307C423884706CE26CA4AC801E9C4
:1040CC000545F2406244D2444249056182801304A2
:1040DC00C4231C5CF5D7585C65D770008545829766
:1040EC001844B247E30EF7FC4A249305E004B734B6
:1040FC00002097C0FB1FE78020F41387C41E08D351
:10410C009384C41E55DD52249305F00F014997C0CA
:10411C00FB1FE78020287C249050634DF9003285EA
:10412C0097C0FB1FE78040FE014523A0040223A299
:10413C00040241BF4E240844585CB387250389818F
:10414C0005093E9508C20297F9B701114EC6B73959
:10415C0000209387C9239C4726CA4AC852C406CE5E
:10416C0022CC56C25AC02A8AAE8432896388071E72
:10417C009389C92303A78903630207121307F01F4E
:10418C006360A712373400201307C41E832A07026A
:10419C001304C41E63980A0803D5C900956593855A
:1041AC0015E097C0FB1FE78020E908D02A867DC563
:1041BC0083D5C90083A7890303A5890089818297C8
:1041CC0083A78900832A04025CD089476314FA0808
:1041DC00C1476395F40C83D5C9009147938505FCC1
:1041EC00B3C5F5028A05D695B8219307A0056313CC
:1041FC00F70A9E216390470B4A852686910597C046
:10420C00FB1FE78080121C505685639157130145A4
:10421C00F2406244D2444249B249224A924A024B89
:10422C00056182805850E382E7FA03D5C900956591
:10423C00938525E097C0FB1FE78000E0AA8A39CD63
:10424C0083D5C9002A8683A7890303A589008981A0
:10425C008297A5BF8D47631BFA00C1476390F40496
:10426C0083D5C900938545FDF199B5BF9147631876
:10427C00FA006395440383D5C900A115F5B79307DC
:10428C000010631DFA00A14763EA970083D5C900AB
:10429C00C115D9BF1C505685639D570B29458DBF41
:1042AC009D6A637A5509930A05E01947B3CAEA0275
:1042BC0003D7C900373B0020B38AEA02BE9A9307A2
:1042CC00CB1EDC53130BCB1E6395570103240B023F
:1042DC001DE003D5C9009305E00497C0FB1FE780E0
:1042EC00A0D52A8445DD83D5C90083A789032A86F6
:1042FC0089815685829791451307A00589819397EB
:10430C002500A297B4236391E6049623639C46038D
:10431C0085058A052686A2954A8597C0FB1FE780EE
:10432C00C00083270B02E38487EE228597C0FB1F16
:10433C00E78080DDE9BD21677917E361A7F6B30A51
:10434C005541BDB7AC335DBF83270B02E38887F4BF
:10435C00228597C0FB1FE78020DB89B7B737002089
:10436C0083A5C72085DD91479306A0058983139704
:10437C0027002E973023E313D6F21223631C460139
:10438C0085078A072686BE954A8597C0FB1FE7805E
:10439C00C0F9B5BD3C33D9BFB73700209387C723CD
:1043AC00984721C3D85F15CF8546631CD5024111B0
:1043BC0022C4373400201304C41E105006C611CE7C
:1043CC00CE27485089810297085097C0FB1FE78081
:1043DC00A0D32320040223220402B2402244410130
:1043EC0082808280011122CC373400209307C423B1
:1043FC0056C283AA870026CA4AC84EC606CE52C4E5
:10440C002A89AE84B2891304C423638D0A1A5C5CB6
:10441C0099EB2945F2406244D2444249B249224ABE
:10442C00924A056182801C5CEDD79307F01F63E113
:10443C00A70C373A00209307CA1E9C53130ACA1EB6
:10444C00A9C7084483274A02639CA70489476313BE
:10445C00F906C147E39FF4FA4A249147130505FC7A
:10446C003345F5029317250003250A022686CE85CF
:10447C003E959307A0053CA123102501110597C07B
:10448C00FB1FE78080EA014571B74A249305E004DD
:10449C0097C0FB1FE78040BA2320AA025DF195BFAD
:1044AC004E241C5C03260A02898182971C44232219
:1044BC00FA0269BF8D47631BF900C147E39BF4F413
:1044CC004A24130545FD9377C5FF79BF91476317C0
:1044DC00F900E39024F54A242115F5B79307001051
:1044EC00E319F9F2A147E3E697F24A244115E1BF3B
:1044FC009D676375F506930705E01947B3C7E70297
:10450C005A24373A0020B387E702BE9A9307CA1E93
:10451C009C53130ACA1EB1CB83274A0263925707D6
:10452C0003250A0291461308A0059305F00F93D7B3
:10453C002600139727002A97302363120607835807
:10454C000700303363992805B306D64063C496043C
:10455C0085078A072686CE853E9515B7216779177C
:10456C00E369A7EAB307F54061BF4A249305E00469
:10457C0097C0FB1FE78040AC2320AA0251FD51BD20
:10458C004E241C5C03260A028981568582972322BD
:10459C005A0379B70EA393160601C18249BF522460
:1045AC00B38596009105130606FCE3F4C5E6138665
:1045BC003400719A1106B2962301070123102701CA
:1045CC0034B379B7373A00209307CA1E9C53130AA9
:1045DC00CA1E95CF03250A0291461308A005930520
:1045EC00F00F93D72600139727002A9730236310D8
:1045FC00060583580700303363972801B306D6406D
:10460C00E3D896F40EA393160601C182D9BF682491
:10461C005E249305E0043305F5024205418197C001
:10462C00FB1FE78060A12320AA024DF5DDB35224C5
:10463C006C24B385C502338696001106E3EBC5DC0A
:10464C00BDB7014582809C211CA1BE211CB1BE219D
:10465C00A1833CA1DC213CB111458280B7370020FD
:10466C0023AA07F4B737002023A807F482800DCDC6
:10467C00411126C206C622C4AA8401458DC12E84CE
:10468C00B7E50600228541469385055697C0FB1F6A
:10469C00E780A0C99C2005455CA49C305CB4B2406A
:1046AC00224492444101828001458280011122CC36
:1046BC0026CA06CE0947AA8432846381E5044146A2
:1046CC008147639BC500638FE6006397B6000DA816
:1046DC0041478147638EE600F2406244D2443E85F6
:1046EC00056182808A852285593741468A8519A8B9
:1046FC008A85B53F41468A85228531A0E39AB6FC6E
:10470C002E86A285268597C0FB1FE78000D3AA873B
:10471C00E1B7B737002023A8A7F48280B737002071
:10472C0023AAA7F48280011122CC622106CE26CACC
:10473C004AC84EC62DCC83298500AE842A8803C96D
:10474C000900814713178901618763550702B14737
:10475C00054563F787045114420403552800418032
:10476C0033878900A2864E868545EFB05028B33733
:10477C00A00085077D14135569004204058913793F
:10478C00F90341809CA088B023812401C2A0014779
:10479C0019C01387190098C409476383E7000145C2
:1047AC00F2406244D2444249B249056182800545D7
:1047BC00C5BFC167F917630AF502D94763F7B7029A
:1047CC00011122CC2EC606CE2A84EF90A021B24530
:1047DC006368B50022856244F24005616FA05015F4
:1047EC00F240624405450561828005458280C167BF
:1047FC00F9176314F5006F90E01E411106C6EFA087
:10480C00B00111E15D45B240410182809147639D49
:10481C00F5001C211CA23C211831A207D98F3EA205
:10482C003C3101455CA28280114582804111814559
:10483C0022C426C206C6AA84BD232A8409E9B73736
:10484C00002083A707F581C7F94526858297228525
:10485C00B240224492444101828039714ED656D2E4
:10486C005AD006DE22DC26DA4AD852D4AA8A2E8BFB
:10487C00B28951EB36C6A53F9145EF904025AA84ED
:10488C004D493DC5B246054A238034010544630AAF
:10489C000B00B68513851400029B05051314050146
:1048AC004180E20993D9894163D30902C1455685F8
:1048BC00EFA0F004654915E533868400A2852685B2
:1048CC00EFB0E0582A8911ED310442044180914740
:1048DC002C085685FC8426CEE085EFA0A01B2A89E7
:1048EC0001C963070A00268597C0FB1FE780C081BA
:1048FC00F25062544A85D2544259B259225A925AB1
:10490C00025B21618280BA84014ABDBF011122CCB5
:10491C0026CA4AC84EC606CE2A893284B689353F85
:10492C00AA840DE1B737002083A747F581CF05474F
:10493C006317E40003C4090005041374F40FA28583
:10494C004A858297F240624426854249D244B24954
:10495C0005618280AE86B745040001470546938504
:10496C0025656DB79E211CA19E21A1831CB1094513
:10497C0082809E211CA19E21A1831CB1BE213CA141
:10498C00BE21A1833CB1114582809E211CA19E2198
:10499C00A1831CB1BE213CA1BE21A1833CB1DC3161
:1049AC005CA1FC215CB18A251905420541818280FC
:1049BC009E211CA19E21A1831CB1094582809E21B0
:1049CC001CA19E21A1831CB1BE213CA1BE21A183AF
:1049DC003CB111458280CA21060542054181828085
:1049EC009E211CA19E21A1831CB1AA21090542056F
:1049FC00418182809E211CA19E21A1831CB1BE21DC
:104A0C003CA1BE21A1833CB1CA21110542054181C3
:104A1C0082809C211CA1054582809E21411122C4CB
:104A2C0006C61CA19E212E841105A183A30EF5FEA2
:104A3C00BE219505230FF5FE83D7D5FFA183A30FC8
:104A4C00F5FE03C6F5FF97C0FB1FE780008E4820DC
:104A5C00B240224411054101828089476399F500D7
:104A6C001C3118210145A207D98F1EA28280114545
:104A7C0082809A21D94763FDE702011122CC06CE30
:104A8C002EC62A84EF801076B2469E22636DF50006
:104A9C0022856244F240B7550400014709469385CC
:104AAC00059705615DBBF240624409450561828052
:104ABC0009458280914785C51421FD15C20585479E
:104ACC00C1816390F60213D725008D89914781E946
:104ADC00914711C7050534A21AA248C281473E85E9
:104AEC00828009479147E39CE6FEC94733D7F5021C
:104AFC00B3F5F502E1BFAE86B75504000147114688
:104B0C009385E59799BB93F7350089EB898191479C
:104B1C0081C50EA248C281473E8582809147EDBF78
:104B2C00D8218947631CF702011122CC2A84C8457D
:104B3C0006CEAE86014709C92EC69D4597B0FB1F10
:104B4C00E780C069B2462A8722856244F240B75595
:104B5C000400194693856599056101B30945828066
:104B6C0099E1114582801C2105473EA2E37BF7FEAB
:104B7C00FD1593F5F50F33D7F502B387E702E392F2
:104B8C00F5FE050548C21AA201458280DC210947C1
:104B9C00AE866385E70041476399E700B75504008B
:104BAC0001472146938565A24DB9094582800EA225
:104BBC0091E1014548C201458280AE86B75504009B
:104BCC00014729469385C59B49B90EA291E1014540
:104BDC0048C201458280AE86B75504000147314674
:104BEC009385A59C9DB90EA291E1014548C2014552
:104BFC008280DA21854763FFE702011122CC2A84E7
:104C0C00884106CE1DC12EC6854597B0FB1FE78097
:104C1C00E05C2A8722856244B246F240B755040014
:104C2C0039469385259E05610DB9F24062440945CC
:104C3C000561828009458280914785C518218D4682
:104C4C00914763F0E602FD15C205C181B3C6E502CA
:104C5C003308D70263970501050516A23AA248C28C
:104C6C0081473E858280DC210947AE866385E7005B
:104C7C0041476399E700B7550400014741469385C6
:104C8C0065A2E1BE09458280B335B00013952500BD
:104C9C008280011122CC26CA06CE98258547AA848B
:104CAC002E844946631FF70099363E20491513069A
:104CBC00200963C8A700F2406244D244094505614B
:104CCC008280183485476314F70013660604484045
:104CDC0001C98D4532C697B0FB1FE7802050324684
:104CEC00A2866244F2402A872685D244B755040036
:104CFC009385C59E056195B68D4763F8B7021C3147
:104D0C001821F115A207D98F1EA23C313821C205FA
:104D1C00A207C181D98F3EA24EA289C5110508C632
:104D2C000145828023240600E5BF114582800111D4
:104D3C0022CC2A84884506CEAE8601C92EC695455E
:104D4C0097B0FB1FE7808049B2462A8722856244D0
:104D5C00F240B75504005946938505A00561F5BC92
:104D6C00B335B000139525008280AE86B75504008C
:104D7C00014761469385E5A1CDB48547114563F0A4
:104D8C00D7021C320C22A207CD8F1EA39387E6FFFD
:104D9C003EA389476386F600090650C3014582800D
:104DAC0023220700E5BF014781467946814575B44A
:104DBC009E211CA19E21A1831CB109458280BC218E
:104DCC0005471CA18A216397E7000A0505054205E2
:104DDC0041818280C9473305F502CDBF8A210A057E
:104DEC00420541818280BE211CA18A21BE2133054E
:104DFC00F50205054205418182808A2182808A2143
:104E0C0082808A218280BE211CA18A21BE21330589
:104E1C00F50205054205418182809E211CA19E213F
:104E2C00A1831CB1BE213CA1BE21A1833CB1CA21EE
:104E3C0011054205418182809E211CA19E21A183E6
:104E4C001CB1AA210905420541818280894711457F
:104E5C006398F6001C3214220145A207D58F1EA3BD
:104E6C0082809A21D947AE8663F9E700B7550400D2
:104E7C0001470D469385C5DB51BC09458280114520
:104E8C00639DA6001C3214220145A207D58F1EA3D8
:104E9C003C323422A207D58F3EA38280BC21054729
:104EAC00FD1793F7F70F6361F7049E2195CF01115E
:104EBC0022CC2A84C84106CE1DC12EC6894597B086
:104ECC00FB1FE780A0312A8722856244B246F2405C
:104EDC00B755040015469385A5DC056105BCF24069
:104EEC0062440945056182800945828095471145D8
:104EFC0063F1D706411122C426C24AC006C61C3231
:104F0C00BA841822A2073284D98F9EA03C32382250
:104F1C0093054400A207D98FBEA08947DCA009469F
:104F2C0013855400368997B0FB1FE7800040930728
:104F3C00A9FF9EA49947631BF90023A60400B24065
:104F4C002244924402490145410182801904C0C4A3
:104F5C00FDB782809E2195CF011122CC2A84C841B5
:104F6C0006CE1DC12EC6854597B0FB1FE7800027D6
:104F7C002A8722856244B246F240B75504001D468A
:104F8C00938585DE056159B2F2406244094505619D
:104F9C008280094582809947639DF60289474111B9
:104FAC0006C65CA31C321422B285A207D58F1EA3A1
:104FBC003C3234225023A207D58F130557003EA351
:104FCC00910597B0FB1FE7804036B2400145410187
:104FDC008280D14711456394F600C147C9B78280DE
:104FEC009E219DCF011122CC2A84C84106CE05C535
:104FFC002EC6894597B0FB1FE780401E2A87228565
:10500C006244B246F240B75504002546938525DF2D
:10501C0005616FF0BF8FF2406244094505618280E3
:10502C0009458280894711456398F6001C32142289
:10503C000145A207D58F1EA38280011122CC2A84A0
:10504C00C84106CEAE86014709C92EC6854597B024
:10505C00FB1FE780A018B2462A8722856244F240E3
:10506C00B75504002D46938565E005616FF01F8AE6
:10507C001145639DA6001C3214220145A207D58F51
:10508C001EA33C323422A207D58F3EA3828001118D
:10509C0022CC2A84C84106CEAE8601C92EC68545CF
:1050AC0097B0FB1FE7808013B2462A8722856244A3
:1050BC00F240B755040035469385A5E005616FF0C5
:1050CC00FF8493F71600114581EB89476386F60040
:1050DC00858256A310C301458280011122CC2A84FB
:1050EC00C84106CE05C52EC6854597B0FB1FE78087
:1050FC00E00E2A8722856244B246F240B75504007E
:10510C003D469385E5E005616FF05F80F2406244B7
:10511C000945056182809E219DCF011122CC2A84F4
:10512C00C84106CE05C52EC6894597B0FB1FE78042
:10513C00E00A2A8722856244B246F240B755040041
:10514C004546938525E105616FF04FFCF2406244C2
:10515C0009450561828009458280854763F6D7023F
:10516C0008A70CB71C320C22A207CD8F1EA3938765
:10517C00E6FF3EA389476386F600090650C3014546
:10518C00828023220700E5BF1145828001478146BA
:10519C004D4681456FF08FF78D47114563F4D7026B
:1051AC001C320C22A207CD8F1EA33C322C22A2074C
:1051BC00CD8F3EA39387C6FF5EA36386A600110620
:1051CC0010C70145828023240700E5BF011122CCC2
:1051DC002A84884506CEAE8601C92EC6954597B061
:1051EC00FB1FE780A0FFB2462A8722856244F2406B
:1051FC00B75504005D46938565E205616FF00FF1CC
:10520C00854711456395F6001C2201451CA382803D
:10521C0001478146654681456FF04FEF011122CC65
:10522C002A84C84106CEAE86014709C92EC68D45D3
:10523C0097B0FB1FE78080FAB2462A87228562442A
:10524C00F240B75504006D46938545E405616FF057
:10525C00CFE0011122CC2A84C84106CEAE8601478C
:10526C0009C92EC68D4597B0FB1FE78020F7B246C3
:10527C002A8722856244F240B7550400754693850F
:10528C0045E405616FF06FDD011106CE2EC6EF907F
:10529C00D05419C5B245F2402A2105616FE00015C2
:1052AC00F240494505618280B7370020A38007F89A
:1052BC00B7370020238007F8B737002023A407F660
:1052CC00B737002023A607F6B737002023A807F628
:1052DC00B737002023AA07F6B737002023A207F61A
:1052EC00B737002023A007F6B7370020239C072AE6
:1052FC00930640389387872BB6B3F1761307400B90
:10530C00938606B8BAA3D6B311679D46130600055B
:10531C009305000A1305007DDAA3F6B341478546D1
:10532C00130810F8BAA7DAA7BAABDAABFAAB9AAF94
:10533C009AB7EEA38EA7F2A792ABAAAF239E070053
:10534C00239F070023900702B6B7239607032397E2
:10535C0007029308F007239807022392E70423938C
:10536C00E704239FE7042390E7062391E7062392A3
:10537C00E706239917031307C01CD6BBF6BB239C67
:10538C000702239D0702239E0702239F07022390F7
:10539C0007042391D7042394070423950704239629
:1053AC00D7042397C7042398C7042399A704239AE7
:1053BC000704239B0704239C0704239DC704239EF7
:1053CC00C7042393A7062394070623950706239661
:1053DC0007062397B7062398B70623990706239A3F
:1053EC00E7065147239DE7067D57239B0706239C21
:1053FC000706239ED706239F0706239007082391B1
:10540C000708239207092393E7088280011126CA13
:10541C00AA84214522CC06CE2E8432C636C43AC28A
:10542C0097B0FB1FE780A0E00DC5A246124732469D
:10543C00930700FD1CA1994704B13CA174A178B15C
:10544C0052A1AA8522856244F240D24405616FD0F4
:10545C00BFE3F2406244D24405618280B73700203A
:10546C0023A4A7F68280B737002023A6A7F6828054
:10547C00B737002023A8A7F68280B737002023AACD
:10548C00A7F68280011122CC4AC806CE26CA2A89E8
:10549C000144B30489006368B400F2406244D2440E
:1054AC004249056182802EC6EFD01FF89317050183
:1054BC00C183A183B2459CA09307140093F7F70F07
:1054CC00850463F8B700CA97090488A31374F40F12
:1054DC00C9B73E84C9B7411122C437340020130424
:1054EC0084296A20C16706C6FD17630EF500B7371D
:1054FC00002003C6C73FB7350020938585F7EF9092
:10550C00F00FFD577EA0B24022444101828009C9B0
:10551C0025151375F50F1335850E1345150082806F
:10552C000145828023900500C1C6797122D426D210
:10553C004ECE52CC5AC806D64AD056CA5EC636840F
:10554C00328AAE892A8B814463F24407B3079400F4
:10555C009C23138914004209939A070193DA0A01D8
:10556C001359090163840A04CA976341FA04B30707
:10557C00240183CB07005E85593F0DC99387FAFF41
:10558C002390F90063906B03130519002295B25018
:10559C00225492540259F249624AD24A424BB24BBB
:1055AC0045618280D694C204C18079BF0145C5B7DC
:1055BC0001458280011122CC3734002026CA4AC80A
:1055CC004EC69307842906CE2E89D0CB8CCBC8C768
:1055DC00AA8441469305F00F4A8597B0FB1FE780DC
:1055EC0060ED854913048429631935030848C145C6
:1055FC00513D41469305F00F268597B0FB1FE78080
:10560C0060EB05496315250348446244F240D244DB
:10561C004249B249C1450561B5B5414681454A8506
:10562C0097B0FB1FE78000E9E31535FDC1B7414694
:10563C008145268597B0FB1FE780C0E7E30625FD73
:10564C00F2406244D2444249B24905618280411120
:10565C0022C43734002026C24AC0AE842A891306DD
:10566C00000281451305842906C697B0FB1FE7800D
:10567C0060D293078429A3812701B73700202380A8
:10568C009740EFD0F058854719C181474945230C05
:10569C00F428B2402244924402494101828081475D
:1056AC0091C909C985476319F500DC3193E707FCFB
:1056BC00DCB185473E85828089476316F500DC3175
:1056CC0093F7F703F5B70D478547E315E5FED8319A
:1056DC001377F70313670704D8B1E9BF814785C176
:1056EC0019CDD8319306000C85471377070C630846
:1056FC00D700930600048D476303D70089473E8586
:10570C008280411122C4005D06C626C21DC8AA842F
:10571C00085009C597B0FB1FE780009F485009C58A
:10572C0097B0FB1FE780409E085409C597B0FB1F3C
:10573C00E780809D228597B0FB1FE780E09C23AC1F
:10574C000402B240224492444101828019E9B737E5
:10575C00002083C7A72991C737350020130585F58D
:10576C008280373500201305052B8280B737002047
:10577C0003C5A7298280B737002003A5472A82805A
:10578C00B737002003A5872A8280B737002083A76C
:10579C00C72A88438280B737002093878729D44B48
:1057AC009842050798C2A8339307F00F6305F500DC
:1057BC0091656FD09FE18280011122CC06CE2E84A0
:1057CC0032C6EF9030129147B2456310F502B737ED
:1057DC00002083A747F795C303A30700630F0300BB
:1057EC0022856244F24005610283B737002083A70B
:1057FC00C7F681C703A34700D5B7F24062440545FD
:10580C0005618280011122CC2A844A2106CE26CA47
:10581C004AC84EC697B0FB1FE78040272DC52A8982
:10582C0004218349C500F13D4A85EF90F0494A2097
:10583C00EF90900637390020130909F883470900C7
:10584C00B9C763969704B737002083C517F8268528
:10585C00253C19E1230009004A20EF90B00891473C
:10586C00631CF500B7370020938787295620FA234D
:10587C006394E6007D57FAA3F2406244D244424955
:10588C00B2490561828081499304F00F65B7930793
:10589C00F00FE383F4FC7420522028204E87A68559
:1058AC00B5365DBF79715EC6AA8B2E8552CC56CAB1
:1058BC005AC806D622D426D24AD04ECEAE8A328BC5
:1058CC00368A97B0FB1FE780601C7DC1045D2A8976
:1058DC00E5C09C50614599C3130540039C5481C796
:1058EC0051054205418163050A007105420541815C
:1058FC00DC5081C75D054205418197B0FB1FE780F5
:10590C0000932A8455C56146814597B0FB1FE780FB
:10591C0060A8B737002083C9872E63940900834998
:10592C000900930700FD1CA0A947A30074013CA02B
:10593C00230364018C50231254011305840191C973
:10594C0008C47146930A440397B0FB1FE780E09D9F
:10595C0056858C5491C948C45146930A450197B059
:10596C00FB1FE780809C5685630C0A0008C87146B3
:10597C00D285930AC50197B0FB1FE780009B568523
:10598C00CC5099C548C85D4697B0FB1FE780E0999D
:10599C00A2854E85EFD05F8F2254B2509254F249BB
:1059AC00624AD24A424BB24B4A850259456191BB7D
:1059BC00B250225492540259F249624AD24A424B92
:1059CC00B24B4561828001114EC6AA892E854AC808
:1059DC0006CE22CC26CA2E8997B0FB1FE780000B7F
:1059EC0039C5B737002083C4872E91E004211945AF
:1059FC0097B0FB1FE780A0832A8415C981451946FF
:105A0C0097B0FB1FE7800099930700FD1CA0B947D6
:105A1C00A30034013CA023122401A2856244F2406D
:105A2C004249B2492685D24405616FD0FF85F240C8
:105A3C006244D2444249B2490561828039715ECEDA
:105A4C00AA8B2E8526DA4ED652D456D25AD006DEE2
:105A5C0022DC4AD8AE84328BB68A3A8ABE8942C6D8
:105A6C0097B0FB1FE780800239C92A89414597A06E
:105A7C00FB1FE780C07B2A8439C14146814597B022
:105A8C00FB1FE7802091B737002003C5872E19E153
:105A9C0003450900930700FD1CA0BD473CA0B2477D
:105AAC00A300740146A023046401A304540123053C
:105ABC004401A30534015CC4A285EFD0EFFCF25085
:105ACC006254D2544259B259225A925A025BF24B46
:105ADC0021618280797126D2AA8439454AD04ECE72
:105AEC0006D622D42EC6B289368997A0FB1FE78032
:105AFC0000740DCDB2459307000D1EA1B1472A8449
:105B0C004EA13CA1CE851905194697B0FB1FE78025
:105B1C00C08123062401A2852254B2500259F249B5
:105B2C0013F5F40F925445616FD00FF6B250225416
:105B3C0092540259F24945618280411126C2B73410
:105B4C00002093848429B83006C622C44AC0930727
:105B5C00F00F6308F7042A89394597A0FB1FE780EB
:105B6C00006D2A841DCD930700FDB73500201CA1C4
:105B7C00A3002501230105009385052B0D0519466E
:105B8C0097A0FB1FE780607A9E24A285A8303EA4D4
:105B9C009C305CA42244B2409244024941016FD033
:105BAC00AFEEB2402244924402494101828001117D
:105BBC005AC02A8B314526CA4EC652C456C206CE8E
:105BCC0022CC4AC8AE84B28A368ABA8997A0FB1F07
:105BDC00E780E0652DCD2A84268597B0FB1FE780F2
:105BEC00E0EA09C55825A1476311F704B73700202F
:105BFC0003C9B729930700FD1CA09D47A3006401AE
:105C0C003CA046A023135401231444012315340152
:105C1C00A2856244F240D244B249224A924A024BD3
:105C2C004A85424905616FD02FE6B737002003C97A
:105C3C001740E3110BFCB737002083A707049C47E0
:105C4C00D5DBCE865286D6852685829765B7F240FF
:105C5C006244D2444249B249224A924A024B0561FB
:105C6C008280011122CC2A84214506CE2EC697A013
:105C7C00FB1FE780C05B15C5B245930700FD1CA157
:105C8C00C5473CA1BC313CB1DE215EA1FC217CA10D
:105C9C00FC31AA857CB122856244F24005616FD04B
:105CAC00AFDEF24062440561828041114AC02A890C
:105CBC00714526C206C622C4AE8497A0FB1FE7809E
:105CCC0000573DC5930700FD1CA1F5473CA1BC3016
:105CDC002A849385C4003CB1DE2031051946231C6F
:105CEC00F5FEFE20231DF5FE9E24231EF5FEBC248E
:105CFC00230FF5FEBC34A30FF5FE97A0FB1FE78026
:105D0C00C062BC28A2854A853CA8DE285EA8FC2877
:105D1C007CA8FC387CB89C2C1CAC9C3C1CBCBC2CC3
:105D2C003CAC2244B2409244024941016FD0CFD5E1
:105D3C00B2402244924402494101828001114AC876
:105D4C002A89614526CA4EC606CE22CCAE89B284BB
:105D5C0097A0FB1FE780A04D25C1930700FD1CA158
:105D6C00BC302A84938584001CB195473CA1FC303F
:105D7C0011051946A30FF5FE97A0FB1FE780E05A0B
:105D8C00DE2023063401A2853EA4BE2C4A857EA4C7
:105D9C00DE2C1EA8FE2C3EA883C704025CA883C779
:105DAC0014025CB8BE30F240D2447EA86244424930
:105DBC00B24905616FD04FCDF2406244D2444249A2
:105DCC00B24905618280411122C43734002013048A
:105DDC0084293C2006C626C285CBB7340020AA8570
:105DEC001946138584F597A0FB1FE78000542820E3
:105DFC00938584F5EFF0BF8A2244B240138584F575
:105E0C00924441016FD08061B240224492440145DA
:105E1C0041018280411126C2B73400209387842926
:105E2C0006C622C44AC0B8339307F00F9384842962
:105E3C006301F7042A89294597A0FB1FE780203FBF
:105E4C002A8405C9930700FD1CA1A147A3002501C5
:105E5C003CA1BC20B7350020938585F53CB1194693
:105E6C00110597A0FB1FE780404CA830A285EFD00E
:105E7C00AFC1B8208D476311F702B737002083A755
:105E8C0007F799CB03A38700630803002244B240B1
:105E9C009244024941010283B24022449244024995
:105EAC0041018280797122D406D626D24AD04ECEB8
:105EBC0052CC56CA09444DCD2A890A21AE89514487
:105ECC0097B0FB1FE78080BCAA845DC137370020E8
:105EDC009307C73FDC238546BA8AFD1793F7F70F64
:105EEC00494463F7F6085825A1476314F7006391FA
:105EFC0009089C5C4544ADEF91659385457113058C
:105F0C00C00297A0FB1FE780201388DC2A8A4D442F
:105F1C0025C11306C002814597A0FB1FE78080476F
:105F2C008357090093064A0036852311FA007146FF
:105F3C009305490036C697A0FB1FE780003F8947B1
:105F4C002300FA00C824B2460356090083C5CA3F91
:105F5C00611513351500EFA0201D2A8463860900F6
:105F6C00CE852685EF90300401C42685EFF06FF9BD
:105F7C002285B250225492540259F249624AD24AB2
:105F8C0045618280B737002083C707400547FD175E
:105F9C0093F7F70F6377F708894749C6011122CCAD
:105FAC0026CA4AC84EC652C406CEAA89368AB284BC
:105FBC002E8997B0FB1FE78060AD2A84D14731C58D
:105FCC00485509C597A0FB1FE7800014F1452685AD
:105FDC0097A0FB1FE780A04148D4CD471DC5542492
:105FEC0021478147639DE600630B0A00382D122977
:105FFC0093062501AA854E85EF905001AA8758205B
:10600C00630E09001367670058A0F2406244D24443
:10601C004249B249224A3E85056182801367470096
:10602C00E5B7C9473E8582809307200463EAA70041
:10603C00B73700209387872B06053E950A2182806F
:10604C0041657D158280011122CC2A842E8526CAB9
:10605C0006CEAE8497B0FB1FE78040A30DCDB747AB
:10606C000F009387F723094563E2870281450A8570
:10607C00414697A0FB1FE780E031A68560800A852A
:10608C0041804081A3010100EF90D06AF24062444C
:10609C00D244056182804945D5BFB7370020238F94
:1060AC00A73E82806FA0A002797152CC2A8A3285D9
:1060BC0022D426D24AD04ECE56CA5AC85EC606D66E
:1060CC0062C4AE8BB28A368BBA843E89C28946844E
:1060DC0097B0FB1FE780809B0DC92A8C63130A02C3
:1060EC0013774B005C2115CF93E727012302FC00AB
:1060FC008DEC631C0902639A090205E8ED9B2302EF
:10610C00FC00832B8C0363910B08B25022549254E5
:10611C000259F249624AD24A424BB24B224C456177
:10612C008280F59B93E70701D1B793E747002302E1
:10613C00FC0001CC1C484146A2852324FC0213051B
:10614C008C0197A0FB1FE780401E63930B02D5D8F0
:10615C000325CC0209C597A0FB1FE780E0FAF145A7
:10616C00268597A0FB1FE78080282326AC0251BF11
:10617C00E30909F80325CC0209C597A0FB1FE780AA
:10618C00A0F8F1454A85F1BF9DC483A70B0299EB9A
:10619C00916593853571714597A0FB1FE780C0E928
:1061AC0023A0AB0203A50B0219C57146A68597A0C7
:1061BC00FB1FE78080176388090283A74B0299EBCA
:1061CC009165938525715D4597A0FB1FE780C0E61F
:1061DC0023A2AB0203A54B0219C55D46CE8597A041
:1061EC00FB1FE78080141DC483A78B0299EB91657C
:1061FC0093851571514597A0FB1FE780E0E323A41D
:10620C00AB0203A58B0219C55146A28597A0FB1FB3
:10621C00E780A0112254B2509254F249B24B224C56
:10622C00CA865A860259424BD6855285D24A624A50
:10623C0045616FF02FE7011126CA52C406CE22CC5D
:10624C004AC84EC62A8AAE8497B0FB1FE7800084EA
:10625C0035C1AA89394597A0FB1FE78040FD2A84E8
:10626C0031C9B737002003C9872E6314090003C94D
:10627C0009009307000D1EA0AD473CA09385690053
:10628C0013053400194697A0FB1FE780000A93F70B
:10629C001400858085885CA444B423154401A28530
:1062AC006244F240D244B249224A4A8542490561CD
:1062BC006FC09FFDF2406244D2444249B249224A27
:1062CC000561828001114EC652C456C206CE22CC44
:1062DC0026CA4AC8AA8A2E8AB28997A0FB1FE780D1
:1062EC00E07A2DCD2A891305C00297A0FB1FE78009
:1062FC0000F42A8425C5B737002083C4872E99E083
:10630C00834409009307000D1EA0E9473CA09305A8
:10631C00690013053400194697A0FB1FE780E000C5
:10632C00D285231554011305C400414697A0FB1FC9
:10633C00E780A0FFCE851305C401414697A0FB1F43
:10634C00E780A0FEA2856244F2404249B249224A4B
:10635C00924A2685D24405616FC01FF3F240624415
:10636C00D2444249B249224A924A05618280411183
:10637C0022C437340020130404F6084006C619C59D
:10638C0097A0FB1FE78040D823200400B240224492
:10639C0041018280011106CE22CC26CA4AC82EC6E3
:1063AC0097A0FB1FE780806E31CDB245B737002038
:1063BC0003C9872E0CD5AA84631409000349050070
:1063CC00414597A0FB1FE78080E62A8405CD930703
:1063DC00000D1EA1A5473CA1DC309385640011057E
:1063EC00A30FF5FE194697A0FB1FE78000F49C5401
:1063FC00A285F2405CC46244D2444A85424905619C
:10640C006FC09FE8F2406244D244424905618280E9
:10641C001D71A2CC86CE2A842EC697A0FB1FE780C6
:10642C00E06615C954251147AA8749456391E602D0
:10643C009C5FB24591C3EC2BB71605002308B10045
:10644C009386E6FE100889452285EF90E02CF640F5
:10645C006644256182805145DDBFB737002083C774
:10646C0007400547FD1793F7F70F637AF704894741
:10647C0021CA411122C426C24AC006C6B2842E8942
:10648C0097A0FB1FE78080602A84D14715C1630663
:10649C0009005C2193E727005CA14146A685130502
:1064AC00840197A0FB1FE78040E89C481CD48147DF
:1064BC00B2402244924402493E8541018280C94740
:1064CC003E858280797122D406D62A842EC697A066
:1064DC00FB1FE780A05B01CDB2452285230EB100E6
:1064EC006C08EF90E028B2502254456182805145EF
:1064FC00DDBF6F801034C1671387E7FF6395E5023A
:10650C00B737002083A7C7F691EB494582804945F0
:10651C00B2402244924402494101828003A3070005
:10652C00E30503FE0283411122C426C24AC006C6FB
:10653C00FD172A892E84B284639AF502B73700209E
:10654C0083A7C7F691CF9C4381CF829711E9B737C8
:10655C000020238027F9B7370020A38097F84DBF80
:10656C00A6854A85EFE05FD245F5D5B72E8597A075
:10657C00FB1FE780A05141DD1C210D45E39A27F953
:10658C0022852244B2400249A685924441016FC043
:10659C00F0659307200463E1A7064111C16722C48B
:1065AC0006C626C2FD172A8409456381F502C54734
:1065BC00AE846312F4022E85EFC0D06A373500200A
:1065CC001305852B06042A9406A00145B2402244EB
:1065DC009244410182809307A0036316F4002E8538
:1065EC00EFC09061E1BF9307B003E319F4FC13F51E
:1065FC00F50FEFC0B060D9B709458280011106CE06
:10660C002AC6EFE07FCAEF20C06DEF10F012EF70DA
:10661C004225B737002093878729130700F0BAA3C8
:10662C0023820700B737002032451387C73FFD563A
:10663C0034A3F240238EA73E954505616F70C0438D
:10664C007571939705014AC106C722C526C3CEDED4
:10665C00D2DCD6DADAD8DED6E2D4E6D2EAD0EECE86
:10666C00C1872E8963D30754B734002003C5C43FB8
:10667C00B7390020373B002097A0FB1FE78080C074
:10668C002A8426CCB73A0020B73B0020373D0020A7
:10669C0093848929B73C00201DE021653345A9006E
:1066AC00BA402A449A440A49F659665AD65A465B65
:1066BC00B65B265C965C065DF64D496182801C20BB
:1066CC001307200A639BE70003CA34002A20C16524
:1066DC002286FD15EFF04F8EA1AA62471307C73F24
:1066EC00034A270013071009639FE7141C30154752
:1066FC006391E7022285EFF0EF902285EFC0FFB3A4
:10670C00E24703C5C73F97A0FB1FE780A0B72A84C9
:10671C0061B739476391E7164A208567A50763156A
:10672C00F5040C4403CC0500631D0C00850591C9D0
:10673C003735002019461305052B97A0FB1FE78062
:10674C00C0BE03C789298547631FF70E63080C0079
:10675C00238C09286285EFF04FBE45B78947238CFF
:10676C00F928EFC0704B51BF896713872700631856
:10677C00E504032C840063080C0C83470C0099EB94
:10678C0083472C0003471C00A207D98F9EA4834784
:10679C003C009CB003C7892989476316F70A8347D5
:1067AC000C0091C7238C092803450C006DB78C3065
:1067BC008A248D47238CF928EF70C02EF5B79507E6
:1067CC006317F5001C448823EFF0CFE43DB7F9774D
:1067DC001387A7FF2A9742074183914663F1E6048A
:1067EC009387A7FCAA97C207C18371476371F7020D
:1067FC0089671387B7006310E50483A78AF6E38ED5
:10680C0007EE9C43A285E38A07EE829715A0370713
:10681C0000181307F770B357F700858BB9C7832798
:10682C000BF7E38C07EC9C43E38907EC22858297FA
:10683C00E31505EC09A81387C700631FE5001C448A
:10684C009C23E38C07EA9307F00FE308FAEAA2858E
:10685C005285EFC07FA36DB5B9076318F50083A708
:10686C00CCF6E38C07E8DC4371BF89679387170488
:10687C00E305F5F8C9BF3D476397E7044A208967EC
:10688C001387D700E30DE5FC13879701E309E5FCBB
:10689C00CD07E31AF5FAFA20C167FD17631DF7005F
:1068AC0083A7CCF6E38B07E4DC43E38807E40965B4
:1068BC00A2854D0599BFB737002083A747F7E38E14
:1068CC0007E29C43DDB71307E003E39EE7F63C20A9
:1068DC000547639BE7107C2037370020930D07F6A4
:1068EC006397070E83A70D00E5C303CC0700214A6D
:1068FC00683013078400BA853ACEEFE03FDE68B00B
:10690C00130640028145681097A0FB1FE78080A802
:10691C003C3072471946A307F1027C30BA854818FF
:10692C00A309F10297A0FB1FE78020A05E20701046
:10693C00D2852318F1027E2462852313F1041E28CC
:10694C002314F1043E282315F1045C282306F104DA
:10695C00FD57A306F104FD572317F104EFF00FBE0A
:10696C003C3072478DE3DD47835804010358E40043
:10697C0074304E203EC23E283EC00546D28762850A
:10698C00EF80300D28B083A70D0081C71145EFF0C3
:10699C001F9E03C50BF8138C0BF8E30005D683453B
:1069AC001DF8EFE07F8EE30A05D434309307100313
:1069BC006389F600522083450C0052873685EFE040
:1069CC00FFA423000C0015BB03CC34000DB78327A8
:1069DC000BF703CC3400114A81DFDC43E38A07F068
:1069EC0081450145829729B7130790026390E70808
:1069FC007C2037370020930D07F6A9E783A70D00FD
:106A0C009DCF03CC0700214A683093772500B9C786
:106A1C0005891307440168B02286D28562853ACE77
:106A2C00EFF0CFB13C307247B9FFDD478358C4015A
:106A3C000358A40174304E203EC27E2C35BF03CCCB
:106A4C003400D1B783270BF703CC3400114ACDDFC8
:106A5C00DC43DDDB8145014582977DB7130784005C
:106A6C00BA853ACEEFE09FC7724775B70947639C6A
:106A7C00E70083A78AF6E38207C8DC43E38F07C6E7
:106A8C00228582979DB92D476398E70083A78AF6E4
:106A9C00E38507C69C47DDB70D476396E700228662
:106AAC008D454A2005B91947639CE7049305A1025B
:106ABC0013051031EF60D2626C1013052031EF60BA
:106ACC00326272208357C1024A2063E7C700162442
:106ADC000357A10263F7E60093050002EFC090177D
:106AEC0029B96373E6007AA063F3D7001EA45A2475
:106AFC00362412246E2001488147EFC07015F5BE74
:106B0C001D47E382E7D431476395E7002286B14500
:106B1C0049BF35476398E70083A78AF6E38F07BC24
:106B2C00DC47A9BF130740026396E7002285EF00FC
:106B3C00407EE1B6130750026398E70083A78AF6FC
:106B4C00E38D07BA9C4B1DBF41476396E700228536
:106B5C00EF0090065DB645476396E7000145EF00F0
:106B6C00701561BE4947639DE70083270BF7E38CE3
:106B7C0007CCDC43E38907CC814505458297E1B11D
:106B8C004D47639CE70083270BF7E38E07CADC4372
:106B9C00E38B07CAA2850945D5B713076002E394B6
:106BAC00E7CA228693056002EDBD93F7150089CFE5
:106BBC00B737002083A787F689C7DC4399C3014503
:106BCC00829713451900E9BC93F7250091CFB7378D
:106BDC00002083A707F791C7DC4381C78145054592
:106BEC008297134529006DBC93F745000145E38955
:106BFC0007AAB737002083A747F6373400201304C1
:106C0C00842989CF85475CA0B737002083A707F775
:106C1C0091C7DC4381C781450545829748446C1078
:106C2C00EF90E01D6810EFF00F9AB737002083D774
:106C3C00A72D81CF130600643386C702B737002017
:106C4C0003C5C73F9145EFC03FB61345490089BC0A
:106C5C00011122CC2A84554506CE26CAEFF0CFBCB2
:106C6C00AA8413054002EFF02FBC2AC6130550026C
:106C7C00EFF08FBBAA86228562443246F240B335D0
:106C8C009000D24405616FC0D004397122DC06DE5D
:106C9C008D472E84631AF500BA259625F2212830EB
:106CAC00CE21EFE0DFF001A889671387D700631DC1
:106CBC00E504BC2199E78547F25062543E85216179
:106CCC00828037340020832504F6F5D5DC87BC316F
:106CDC00480819469105A309F1009790FB1FE7801E
:106CEC00C064930700F03ED6832704F623180100F6
:106CFC002313010202D4882370008145EFF00F8426
:106D0C000545EFF0CFE645BF1387E700E305E5FA4D
:106D1C00138737016319E500A82151DD014781462E
:106D2C0001468145BDBFE507E307F5F8B147631997
:106D3C00F500B737002003C5B729EFE09FF2A5BFD8
:106D4C00930760026319F500B737002003C5B72914
:106D5C00EFE0BFF58DB741677D178147E31EE5F482
:106D6C00D831C947E319F7F4F625D2250A24AE2504
:106D7C00EFC0C07D2DC55D45EFF00FAB3335A000E6
:106D8C0068844C202A203000EF80A0083C8485F7D2
:106D9C009305A10013051031EF6092346C001305BC
:106DAC002031EF60F2333C851A246373F7001EA484
:106DBC003C863A2463F3E7003EA41E243A24637312
:106DCC00F7003EA42A20EF30411B7A2456243224AB
:106DDC000E242A2001488147EFC08065E9BD854714
:106DEC007C8445B7B73700201387C73F743313072C
:106DFC00F00F638FE6062DCD411122C426C24AC086
:106E0C0006C6AA8468251389C73F51059790FB1FB6
:106E1C00E780E0412A8439C59307000D1EA1D947AC
:106E2C003CA1DE205EA1FC207CA1FC307CB19C242A
:106E3C001CA5DC345CB5F02470A515C28C4851053A
:106E4C0008C89790FB1FE780404EA285224403455B
:106E5C007900B2409244024941016FC0EFC223282D
:106E6C000500E5B7B24022449244024941018280B8
:106E7C008280C1671387E7FF639DE500B737002069
:106E8C0083A707F695C39C230D47639DA7006FC08E
:106E9C006059FD1749476397F500B737002083A762
:106EAC0007F6F5F73A8582804947EDBF397122DC48
:106EBC0006DE26DA4AD84ED652D456D25AD05ECEF8
:106ECC0062CC182185472A846309F70410259306A0
:106EDC0095009305E1000545EFE0CFE4814711C132
:106EEC001C21142011476382E60437370020032746
:106EFC0047F88D461833630AD70285CB1DC70DE1C1
:106F0C000145F2506254D2544259B259225A925A03
:106F1C00025BF24B624C2161828081470145D1B703
:106F2C008546631ED7088D8BE1DF0830130A2400D9
:106F3C00D285EFE0AFFA3739002008B0832789F803
:106F4C002A8B130989F88149C1C3B73A00209304ED
:106F5C00F00F83C72AF8138C2AF863FAF902032579
:106F6C000900939B49005E951C21638197061C3197
:106F7C00639E67051946D28509059790FB1FE7802C
:106F8C00C04B29C5832409001820DE94B1E41420D9
:106F9C009147E387F6F683270900BDD303460C001F
:106FAC0001479305F00FE30DE6F4BE84C10703C55A
:106FBC0007FF6301B50C05071377F70FEDB789468B
:106FCC00E310D7F4858B8DB7054525BF850993F95B
:106FDC00F90F41B788C4C9A891476312F706C84492
:106FEC000DC11C241021630EF60418209147631860
:106FFC00F706C84419C59790FB1FE780E01023A63D
:10700C000400082491659385E57105059790FB1F95
:10701C00E78080020DC118209147631BF704C8C498
:10702C001C24930594000505A30FF5FE10249790DE
:10703C00FB1FE780802F08243335A000D9B5884486
:10704C0045B79305940005059790FB1FE780E03E3C
:10705C008547E31CF5F85545EFE01FFDADA08844CE
:10706C004DD19790FB1FE780200A23A4040051BF49
:10707C0088C47DB794A01C30D285138524009CB0A5
:10708C0019469790FB1FE780402A08249165938549
:10709C00F57105059790FB1FE78000FA0DC11820CC
:1070AC009147E319F7F2C8C41C2493059400050515
:1070BC00A30FF5FE10249790FB1FE78000271C24DC
:1070CC0081F708207D151335150025BD397122DC9B
:1070DC0026DA4ED652D406DE4AD856D25AD05ECED6
:1070EC002A84930925000831CE85B7340020EFE0BF
:1070FC00EFDE08B0938444F89C400D472A8A9C33F9
:10710C006390E70437390020832789F8814A1309F3
:10711C0089F863810714B73B002003C72BF89397BA
:10712C000A01C18303250900138B2BF863E0E70CDC
:10713C0083460B000327090081471306F00FBDAAF5
:10714C00F1D3144C70389305E1000545EFE08FBD89
:10715C0015C9984085461C2118336310D7028D8BB6
:10716C00D5F30145F2506254D2544259B259225AC5
:10717C00925A025BF24B216182808946858BE31324
:10718C00D7F8F9BF1C2011476385E7002D47E39A18
:10719C00E7FCB734002083A784F8938484F8F1D3F8
:1071AC00814A0149B73B002005A88840139B4A003F
:1071BC001C205A9518216310F7021C31639D47015E
:1071CC001946CE8509059790FB1FE780002701C55E
:1071DC0003A904005A99850A03C72BF893970A014F
:1071EC00C183E3E4E7FCE31F09F0A5BF93944A00D5
:1071FC00269518211C206318F70A1C316395470B40
:10720C001946CE8509059790FB1FE780002341CDD9
:10721C00832709001147BE941C206385E7002D4786
:10722C00639CE70203AAC4007C3803460A00630887
:10723C00F60252859790FB1FE78000ED6838916548
:10724C009385E57105059790FB1FE780E0DE1DE552
:10725C00E38004EE054539B703AA8400F1B70C4C62
:10726C0013051A009790FB1FE780201D8547E3123A
:10727C00F5FC5545EFE05FDB61DDE5B51C20114702
:10728C006385E7002D47639EE700C8C47C3805057D
:10729C00A30FF5FE70380C4C9790FB1FE780E008AD
:1072AC0045BF88C4E5B7850A8DBDBA8441078345BF
:1072BC0007FF638AC5008507C207C183E3E7D7FED2
:1072CC0051BF88C425A81C20CE85138524009CA002
:1072DC001C3019469CB09790FB1FE780000568385E
:1072EC0091659385F57105059790FB1FE780C0D4D8
:1072FC0035D118209147E316F7FCC8C47C38050536
:10730C00A30FF5FE70380C4C9790FB1FE780E00143
:10731C0091B701114AC8373900201309C93F0347F7
:10732C00790006CE22CC26CA4EC69307F00F630E08
:10733C00F70625CDAA8461459790FB1FE78020EFC7
:10734C002A8425C59307000D1EA1D5473CA1BC304E
:10735C0093898400CE853CB1DE205EA1FC207CA10B
:10736C00E830EFE0AFB768B0CE851305840019465E
:10737C009790FB1FE78060FBFC24A28503457900F6
:10738C007CA49E281EA8BC283CA8BC383CB8DC2891
:10739C005CA8DC385CB8FC287CA86244F240D2447F
:1073AC004249B24905616FB03FEEF2406244D244AB
:1073BC004249B24905618280411122C43734002010
:1073CC001304C43F783006C626C29307F00F630936
:1073DC00F7021DC5AA8419459790FB1FE78020E58D
:1073EC00AA8519CD9307000D1EA1DD473CA1DE2017
:1073FC00B24092445EA16830224441016FB0DFE894
:10740C00B2402244924441018280011122CC373493
:10741C000020832784F806CE26CA4AC84EC652C41A
:10742C008DC3130484F82E8AAA8401490840631280
:10743C009902630C0A049790FB1FE780E0CC232091
:10744C000400F2406244D2444249B249224A0561E6
:10745C00828093194900B3073501884709C9979071
:10746C00FB1FE78060CA1C40CE9723A407001C407A
:10747C00CE97C84709C99790FB1FE780E0C81C400E
:10748C00BE9923A60900050955B745DD139644009E
:10749C0081459790FB1FE780E0EF144081477D56B4
:1074AC0013F7F70FE37F97F813974700369710A35E
:1074BC008507FDB779714AD037390020832749F801
:1074CC0006D622D426D24ECE52CC56CA5AC85EC646
:1074DC00C5C7B73A0020AA89130949F8938A2AF834
:1074EC00014405E1B737002083A687F899CA03C683
:1074FC000A002A8481479305F00F13F7F70F63688E
:10750C00C7081315340021059790FB1FE78020D284
:10751C00AA8411E921459790FB1FE78040D1AA84EA
:10752C0021C10144CD49930700FD9CA08547A38050
:10753C003401BCA0A0B045C49389840023A23401BB
:10754C00014A373B0020930BF00F83C70A0063738B
:10755C00FA0029E883270900A6858823EFB0DFD23B
:10756C0003C50A0081455535032509009790FB1F7B
:10757C00E78080B923200900B2502254925402595A
:10758C00F249624AD24A424BB24B45618280139710
:10759C004700369718236305B70005041374F40FDE
:1075AC008507A1BF83278BF893154A00BE959C21B4
:1075BC00638377032380F9009C31138529007D14A4
:1075CC00A380F900194689051374F40F9790FB1FDB
:1075DC00E780A0D5A109050A137AFA0FBDB723A23B
:1075EC0004008DBFB737002083A747F8B1C74111FE
:1075FC0022C406C62A841DE10945EFE0FFA22A86B3
:10760C0001C9B737002003C5C73F8545EFC0CF99E7
:10761C000545EFF0EFE32A84054519C8B73700207C
:10762C0003C5C73F8545EFC02FC022856135054591
:10763C00B240224441018280014582808967938651
:10764C00B7006315D5009C45882369BF9386C70096
:10765C006317D5009C458546882319C9FDB79386C9
:10766C001704E302D5FE938727048146E304F5FE55
:10767C0036858280797106D622D426D24AD04ECE57
:10768C0052CC56CA5AC85EC662C479C53C31AA8966
:10769C0085C7404115C05945EFE01F99931A8501E4
:1076AC0093DA8A410149373A0020130B000DB54B90
:1076BC0083C73900636EF900B250225492540259B8
:1076CC00F249624AD24A424BB24B224C456182800B
:1076DC008307840263C9570783274AF8130C4AF8B7
:1076EC00BDC32285EFF08FFC39CD0824510597904E
:1076FC00FB1FE780C0B3AA8439C5231065012301A1
:10770C0075011C201946930524003CB183078402A3
:10771C0015057CA11C30A30FF5FE9790FB1FE7808D
:10772C00C0C01024D0A415C61385440188C8930585
:10773C0094009790FB1FE78040BF83270C00A68521
:10774C008823EFB07FB40509130494021379F90F61
:10775C0085B723A80400D5B7B737002083A747F80F
:10776C00A1DF893B2254B25092540259F249624A29
:10777C00D24A424BB24B224C014545616FF04FCD82
:10778C00797106D622D426D24AD04ECE52CC56CAC5
:10779C005AC85EC662C45DCD3C31AA8985C74441D6
:1077AC0095C05945EFE05F88931A850193DA8A41B9
:1077BC000149373B0020930B00FD414C83C7390036
:1077CC00636EF900B250225492540259F249624A43
:1077DC00D24A424BB24B224C456182808387F400E3
:1077EC0063C55707130A4BF883270A00B9CF5145D5
:1077FC009790FB1FE780A0A32A8421C92300750161
:10780C00A3000500230185019C20194693852400C3
:10781C003CB18387F40015055CB59C30A30FF5FED5
:10782C009790FB1FE78060B09C2493859400130510
:10783C00C4003CB419469790FB1FE78000AF832728
:10784C000A00A2858823EFB03FA40509C10413796F
:10785C00F90FADB7B737002083A747F8A5D79939EB
:10786C002254B25092540259F249624AD24A424BC3
:10787C00B24B224C014545616FF08FBD5D7186C6E0
:10788C00A2C4A6C2CAC04EDE52DC56DA5AD85ED6A4
:10789C0062D466D26AD06ECE630E05263C31AA84C1
:1078AC008DCB832A450063860A025945EFE0CFF75A
:1078BC0093178501E1873EC60144B7390020130AAE
:1078CC00000D054CB54C130D00FDC14DB830636176
:1078DC00E402B640264496440649F259625AD25AFA
:1078EC00425BB25B225C925C025DF24D6161828014
:1078FC000387CA00B2476348F71603A749F81389F0
:10790C0049F86302071683CB0A0013F70B014DCF1E
:10791C004D47639EEB0623800A005685EFF00FFB64
:10792C006303051403C70A00914763E3E714631963
:10793C00870D51459790FB1FE780608F2A8B63045E
:10794C0005122300A501A30005002301B50183C680
:10795C000A00194693852A0034B18386CA0015059E
:10796C0054B583C61A00A30FD5FE9790FB1FE78072
:10797C00C09B83C60A01194693851A01A305DB0037
:10798C001305CB009790FB1FE780209AF9A0554771
:10799C006398EB0005472380EA00A38B0A00B5BF70
:1079AC007547E389EBFE49476396EB000947238053
:1079BC00EA00A5B741476394EB000D47CDBF6D4777
:1079CC00E39DEBF41147E5B713F78B0019C32D4773
:1079DC00F9BF13F61B0013F74B0011C619C315475B
:1079EC005DBF2147E9B713F62B0011C619C3254714
:1079FC005DB719476DBF19C3294755BF1D4745BF13
:107A0C0003C57A0151059790FB1FE78040822A8BB2
:107A1C0039C9231045012301950183C60A00194673
:107A2C0093852A0034B18386CA00150574A183C6D8
:107A3C001A00A30FD5FE9790FB1FE780008F03C69B
:107A4C007A012306CB0001CA13054B012328AB0096
:107A5C0083A58A0105BF23280B0083260900DA853C
:107A6C008822EFB07F820504F10A1374F40FB9BDBC
:107A7C0003C57A01130505029780FB1FE780207B65
:107A8C002A8B75D1C9473CA12310450103C60A00B6
:107A9C0093F60B0693852A00D18E34B183C61A0057
:107AAC0019461505A30FD5FE9790FB1FE780E087BD
:107ABC0083C68A00194693851A01A305DB0083C689
:107ACC009A0013053B012306DB0083C6AA00A3061C
:107ADC00DB0083C6BA002307DB008386CA00A3073A
:107AEC00DB0083D6EA002318DB0083C60A012309D6
:107AFC00DB009790FB1FE780408303C67A01A30C41
:107B0C00CB0011C613050B02232EAB0091B7232E0D
:107B1C000B00A1B7B737002083A747F8E38B07DA30
:107B2C00EFF05F992644B64096440649F259625AE2
:107B3C00D25A425BB25B225C925C025DF24D014513
:107B4C0061616FF0EF90B737002083A747F89DC7AE
:107B5C0098238D476315A702B737002003C5C73F8D
:107B6C004111854506C6EFB03FEC13050003EFF05D
:107B7C007F94B240014541016FF08F8DC9473E851E
:107B8C00828079714AD037390020130949F883274C
:107B9C00090006D622D426D24ECE6398070E37346F
:107BAC0000201304C43F5820C947298B5DC7916539
:107BBC00AA849385D57111459780FB1FE780C04738
:107BCC002320A900CD4751C978309307F00F6314D7
:107BDC00F7009C207CB01146A6859780FB1FE780A0
:107BEC00C074930531001305F041EF40C221B73743
:107BFC00002093878729A02398813334800011C3F8
:107C0C00090413051002EFE02FC21379F50F9377D7
:107C1C00190093794900B1CB1545EFE0EFC0BC20BA
:107C2C00688419455C82EFE02FC06886638E09007A
:107C3C00BC2013052002DC82EFE00FBF6885130522
:107C4C003002EFE06FBE6887AC307C003800540027
:107C5C004A862285EFB0B007AA87B25022549254BC
:107C6C000259F2493E8545618280E147E38709FE6E
:107C7C00BC20130520025C82EFE00FBB6884130567
:107C8C003002EFE06FBA6886C1B7C547F9B77571B6
:107C9C0026C3B734002022C506C74AC1CEDED2DCCB
:107CAC009384C43FDC204944A18B63810724B737FC
:107CBC00002083A747F84144639A0722AA89EFE082
:107CCC005F839C2455446373F522B734002083A74B
:107CDC0004F626894544639B072091659385C571FD
:107CEC0029459780FB1FE780203523A0A4F64D443F
:107CFC00630E051E2946CE859780FB1FE780E06248
:107D0C0013056002EFE04FB2137AF50F93775A0028
:107D1C006144638D071C130600038145880097801E
:107D2C00FB1FE780206793771A0093692A000144B0
:107D3C00B9CF4145EFE04FAF2316A1043D45EFE02D
:107D4C00AFAE2319A1043545EFE00FAE231CA104FF
:107D5C003945EFE06FAD231FA1042145EFE0CFAC17
:107D6C002312A1061D45EFE02FAC83A704F62315C3
:107D7C00A1069C33638507182D45EFE0EFAA23106D
:107D8C00A1043145EFE04FAA2313A10405441305C8
:107D9C00C002EFE06FA9981893171400BA97239EAE
:107DAC00A7FC1305B002EFE02FA8930484009C18E5
:107DBC008604BE942399A4FC13059002EFE0CFA691
:107DCC00239CA4FC1305A002EFE00FA6239FA4FCA8
:107DDC0013058002EFE04FA5930404019C18860460
:107DEC00BE94239AA4FC13057002EFE0EFA3239D2D
:107DFC00A4FC137A4A0063040A0813056003EFE03D
:107E0C00AFA205049C1893141400BE94239EA4FCEA
:107E1C0013055003EFE04FA1130A84009C18060AC7
:107E2C003E9A2319AAFC13053003EFE0EF9F231CA5
:107E3C00AAFC13054003EFE02F9F231FAAFC130598
:107E4C00E002EFE06F9E41049C1806043E94231A56
:107E5C00A4FC1305D002EFE02F9D832709F6231D08
:107E6C00A4FC9C33C5C713051003EFE0EF9B2398CC
:107E7C00A4FC13052003EFE02F9B239BA4FC83277A
:107E8C0009F6A83393854700EFD07F812AD6930556
:107E9C00F1031305F041EF301277B73700209387C9
:107EAC008729AC230347F1033256B335B00011C315
:107EBC008905832609F6FC009308A106A8223EC872
:107ECC00930721053EC6BC083EC49307E1053EC29C
:107EDC00DC103EC0130861049C004E879106EFB085
:107EEC00805F2A8401C50D45EFE06FC82285BA403A
:107EFC002A449A440A49F659665A496182802545B2
:107F0C00EFE08F922310A1042945ADBD1305F002BB
:107F1C00EFE08F912398A4FC13050003A9BFB7379A
:107F2C00002083C707400145A18B89C73735002046
:107F3C00130545356FD02FD3B73700207D572381DC
:107F4C0007F8B7370020A381E740B737002023A4F8
:107F5C0007F837770400B73700201307876423A28C
:107F6C0007F8B737002023A0E7343777040093874E
:107F7C00073413070768D8C3377704001307C7788B
:107F8C0098C73787040013078788D8C7377704004A
:107F9C00130707DF98CB37770400B7370020130798
:107FAC00E7E723AAE73437770400938747351307AD
:107FBC0067C9D8C38280411122C43734002013040E
:107FCC0024F826C2AA840820854506C6EFF0EFC324
:107FDC00B737002083C70740A98BBDC737350020B2
:107FEC0004A013050534B7340020EFD02FC79384B9
:107FFC0084F89C4099C74D45B240224492444101BB
:10800C008280082019E10145C5BF91659385B57142
:10801C0012059780FB1FE780200288C069DD1020C5
:10802C00814512069780FB1FE780C03614209040D4
:10803C008147FD5513F7F70FE377D7FC13974700EC
:10804C0032970CA38507FDB7014523000400EFD040
:10805C00EFC055BF411122C437340020032544F62C
:10806C0006C619C59780FB1FE780000A232204F679
:10807C00B24022444101828001111305700306CEE7
:10808C00EFD09FFA2AC613058003EFD0FFF92AC45C
:10809C0013059003EFD05FF92246B245F240AA8651
:1080AC00054505616FB0E0415D711305D00386C6CF
:1080BC00A2C4A6C2CAC0EFD03FF72A841305C003DE
:1080CC00EFD09FF6AA841305E003EFD0FFF52A89C1
:1080DC001305F003EFD05FF58A871377F50F9376CE
:1080EC00F90F13F6F40F9375F40F0545EFB0A03F9D
:1080FC00B64026449644064961618280757122C55A
:10810C0037340020832744F606C726C34AC1CEDE87
:10811C00D2DCD6DADAD8DED6E2D405456389070E8E
:10812C009305F1051305F041EF30F24D9305F10580
:10813C001305F041EF30324DB73700209387872974
:10814C00BC230347F105B337F00011C3890703279C
:10815C0044F6BEC6283393054700EFD04FD403270F
:10816C0044F6AAC40D452C23AEC2EFD0FFEBAAC037
:10817C001145EFD07FEB032444F62ADE6545382405
:10818C00034CB4003ADCEFD03FEAAA846945EFD047
:10819C00BFE92A897145EFD03FE9AA896D45EFD037
:1081AC00BFE82A8A7545EFD03FE8AA8A7945EFD017
:1081BC00BFE72A8B13050004EFD01FE7AA8B13052A
:1081CC001004EFD07FE6E2042648B6476257F25619
:1081DC00064696451375F50F93FBFB0F137BFB0FB0
:1081EC0093FAFA0F137AFA0F93F9F90F1379F90F2F
:1081FC00E1842AD05ECE5ACC56CA52C84EC64AC466
:10820C0026C262C0930844000545EFB06026BA4010
:10821C002A449A440A49F659665AD65A465BB65BC2
:10822C00265C49618280011122CC06CE26CA8D477C
:10823C002E84631AF504B831B7340020E947CA21FB
:10824C00938484296315F700FE206389A704979013
:10825C00FB1FE780A08319C17E207EA53A2416243B
:10826C0072204E202830EFD09F945A20FE206309B4
:10827C00F7008547F2406244D2443E850561828016
:10828C00FD57FEA0FDB78967CD07631CF500BC2127
:10829C0031476385E7004547E39DE7FCEFD0AFA38B
:1082AC00C9BFB1476319F500B737002003C51740A4
:1082BC00EFD03F9B7DBF930760026319F500B73782
:1082CC00002003C51740EFD05F9E65B741677D174F
:1082DC008147E311E5FAD4314947E39DE6F8CC2117
:1082EC002A20300023140100EF60B02D59B7411142
:1082FC0022C4373400208347C4F826C206C64AC0BD
:10830C001307E00FAE846382E7041307F00F130426
:10831C00C4F86384E70211459780FB1FE78020F1C6
:10832C0009CD930700FD1CA189473CA1854704B1E9
:10833C003CB1AA850820EFA03FF5F9571CA0B2402C
:10834C00224492440249410182802A891145978036
:10835C00FB1FE780C0ED65D5930700FD1CA1894785
:10836C003CA104B1A30125012244B7370020B2403F
:10837C0092440249AA8503C5D7F841016FA0DFF0EA
:10838C0079714AD037390020832749F622D406D692
:10839C0026D24ECE52CC56CA4544C5EBB73400203B
:1083AC009387C43FDC234944958BC5C3B737002062
:1083BC002E8A9165A386A7F8AA8993857571314594
:1083CC009780FB1FE78040C72322A9F64D4435CD8B
:1083DC0023003501A30005002946D28509059780A5
:1083EC00FB1FE78080F4832749F69146B82363E9A5
:1083FC00E60835E74D47B8A3B82313670701B8A3C0
:10840C00930571001305F041EF30F21F9C83F1E7E7
:10841C00B737002003C7A7298D476310F70CEFD09F
:10842C008FB52C00EF70B01D2800EFD0DF994545BB
:10843C00EFD09FBF014411C9130600643306C50277
:10844C0003C5C43F9145EFB02FB62285B2502254DC
:10845C0092540259F249624AD24A45618280854659
:10846C006314D700754741BF89466314D700494749
:10847C0059B78D466314D7004147B5BF5547A5BFC3
:10848C009546CA8A630DD70099466315D7000947EC
:10849C00B8A331A01D466312C702238107006545AE
:1084AC00EFD09FB89307F007E30CF5F403A74AF657
:1084BC003C2393E707043CA3A1B721466314C700F0
:1084CC000547F9B725466314C700B4A3C9BFA9462D
:1084DC000544E31CD7F6114765BFEFF03FC22A8471
:1084EC002DD5EFF03FB795B7011126CAB734002050
:1084FC0083A744F622CC06CE4AC84944B9C39C2370
:10850C000D446390A704373900200345C93F8945C2
:10851C00EFB08FD10345C93FB73700209145239861
:10852C0007F8EFB06FD083A744F60147814680B3BC
:10853C001306F100854785450145DC87EFA03078AF
:10854C002A842285F2406244D244424905618280E9
:10855C00011106CE22CC26CA4AC88547631AF506F5
:10856C0037340020130404F91E20B9C73737002014
:10857C000347C72931E31307B003636BF702B73422
:10858C00002003C5C43F8945EFB00FCA12209307E2
:10859C00006403C5C43F3306F6028945EFB0CFA093
:1085AC0023100400F2406244D244424905618280A7
:1085BC00938747FC1EA0FDB7B737002083A747F66B
:1085CC00F5D36244F240D24442498823056129BF65
:1085DC00B734002083A744F6F1D7373700201309AE
:1085EC00C73F83474900918BD5DF89476310F50658
:1085FC002D452EC69780FB1FE78060C32A845DD172
:10860C00B245930700FD1CA1E547A30005003CA162
:10861C00BC3115051946230FF5FEDC219505A30F7A
:10862C00F5FE9780FB1FE78040D003455900930768
:10863C00F00F6315F50083A744F68823A2856244E6
:10864C00F240D244424905616FA01FC40345C73FA5
:10865C008945EFB06FBD6244F240D2444249B7370E
:10866C000020239807F805616FF0DF9EB7370020D4
:10867C0083C70740958B89CFB737002083A7C7F9ED
:10868C0091CBB73700200547238EE7346FF0DF9E80
:10869C004945828041458280B73700208545014598
:1086AC00238E07346FA07062B737002083C7074052
:1086BC00958B81CBB737002005472387E7F86FF000
:1086CC00BF9E49458280B7370020814505452387E9
:1086DC0007F86FA09061B737002083C70740958BD0
:1086EC00638C07129307C01C63FCC700094582808A
:1086FC00F2406244D2444249B24909450561828044
:10870C00B737002083A747F663880710B7370020D8
:10871C009387C7F803C807001307E00F631EE80E22
:10872C00011122CC4AC806CE26CA4EC688A3130510
:10873C0086004205368932844181A5C991659385AD
:10874C0065719780FB1FE780208FAA8955D1B734BC
:10875C00002003A584F9938484F909C59780FB1F35
:10876C00E780809A1385890023A0A9002286814581
:10877C0023A034019780FB1FE780C0C19C40228658
:10878C00CA8588439780FB1FE78020BA9C40A2864D
:10879C00F240C2A36244D2444249B24998430546CE
:1087AC008D45054505616FA01051916593855571F7
:1087BC009780FB1FE7804088AA891DD9B734002019
:1087CC0003A504FA938404FA09C59780FB1FE7807C
:1087DC00A0931385890023A0A9002286814523A09C
:1087EC0034019780FB1FE780E0BA9C402286CA8543
:1087FC0088439780FB1FE78040B39C40A286F240E1
:10880C00C2A36244D2444249B249984305468D45BD
:10881C00054505616FA0704A494582809307C01CCD
:10882C0063FCA700094582800945F2406244D244AA
:10883C004249B2490561828055C9011122CC2A8472
:10884C0021054EC64205AE899165938565714181BE
:10885C004AC806CE26CA9770FB1FE780E07D2A899E
:10886C0061D5B734002003A584F9938484F909C534
:10887C009780FB1FE7804089130589002320A900FE
:10888C002286814523A024019780FB1FE78080B0BE
:10889C009C402286CE8588439780FB1FE780E0A80A
:1088AC009C40C2A3B737002083A747F685CFB737C4
:1088BC00002083C70740958B85CBB737002083A753
:1088CC0087F991CF9843D6236244F240D24442496F
:1088DC00B24905468D45054505616FA0D03D014760
:1088EC008146DDB7014591B7494581B7B7370020BF
:1088FC0083A747F68DC7B737002083C70740958BF2
:10890C008DC3B737002083A787F999C79843D6231F
:10891C0005468D450545D1B701478146D5BF014573
:10892C008280494582809307C01C63FCA7000945DF
:10893C0082800945F2406244D2444249B249056101
:10894C00828055C9011122CC2A8421054EC64205CC
:10895C00AE8991659385557141814AC806CE26CA68
:10896C009770FB1FE780406D2A8961D5B7340020D2
:10897C0003A504FA938404FA09C59770FB1FE780DA
:10898C00A078130589002320A9002286814523A005
:10899C0024019780FB1FE780E09F9C402286CE85B8
:1089AC0088439780FB1FE78040989C40C2A3B73751
:1089BC00002083A747F685CFB737002083C7074031
:1089CC00958B85CBB737002083A707FA91CF9843B7
:1089DC00D6236244F240D2444249B24905468D4501
:1089EC00054505616FA0702D01478146DDB7014536
:1089FC0091B7494581B7B737002083A747F68DC794
:108A0C00B737002083C70740958B8DC3B73700203D
:108A1C0083A707FA99C79843D62305468D45054584
:108A2C00D1B701478146D5BF014582804945828037
:108A3C009307C01C63F4A70009458280797122D486
:108A4C004ECE06D626D24AD0AE892A8425C121051F
:108A5C00916542059385757141819770FB1FE78085
:108A6C00A05D2A89094563040908B734002003A5D1
:108A7C00C4F99384C4F909C59770FB1FE780C068DB
:108A8C00130589002320A9002286814523A02401F7
:108A9C009780FB1FE78000909C402286CE85884300
:108AAC009780FB1FE78060889C40C2A3B7370020EB
:108ABC0083A747F6014585CFB737002083C707400A
:108ACC004945958B8DC76C001305D030EF40526132
:108ADC00B247014593F7070F99CBB737002083A70F
:108AEC00C7F98D4505459443D223EFA0D01DB25054
:108AFC00225492540259F24945618280B7370020C2
:108B0C0083A787F989CFD2238C43411106C697805E
:108B1C00FB1FE7808081B2400145410182800945FD
:108B2C008280B737002083A787F985C7B737002025
:108B3C0003A707FA894719CF52230C43411106C6E4
:108B4C009770FB1FE780607EB24081473E854101F4
:108B5C00828089473E858280B737002083A787F9BA
:108B6C0085C7B737002003A7C7F9894719CF522308
:108B7C000C43411106C69770FB1FE780007BB24087
:108B8C0081473E854101828089473E85828079718B
:108B9C0006D622D426D24AD04ECE52CC8D4763FC78
:108BAC00A7008944B2502254268502599254F249A6
:108BBC00624A456182803739002003478929C144C4
:108BCC00E312F7FE9307F5FF9309892993F7F70F43
:108BDC008546AE842A8403CA29001309892963EACD
:108BEC00F6068DE199452800EFC0DF89B7390020E2
:108BFC0003C5C93F914523018900EFA0FFE235E48D
:108C0C0081444DB71946814528009770FB1FE780BA
:108C1C00607819462C0026859780FB1FE780E08141
:108C2C0049F119469305F00F28009770FB1FE78058
:108C3C00607619462C0026859770FB1FE780E07F35
:108C4C002DF11946A68528009770FB1FE780E06D73
:108C5C0071BFE31DE5F803A5C9002C00EF70201AC5
:108C6C00AA8449D52381490135BF2800EFD0AF959F
:108C7C00AA8405ED930571001305F041EF30A2189D
:108C8C008483BDFC8D47E31DF4F64545EFD0CFB989
:108C9C0025D9B7771800938707A03306F50203C5CB
:108CAC00C93F9145EFA0FFD0F5BD23014901DDBDC2
:108CBC00B737002083C70740918B8DC33735002011
:108CCC004111130545F906C6EFC02FFBB240B7376B
:108CDC0000207D57239FE7284101828001456FC00A
:108CEC00CFF9B73700207D57A386E7F8B7370020B8
:108CFC0079572386E7F8B7370020238E0734B73728
:108D0C000020238707F8B7370020239807F8B737D8
:108D1C00002023AC07F8B737002023A007FAB73799
:108D2C00002023AE07F837970400B737002093874D
:108D3C0087041307E7F498C3378704001307C75554
:108D4C00D8C3378704001307871098C737870400E8
:108D5C0013074708D8C7378704001307470B98CB6E
:108D6C00B78704003737002093872723232AF7F887
:108D7C008280411126C2B734002083A744F606C670
:108D8C0022C49DCB2A840D459770FB1FE780204A97
:108D9C00AA8501CD930700FD1CA18D4700B13CA114
:108DAC0083A744F68823EFA02FCE19C42244B240E7
:108DBC00924441016FF00FAAB24022449244410107
:108DCC008280797152CC373A002083274AF64AD0F8
:108DDC0006D622D426D24ECE56CA0149A1C703C903
:108DEC001700B73400208547AA899384842963052A
:108DFC00F904DC2005499DE70D459770FB1FE780C2
:108E0C000043AA8509CD930700FD1CA19147A3003F
:108E1C0035013CA183274AF68823EFA0EFC6EFF07B
:108E2C006FA30549B25022544A8592540259F24913
:108E3C00624AD24A45618280B737002083A787F9FE
:108E4C00D28A85E30145EFD02F9E2A8601CAB73717
:108E5C00002003C5C73F8945EFA01F9583A74AF69D
:108E6C00B1A09443D2239305E1000545EFC08FEBED
:108E7C0071D91C21858BF9D70545EFD0EF9A930753
:108E8C00B0032A8463FEA702B737002003C5C73F8F
:108E9C005D66130606708945EFA0BFB1B737002099
:108EAC00130444FC239887F883274AF6094798B3A0
:108EBC00DC2081C723820400B5B74E855D3D9DB78C
:108ECC00130600643306C50251B7411122C42A842B
:108EDC000D4506C69770FB1FE78060350DC19307E3
:108EEC0000FD1CA1CD473CA100B12244B7370020A6
:108EFC00B240AA8503C5D7F841016FA0EFB8B240C4
:108F0C00224441018280411122C42A840D4506C6A7
:108F1C009770FB1FE780A0310DC1930700FD1CA1CA
:108F2C00ED473CA100B12244B7370020B240AA85DE
:108F3C0003C5D7F841016FA02FB5B24022444101BF
:108F4C0082805A210111896606CE22CC26CA13864C
:108F5C006600AA876316C7009C4701458C2301A8AD
:108F6C00138686006319C7009C4705458C23EFF0D8
:108F7C000FB805451DA8138696006311C702373735
:108F8C000020032747F601450DC39C47882369E55C
:108F9C0085471CB30545EFA0A048E1BF1386A6008A
:108FAC00631AC7009C478823293DF2406244D2448F
:108FBC000561828013866603E300C7FA1386760385
:108FCC00E304C7FA13868603631BC7081C453734B2
:108FDC0000201307E00F84238347C4F81304C4F85C
:108FEC00638BE7021307F00F6384E7021145977058
:108FFC00FB1FE780C023AA8501CD930700FD1CA1B0
:10900C00894704B13CA1A30105000820EFA0CFA71C
:10901C00F9571CA0B9BFB737002003A747F63E8409
:10902C00014541D78DE885447D454485EFC0DFFF80
:10903C00688613050002EFC03FFF832744F6C885FE
:10904C001307B10084B374001306A10085450545D0
:10905C00EFA0E04639BF2685EFF0BFD119BF1386CC
:10906C009603E301C7F41386E6036316C7001C4599
:10907C0009458C23EDBD9386F603631BD7021C4573
:10908C00882335E96C001305D030EF407205B247E8
:10909C00414793F7070FE38EE7EC9305B1001305F7
:1090AC006031EF40F20388858545EFA00042D1B5D1
:1090BC008966138606046312C7041C458023B737E0
:1090CC00002083C7C73522859DE70D459770FB1F90
:1090DC00E780E015AA85E30E05E8930700FD1CA1C7
:1090EC00D1473CA100B1B737002083A747F68823AE
:1090FC00EFA08F99BDBDD13BADBD13861605631A8C
:10910C00C7001C45882331E585450545EFA0E03DAA
:10911C008DB5938626050145E319D7E89C47802336
:10912C00B737002083C7E7F8228585E70D45977090
:10913C00FB1FE780C00FAA85E30D05E2930700FD36
:10914C001CA1F1473CA1B737002000B103C5D7F8EB
:10915C0045B7553B39BDB737002083C70740411190
:10916C0006C6958B99CB3735002013058504EFC0C7
:10917C002FB04D45B240410182800145EFC04FAF49
:10918C000145CDBF9821937625009377D70F99C2CF
:10919C0093672700131885011358884113F7F707B5
:1091AC006354080013E70708937685009377770FCD
:1091BC0099C2936787001377050293F6F70D19C3CD
:1091CC0093E6070294A1634508009377A50291C723
:1091DC001C2293E7C7001CA282807DFD1C22CD9B24
:1091EC00DDBF2D45631B0710882109476313E5106C
:1091FC0001114EC6BE89DC4122CC26CA4AC806CE15
:10920C0098339C23B68422075D8F42078D66418775
:10921C00938736A032842E89630BF70A63C0E7026A
:10922C00938716A06307F70863CAE70A938606A01C
:10923C00630BD70423900400054559A0938766AAB5
:10924C00630EF708938786B86301F70A938646A0E6
:10925C00E312D7FEDC45C1C321479AA09A2318A27A
:10926C009A23218318B2BA2338A2BA23218338B2A5
:10927C00DA2358A2DA23218358B2FA2378A2FE23E8
:10928C00A1837CB22DA8C8459770FB1FE7806013A3
:10929C00420541814E86637335012A8692A04206AF
:1092AC0041828325C90022859770FB1FE780E00768
:1092BC0039A0DC459E238AA01CA2A1831CB20145C7
:1092CC00F2406244D2444249B249056182809947D6
:1092DC009EA01946F9B723900400D5B785479EA0E8
:1092EC008327C9009C231CA0D9BFE1479EA06146DF
:1092FC004DBF2390060005458280828083C80500FF
:10930C008947639BF816DC41797122D406D626D2A4
:10931C004AD04ECE52CC56CA03C817009C232E847A
:10932C0022083368F80042088D67135808411383EC
:10933C0027A0630F68102A8A3A89B684B285634CD9
:10934C000301138707A0630BE802938717A063013F
:10935C00F80A854711A8138737A06300E80C138718
:10936C0067AA8D47E317E8FEB25022549254025973
:10937C00F249624AD24A3E8545618280484432C6EF
:10938C009770FB1FE780E003420541819D47E36D29
:10939C0025FDB73A0020938A7AFA83C70A00B309ED
:1093AC009900B24563D43701B5477DBF4844268642
:1093BC00C2094A959770FB1FE78020F703C60A0085
:1093CC00484493D9090105063306364181454E952B
:1093DC009770FB1FE78000FCB737002083A7C7FA04
:1093EC0099E3814751B79C438145E5DF528525A020
:1093FC00AD47E31B09F6E39916FB1C3214225844C3
:10940C00A207D58F1EA3B737002083A7C7FAF1DBBD
:10941C009C43E1DB85458297E9B7B737002003C74A
:10942C0007FB8D4731D3AD47E31009F49947E39D12
:10943C00F6F6484419469770FB1FE78000EFB737E4
:10944C00002083A7C7FAD1DF9C43C1DF8D4579BFCC
:10945C00B737002083C5C7F28D47A18991D5AD4799
:10946C0001F78547E392F6F4182293070008E3ED21
:10947C00E6EE5C4498A3B5B785473E858280B73746
:10948C000020411123A607FAB737002022C42385F8
:10949C0007FA0944B7370020A38F87F0B7370020AD
:1094AC00A38307FAB7370020238E87F0B737002045
:1094BC00239207FAB7370020238687F2373500202E
:1094CC00B73700202147238807FA1946B737002001
:1094DC008145130545FB06C6A386E7F29770FB1F73
:1094EC00E78040EBB7370020238187F23707A000D5
:1094FC00B7370020938747F21307070598C3370740
:10950C00E803D8C3B7370020238F87F00547B73758
:10951C000020A38EE7F0B7370020238787F237357A
:10952C000020B7370020238D07FA6146B73700209B
:10953C0081451305C505238087F29770FB1FE780D3
:10954C0060E5B7370020A38087F2B7370020A384EB
:10955C0007FA37970400B73700209387C7EB130738
:10956C00E71E98C3B2402244379704001307873094
:10957C00D8C323A407004101828095476302F51AE2
:10958C00797122D426D206D64AD04ECE52CCB28491
:10959C002E8463E4A7048947630DF51463EFA700D9
:1095AC004DC50547630FE5120945B250225492543C
:1095BC000259F249624A456182808D476304F51471
:1095CC009147E313F5FEA1476395F5083735002065
:1095DC002146A685130545F23DAA93072004630591
:1095EC00F51663E1A7029D476306F514A147E31D39
:1095FC00F5FA8547639FF5041822B7370020A3843A
:10960C00E7FAF1A8930710086309F51493072008EB
:10961C00630DF51493070008E318F5F88547639A72
:10962C00F502B737002083C787FA1387F7FFB735E2
:10963C0000209385450712072E97920750478820E4
:10964C00A107BE95EFF01FB459A89307800F63F4E0
:10965C00B700614599BF373A002083468AFAB7377D
:10966C000020138747079206369748479389470788
:10967C00130A8AFA09C99770FB1FE780E0A8B7376D
:10968C000020A38307FA13061400916593850571D6
:10969C00328503490A0032C69770FB1FE780C099D8
:1096AC0083470A0012094E9992072326A900CE97E8
:1096BC00C84745D1324681459770FB1FE78080CD66
:1096CC0083470A002286A6859207CE97C8479770D3
:1096DC00FB1FE78080C5B7370020A38387FA0145BD
:1096EC00E9B5E398F5F61A22B73700202392E7FA8A
:1096FC00FDB78547E39FF5F41822B7370020238880
:10970C00E7FAF1BF9947E396F5F43735002019468F
:10971C00A685130545FB9770FB1FE78000C1C1B7F9
:10972C008547639DF5061822B73700200145A38EA7
:10973C00E7F08280E147E39EF5F037350020614683
:10974C00A6851305C505C1BF8547E394F5F018221E
:10975C00B73700202386E7F259B78547E39BF5EE30
:10976C00B737002083C767FAC9B58547E393F5EE91
:10977C00082293772500E39E07ECB737002083C7B8
:10978C0017FBB7350020938545071387F7FF1207A2
:10979C0092072E97A1075047BE956DB56145828003
:1097AC004111AA8706C611472E856386E70A6361B5
:1097BC00F7020547638EE706A9C709476381E708E7
:1097CC000D476384E7088947B2403E85410182809A
:1097DC001D47638AE708636AF7001547E395E7FEC0
:1097EC00B737002083C7D7F1B9A821476383E708AF
:1097FC0013072004E399E7FCB737002083C7C7F2AF
:10980C0099A0B737002083C787FA13974700B7375B
:10981C00002093874707BA97CC478947D5D5B737E8
:10982C00002003C677FA9770FB1FE78000B031A0C9
:10983C00B737002083D747FA9EA1814771B7B73756
:10984C00002083C707FB1CA1CDBFB73500201946EC
:10985C00938545FBC9BFB73500202146938545F25A
:10986C00EF401243D9BFB735002061469385C5053B
:10987C005DBFB737002083C797FAF1B7630F053880
:10988C00B73700209387A7FA9823631807388546C3
:10989C003738002094A309479307480798A337F754
:1098AC000600130707C8D8C337F706001307C7C449
:1098BC00D8C794A7239507007D57630DE53413771C
:1098CC001500854539C3B7F606009386C6C5D4CBBB
:1098DC00B73600209386F6F10947D4CFB73600206F
:1098EC0098AB2384E6FA2380E70237F70600054697
:1098FC00130747C690AF239D0700D8D32384C70214
:10990C002395070223A607028D45137725002DC347
:10991C0013974500B7F606003E979386C6C554C309
:10992C00B7360020894805469386C6F154C72300F4
:10993C00170110A723150700138715004207418351
:10994C00B73600202383E6FA1207B7F606003E97D7
:10995C00938646C554C38905B7360020938646FACC
:10996C00C2052300170110A72315070054C7C18196
:10997C00137745002DC313974500B7F606003E97A5
:10998C009386C6C554C3B7360020894805469386CE
:10999C00C6F254C72300170110A72315070013871D
:1099AC00150042074183B7360020A388E6FA120758
:1099BC00B7F606003E979386C6C754C38905B736DB
:1099CC000020938606FBC2052300170110A7231560
:1099DC00070054C7C1811377850021CF1397450029
:1099EC00B7F606003E979386C6C554C3854614A7A2
:1099FC00B736002009469386D6F254C710A3231518
:109A0C00070013871500420741831207B7F60600BB
:109A1C003E97938686C854C3A14614A78905B736CA
:109A2C000020938646FBC20510A32315070054C7DC
:109A3C00C1811377050129CF13974500B7F60600AE
:109A4C003E979386C6C554C3B73600208948054651
:109A5C00938626F254C72300170110A7231507007D
:109A6C0013871500420741831207B7F606003E978D
:109A7C00938686C754C38905B7360020938646F271
:109A8C00C2052300170110A72315070054C7C18175
:109A9C001377050229CF13974500B7F606003E97BA
:109AAC009386C6C554C3B7360020894805469386AD
:109ABC00E6F154C72300170110A7231507001387DD
:109ACC001500420741831207B7F606003E979386AE
:109ADC0086C554C38905B73600209386D6F1C205D6
:109AEC002300170110A72315070054C7C181137752
:109AFC00050429CF13974500B7F606003E979386C9
:109B0C00C6C554C3B7360020894805469386E6F28D
:109B1C0054C72300170110A723150700138715003E
:109B2C00420741831207B7F606003E97938646C854
:109B3C0054C38905B73600209386A6FBC2052300C3
:109B4C00170110A72315070054C7C1811377050807
:109B5C0021CF13974500B7F606003E979386C6C5EE
:109B6C0054C3D14614A7B73600200946938606F293
:109B7C0054C710A323150700138715004207418310
:109B8C001207B7F606003E97938686C654C38546E1
:109B9C0014A78905B73600209386C605C20510A305
:109BAC002315070054C7C1811375051039C91397C4
:109BBC004500B7F606003E979386C6C554C3B73624
:109BCC00002009450546938616F208A310A7231515
:109BDC00070054C713871500420741831207BA9731
:109BEC0037F70600130787C6D8C389053737002017
:109BFC00130797FAC20588A390A723950700D8C727
:109C0C00C181B73600209386C6EB41461305480741
:109C1C006F30E039130530037DB1014582800111AD
:109C2C001388F5FF06CE22CC26CA4AC84EC652C4AB
:109C3C001378F80FAD4563ED050BB7E506000A0880
:109C4C00938505572E983E8A83270800BA89368952
:109C5C00B28482878545EFB09F9F2A8419E1EFF08B
:109C6C008FCF2285F2406244D2444249B249224A03
:109C7C00056182808945EFB09F9D2A847DF1268500
:109C8C00EFE06FB3F9BF9145EFB07F9C2A8471F977
:109C9C005286CE854A85EFB0FF91EFF0CFCBEFF037
:109CAC002F81EF60E07D75BFA145EFB05F9A2A84EC
:109CBC004DF95286CE854A85EFB0DF8F2685EFE0D1
:109CCC008FAFEFE0CFA5EF60A07961BFB145EFB0EA
:109CDC001F982A8459F55286CE854A85EFB09F8D00
:109CEC002685EFE04FADEFE08FA3EF60607775B79F
:109CFC00094485BF79714ECEAE896C0022D426D230
:109D0C004AD006D62A89B284EF0070692A840DE104
:109D1C00CE854A85EFA07FEA2A8419E93245B756E9
:109D2C00040026879386A6BB2D468145EF10400183
:109D3C002285B250225492540259F24945618280D4
:109D4C0079714ECEAE896C0022D426D24AD006D67A
:109D5C002A89B284EF00B0642A840DE1CE854A854D
:109D6C00EFA03FF32A8419E93245B7560400268741
:109D7C00938646C94D468145EF00907C2285B250B2
:109D8C00225492540259F24945618280397126DA83
:109D9C00AE844C0022DC4AD84ED652D406DEAA89B8
:109DAC003289368AEF00B05F2A8421E9A685630DDB
:109DBC0009009E202C007C84BE207C8593072030DB
:109DCC007C86930780025C874E85EFA03FDC2A845B
:109DDC000DE55946A6851305A100230421019760C2
:109DEC00FB1FE78080541245B756040052879386B8
:109DFC00C6B625462C00EF00B0742285F250625492
:109E0C00D2544259B259225A21618280797126D298
:109E1C00AE846C0022D44AD04ECE06D6AA893289A2
:109E2C00EF00F0572A840DE1A6854E85EFA0BFDA2E
:109E3C002A8419E93245B75604004A87938666BDD1
:109E4C003546A685EF00D06F2285B250225492542D
:109E5C000259F24945618280BD47638CF50663E97E
:109E6C00B702A5476387F50663EDB7009947638C86
:109E7C00F5049D47638FF5049547638CF504014504
:109E8C008280B5476387F50463E1B704AD47F5B746
:109E9C00DD47638EF50263EAB700C947638BF502B1
:109EAC00D9476386F502C547C9BFF5476383F502F9
:109EBC0063E4B700ED47D1B793072005638BF5003A
:109ECC009307200D5DBF484582800841828008457C
:109EDC008280484182809307F00F630FF5060111D1
:109EEC0026CAAA841305000222CC4AC84EC652C404
:109EFC0056C206CE3A89B689B28A2E8A9760FB1F63
:109F0C00E780E0322A844D450DC8930700FB1CA066
:109F1C00A3005401231144012302340113058400CE
:109F2C00614663050902CA859760FB1FE780E03F25
:109F3C00A2852685EF904FB50145F2406244D2448C
:109F4C004249B249224A924A056182808145976012
:109F5C00FB1FE7802044E9BF09458280011122CC18
:109F6C0006CE2A844C86D0869770FB1FE78000B201
:109F7C0005C15425B737002021479387C73F639D00
:109F8C00E600E82378009306E0070146A285A13796
:109F9C00F24062440561828078009306E007014636
:109FAC00A285C833EDB7930700643306F6026F90B1
:109FBC007F9415C5182185469307270093F7F70F53
:109FCC0063FFF600411122C42A843A8506C6EF903D
:109FDC007FACFD571CA0B24022444101828082809C
:109FEC001A219307000B6310F7025C214947639A0F
:109FFC00E700183985476398E7002A2185456F30BB
:10A00C00101F6D47CDBF828001116C846C0022CC77
:10A01C0026CA4AC806CE2A89B6847085EF00303825
:10A02C002A840DE12C004A85EFA0FFAC2A8419E9A3
:10A03C003245B75604002687938606AC15462C008D
:10A04C00EF0010502285F2406244D244424905612F
:10A05C0082807971930720306C8470857C862C000B
:10A06C0093078002014606D65C87EFF03FD2B250D0
:10A07C0045618280C177797185073EC4894726D2B4
:10A08C007C86AE84930780024C0022D44AD006D63C
:10A09C002A895C87EF00B0302A840DE12C004A85B8
:10A0AC00EFA07FBC2A8419E91245B7560400268715
:10A0BC00938646C445462C00EF0090482285B2504A
:10A0CC0022549254025945618280B28605466FF043
:10A0DC00FFCB797126D2AE846C0022D44AD04ECEFE
:10A0EC0006D6AA893289EF00902B2A840DE1A68529
:10A0FC004E85EFA01F982A8419E93245B756040003
:10A10C004A87938666A60D46A685EF007043228586
:10A11C00B250225492540259F249456182807971AD
:10A12C00930720206C8470857C862C00930780021A
:10A13C00014606D65C87EFF07FC5B2504561828040
:10A14C00011122CC06CE2A842EC632C436C2977098
:10A15C00FB1FE780A09315C94825B7370020A146FF
:10A16C009387C73F12472246B245631BD500E823AD
:10A17C00B2862E86A2856244F24005616FF0BFD58F
:10A18C00B286C8332E86A285FDB7F24062440545DF
:10A19C00056182806FF01FB66FF0DFB56FF01FC7DF
:10A1AC006FF0DFC679714ECEAE896C0022D426D208
:10A1BC004AD006D62A89B284EF00701E2A840DE19B
:10A1CC00CE854A85EFA0FFA22A8419E93245B756FD
:10A1DC0004002687938626BF3D468145EF00503606
:10A1EC002285B250225492540259F2494561828020
:10A1FC00B28601466FF09FB9011122CC2E846C00FF
:10A20C0026CA06CEAA84EF009019DD476309F50033
:10A21C00930710101EA4A2852685EFA09FA7F240DD
:10A22C006244D24405618280239405009E2599E303
:10A23C006FF01FB109458280C5BFB737002003C737
:10A24C0027FF854763F8E702011122CC2E846C00AE
:10A25C0026CA06CEAA84EF00901401E993070010D9
:10A26C001EA4A2852685EFA0DFA2F2406244D24450
:10A27C000561828059458280B737002023AEA7FA4A
:10A28C008280B737002023A0A7FC8280011122CC4A
:10A29C0026CA06CE2A84AE849760FB1FE780007F17
:10A2AC00A6852285EFA0EFD005E92285648697600C
:10A2BC00FB1FE780A07D0DC15425B7370020214737
:10A2CC009387C73F639FE600E82378009306F00767
:10A2DC000146A285EFF03FC0F2406244D2440561D2
:10A2EC008280C833DDB7011126CA06CEB68422CCD3
:10A2FC00DD4663E3B608D94663FFD50AA5466382FB
:10A30C00D50A63EFB6049546638DD50899466388E4
:10A31C00D50A054441687D18631706093AC6EFA0B3
:10A32C000FCD3306854032474206418242044180BC
:10A33C003305C4004205BA85418132C6EF3020791D
:10A34C00AA8751C199C0324692A0B305804062449D
:10A35C00F240D2443E8505611763FB1F670003E89A
:10A36C00C5466380D504C9460D44E394D5FAC1674C
:10A37C00FD17E31DF6FA5DB7F5466380D50463E47B
:10A38C00B600ED46D5B7930620056388D502930633
:10A39C00200DE390D5F8C167FD170D446319F60045
:10A3AC00B5BF094485BF9306200DE391D5F831065E
:10A3BC0042064182A5BF15445DBF0D444DBFC16728
:10A3CC00FD171D447DB7F2406244D2440561828082
:10A3DC00011122CC26CA06CED0212E8413070002EE
:10A3EC0081469945AA8401372AC621C51E205020D2
:10A3FC00930554007C803E207C8189477C829307A6
:10A40C0080025C839760FB1FE78020F25C208A85CA
:10A41C0026857C84EFA0CFF02A8411C53245976045
:10A42C00FB1FE78060CE2285F2406244D244056176
:10A43C0082804D44CDBF5D7186C6A2C4A6C2CAC07F
:10A44C004EDE89476306F600C14709446318F604DB
:10A45C000144A9C52E894C0832C6B689AA84812725
:10A46C002A84324605EDC1778507CA851305D101CB
:10A47C003ECC230EC1009760FB1FE78000EB2C083D
:10A48C002685B9372A8419E95245B75604004E87F8
:10A49C00938626B11D462C08EF00900A2285B64003
:10A4AC00264496440649F25961618280797122D41E
:10A4BC0036844AD04ECE52CCB2892E8A3A89814605
:10A4CC00130710022286D94526D206D6AA84EFF0AD
:10A4DC009FE12AC621C12286CA85608423124101CC
:10A4EC00231331019760FB1FE78020E44C00268585
:10A4FC00EFA0FF832A8411C532459760FB1FE780CC
:10A50C00A0C02285B250225492540259F249624A98
:10A51C00456182804D44F5B7011122CC26CA06CE86
:10A52C004AC8DD472A84AE846389F50281470A2034
:10A53C006C005C86EFA07F8305456380A40808242B
:10A54C00B165938505B8EF908F90E5473CA0B75760
:10A55C0004009387C7D65CC085A058393149B286B0
:10A56C003306270318499C4232971043E310F6FC3C
:10A57C00DE225223E31CF6FA8C4608479760FB1F39
:10A58C00E780A0EB45D55C385828850793F7F70F83
:10A59C005CB863FAE702B387270318480A20BA9716
:10A5AC009847D623B2238E23113749F10824B1657D
:10A5BC00938505B8EF90AF895945F2406244D24477
:10A5CC004249056182807C289DB7011122CC26CAA4
:10A5DC0006CEDD472A84AE846394F5060A21EFA0EB
:10A5EC000FA1522C36285A286D162A964206418203
:10A5FC00B307D640C20752ACC18363FAE706930592
:10A60C00C5FF3308F7406359B802BA96918EC2065B
:10A61C00184C0E280A20C1823E97EFF03FE90DE15D
:10A62C000824B165938505B8EF906F825945F240C7
:10A63C006244D244056182806D1593160501C9BF31
:10A64C0081470A206C005C86EFA02FF20545E38061
:10A65C00A4FE0824B165938505B8EF805FFFE5473C
:10A66C003CA0B75704009387C7D65CC0C1B78547D9
:10A67C00C9BF397126DAAE842C0022DC4AD84ED6FA
:10A68C0006DE2A89B289212B2A8439E54A85EFA076
:10A69C000F96D6206D1563C5A60093160501C182D1
:10A6AC009844B2208E204A85EFF05FE02A840DE5B5
:10A6BC003146A6850808230601009760FB1FE7803A
:10A6CC00C0C6BE202245B75604004E87938646D09E
:10A6DC005D466C00FC86AD252285F2506254D25446
:10A6EC004259B2592161828069B761B7797126D21A
:10A6FC0006D622D44AD04ECE52CC56CA5AC8894419
:10A70C00D9C951CA2E842A89BA8A368B328AEFA0CB
:10A71C000F8E93054400814771159A21635EA7083B
:10A72C00850793F7F70FB105E319FAFE8A854A8579
:10A73C00BD21AA842DE131453305AA02916593858B
:10A74C001570CD449760FB1FE780008FAA8921C547
:10A75C0031463306CA02A2859760FB1FE780E0BC36
:10A76C001844562032200E204A85EFF03FD4AA849C
:10A77C0015ED0245B756040085475687938646D09B
:10A78C005D464C005C824EC423064101A3060100C9
:10A79C00230761017523B250225426850259925425
:10A7AC00F249624AD24A424B456182804E8597609B
:10A7BC00FB1FE7806095C5B7ED44F1BF79714ECEB4
:10A7CC0037F60600AE89C16526D20147AA848946B0
:10A7DC00130606C9FD15054522D406D64AD0EF103E
:10A7EC00407B054429C92A8913073002814611464A
:10A7FC00F5452685EFF03FAF2AC655440DCD83575E
:10A80C00A900CE8601467C8491477C8585471CA196
:10A81C00B2472C002685A38007003247FD573CA386
:10A82C0032473CB3EF10606C2A8411C532459760F7
:10A83C00FB1FE780608D2285B2502254925402593E
:10A84C00F24945618280411106C6EFF0EFE019C56F
:10A85C00B24041011763FB1F6700038BB2404101FB
:10A86C008280011106CE2AC6EF905FDF3245B737E2
:10A87C00002023AE07FAB737002023A007FC914530
:10A88C00B7370020A38EA73EEF30001FF2400561C2
:10A89C006F2050067971939705014AD006D622D4C1
:10A8AC0026D2C187014963DB070AB737002003C5ED
:10A8BC00D73F2E899760FB1FE780C09C2A8441CD2F
:10A8CC0018219307000A6315F70885474C08DC85A7
:10A8DC00EF907FE5AA8405ED8347610171476376AC
:10A8EC00F708138717FE1377F70F9306000263F52B
:10A8FC00E608858BCDC7B737002083A7C7FB9944E3
:10A90C0099C72A201306B1004C088297AA849C850B
:10A91C0099C7084409C59750FB1FE780E07E95E076
:10A92C005247B7070001938707F07D8FB7071200D6
:10A93C0093870710630EF70003476101ED47631916
:10A94C00F7002A208545EF30800ACD476388F40054
:10A95C002285EF809F8EA1673349F900B2502254B3
:10A96C004A85925402594561828037073014050795
:10A97C003357F700058B35DF37370020032707FCEB
:10A98C0059D70347510141F75C8699472308F100D9
:10A99C002A206C0023170100EF90DFFB8DBFB73727
:10A9AC00002083A707FC8DC32A201306B1004C0896
:10A9BC00829731DDAA8483475101B1FB8347610142
:10A9CC00230891005C86E9B79944F5B7397122DC0C
:10A9DC0026DA06DE4AD84ED652D456D25AD0A547DD
:10A9EC002A84B2846398F50E834745021A22835A4F
:10A9FC00260085072302F5029307F7FFB387FA02B7
:10AA0C005442C207C183B69703C917009C2354252F
:10AA1C0022093369F90085476390F602330757031F
:10AA2C00231006008149014A130B3501931A0701C3
:10AA3C0093DA0A0163EA5905C167FD176303F90A42
:10AA4C001E286370F90A0509420954241359090197
:10AA5C002317240105470A209305E400639CE600B4
:10AA6C007C85930720307C86930780022314210178
:10AA7C005C872C00EFA08F910824B165938505B8F5
:10AA8C00EF80FFBC5945B9A8B620DC402C28ED1648
:10AA9C0013865900C206C1823E965A85EF901FC19B
:10AAAC0005C5630B3A01C840B220B3053501529578
:10AABC009760FB1FE7806087BE203E9A9E20420A6B
:10AACC00135A0A0185079EA0BE20BE99C20993D9CC
:10AADC0009018DB75822A9476310F7028347450235
:10AAEC0081CF0145F2506254D2544259B259225A84
:10AAFC00925A025B2161828034281309340137F5A4
:10AB0C0006004A868945130505C8EF903FBA19C15E
:10AB1C000545C9BF342837F506004A868945130513
:10AB2C00C5C8EF90BFB86DF5342837F506004A86D6
:10AB3C008945130545C7EF907FB779F9342837F568
:10AB4C0006004A8689451305C5C5EF903FB669F1E5
:10AB5C00D820BD47E3EEE7FAA56793874712B3D732
:10AB6C00E700858BD5D78347440285072302F4027F
:10AB7C0003D92400D1B5011106CE2EC69760FB1F58
:10AB8C00E78020E611C93C25B24513871700639571
:10AB9C00E50093F707F83CA5F240056182800111AE
:10ABAC0006CE2EC69760FB1FE780A0E31DC1B24501
:10ABBC0091C188C11C251307E00F5D456388E70030
:10ABCC001307F00F01456383E7005945F240056117
:10ABDC0082800945E5BF411122C42A84210506C69D
:10ABEC0026C24AC0EFF0EFBC3C20A51793F7D70F55
:10ABFC0089EB58248547631EF7041C48814431496E
:10AC0C00A1E3FD57230104001CB423020402130525
:10AC1C00C4002244B240924402496146814541013C
:10AC2C001753FB1F67000377B38724033E95084532
:10AC3C0009C59750FB1FE780204D850493F4F40F52
:10AC4C005C280848E3E2F4FE9750FB1FE780C04BFA
:10AC5C004DBF084C75F975B7411122C4416406C645
:10AC6C0026C29307E4FF6301F502AA849DE1976075
:10AC7C00FB1FE78000D709E91305F4FF9760FB1F62
:10AC8C00E78020D611C106A1B24022449244410172
:10AC9C00828085476392F5049760FB1FE78060D440
:10ACAC002A847DD1FD571EA11C241307F00F63824B
:10ACBC00E7021307E00F6389E700342008340147EB
:10ACCC005146A685EFF02FA12285EFF0DFF0FD575E
:10ACDC001CA4230504004DBF8947E397F5FA85456D
:10ACEC00EF40E04155F126859760FB1FE78060CF70
:10ACFC002A845DF951BF21C518259307F00F630015
:10AD0C00F704011122CC06CE2A8434210E210835F9
:10AD1C0001475D46EFF02F9C3820E1476318F700A0
:10AD2C000A206C0023060100EFA02F84F9571CA405
:10AD3C002285EFF05FEAF2406244056182808280F6
:10AD4C009307F00F6306F706011122CC26CA2A845A
:10AD5C004EC6AE84B689AA859306850037B5040025
:10AD6C004AC852C43A89328A130525D0794606CE90
:10AD7C00EFF06FA3A3042401230144012322340127
:10AD8C0085C01305C4006244F2404249B249224ACC
:10AD9C00A685D244614605611753FB1F6700E35833
:10ADAC00F2406244D2444249B249224A056182804F
:10ADBC008280B73700202384A7FC82809547639458
:10ADCC00F50683474502854685072302F5021E22B8
:10ADDC0058423022FD17C207C1836312D6048A077A
:10ADEC00BA9798339C232207D98F7A2563F5E70409
:10ADFC00411106C622C485075EA52A849305C500A9
:10AE0C000A21EF905FCF0824B165938505B8EF80D8
:10AE1C001F84B2402244D9473E8541018280C946F5
:10AE2C00B387D70275BF5422294785476396E6003E
:10AE3C000347450211C381473E8582809D47639B32
:10AE4C00F50483474502762585072302F5021E2269
:10AE5C005842FD178A073E971C331823A207D98F37
:10AE6C00014763F2D704411106C622C485072A8420
:10AE7C005EA59305C5000A21EFF08FD50824B165B6
:10AE8C00938505B8EF80AFFCB240224459473A8510
:10AE9C00410182805422A94705476396F600034777
:10AEAC004502133717003A858280411122C406C629
:10AEBC0026C2B5472A846395F50483474502B284BC
:10AECC0085072302F5020A21EF907F929E2013073B
:10AEDC00F5FF014563C1E7027A240A209305C400FB
:10AEEC00BA977EA4EF903FCF0824B165938505B83F
:10AEFC00EF80EFF55945B2402244924441018280E3
:10AF0C0058229D470545E318F7FE034544021335C7
:10AF1C001500D5B7C5476396F5061E223A22FD17D4
:10AF2C00B387E7020347450205072302E5025842AF
:10AF3C00C207C1833E973C333823A207D98F4167A0
:10AF4C007D176395E70081473E8582801387170044
:10AF5C005AA57A25E3F9E7FE411122C49305C500F1
:10AF6C002A840A2106C6EF901FD00824B165938568
:10AF7C0005B8EF80CFEDB2402244D9473E85410160
:10AF8C008280542229478547E390E6FC034745021B
:10AF9C005DFB5DBF011122CC26CA4AC852C406CE45
:10AFAC004EC6BC2115472A8AAE8432843689639AF0
:10AFBC00E7043686A2852685EFF05FE0AA8955E581
:10AFCC0085476314F40A03474900A9476300F70255
:10AFDC0088344A8785460146D285EFE0DFEF19E5D4
:10AFEC0085454A85EFE05FE713341500B4208834BB
:10AFFC0001476946D285EFE01FEE2685EFF0BFBD15
:10B00C0049A01D476398E7003686A2852685EFF098
:10B01C00FFE26DB725476398E7003686A285268543
:10B02C00EFF0DF9A61BF35476398E7003686A2855B
:10B03C002685EFF09FE759B745476398E7003686BA
:10B04C00A2852685EFF01FED95BF5D47639EE70057
:10B05C00D82585473686A2852685631DF702EFF035
:10B06C00AFCB8547631AF5048549A5476317F402EE
:10B07C00835709009DE30544E38A09F6D947E39E0B
:10B08C00F9F62285F2406244D2444249B249224A3E
:10B09C0005618280EFF06FD3E9B788344A87A286C6
:10B0AC000146D285EFE03FE379F5A2854A85EFE0D2
:10B0BC00BFDA13341500C9B70544E1B7397122DC86
:10B0CC0006DE26DA4AD84ED652D456D29E211944E0
:10B0DC00B9E783C925002A89328A938759FE93F7E9
:10B0EC00D70FAE84DDE3B737002083C687FC130788
:10B0FC00F00F938A87FC19446383E602F547639546
:10B10C00F9049760FB1FE780C08DAA891DCD3025FF
:10B11C000DCE93178601E18763DD0700014422857C
:10B12C00F2506254D2544259B259225A925A216165
:10B13C008280F5454A85EFE07FE283C7A90093E75B
:10B14C0007F82385F900D9BF8149D62090448C306B
:10B15C0088203800EF907FC22A8471F1B42003C597
:10B16C000A0038000146CA85EFE0FFD62A8445F96B
:10B17C00B24799C323000A00BC207547E390E7FA55
:10B18C00E38E09F82385F90059BF9760FB1FE78010
:10B19C004085AA8A41D58547639FF908CE2088440B
:10B1AC003000EF90AFE62A843DF903C72A00C5476B
:10B1BC0063FFE708DD47630DF70AB737002003C5C7
:10B1CC009A0083C7D73F6398A70A014403C72A0094
:10B1DC008D47631EF7043C8403D7CA0063F4E70071
:10B1EC002396FA0083D5CA004A85EFF02F8AB73729
:10B1FC00002083D7C7246D47637BF70283D5CA0031
:10B20C005D476376B7021387350091056349F700F4
:10B21C001307B00FBE856374F7009305B00F11666A
:10B22C00C20513060629C1814A85EF80A01C5685EC
:10B23C00EFF07F9AEDB53C211144E39237EF5C417E
:10B24C00E38F07ECCE20884430008297A9BFB72744
:10B25C0002009387072AB3D7E700858BB9DFB020AC
:10B26C003400D6854A85EFF0FFD22300AA0045BDF5
:10B27C0083A70A01E5B7B42038000146CA85EFE080
:10B28C009FC52A8421F5AC202800EFE0FFBC15DD1A
:10B29C0023000A0025BF011122CC3734002006CE32
:10B2AC0026CA4AC84EC652C49309C43F03C5890076
:10B2BC009307800291653305F502938565703739E4
:10B2CC000020930449FC9750FB1FE780E0D603C68F
:10B2DC0089009307800281453306F60288C0975097
:10B2EC00FB1FE780200B9C404D459DCF9304C43F32
:10B2FC00130949FC0144130A8002FD599C24636D17
:10B30C00F40237B504001305850CEFE0FFF637B5F2
:10B31C000400130525B8EF90CFBF37B50400130513
:10B32C0045C6EF30D0540145F2406244D244424904
:10B33C00B249224A05618280B30744030325090000
:10B34C006146814505041374F40F3E9523103501B5
:10B35C0023010500231435012305050023020502F2
:10B36C0031059750FB1FE780E00249BF0145828001
:10B37C00B737002083C65740814763E5D7000147A4
:10B38C003A8582802E87910503D6C5FFE30AA6FE77
:10B39C008507E5B70DC93C210547890793F7F70FDA
:10B3AC006373F702411122C406C62A840E21283188
:10B3BC000147F9465D46EFE01FB2F9573EA0B24097
:10B3CC002244410182808280B737002003C7574056
:10B3DC00FD56814763E3E700828016A12301050037
:10B3EC0085071105C5BF014582803736002013063D
:10B3FC00F6F3930700021CA237370020FD57230FEA
:10B40C00F7F2373700202308F7F237370020A3076D
:10B41C00F7F28545B7370020239EB7F2B7370020E7
:10B42C00239507FCB737002023AA07FCB737002069
:10B43C0023A207FEB737002023AC07FCB736002049
:10B44C00B7F70600938646F3938707C7DCC2B73776
:10B45C000020238607FCB7370020938787EC094729
:10B46C0098A298A398AB2380E7022388E70237F7CA
:10B47C000600130707C6D4C7D8DBB7F606000D477E
:10B48C00238CE7029386C6C537370020D4CB03271D
:10B49C0007FD37F50600B7F60600130505C89386B9
:10B4AC0006C9C8C38CA7239507008CAF239D070042
:10B4BC00D0CFD4D3238407022395070223A60702F7
:10B4CC00239D0702D8DFB737002037B704009387D6
:10B4DC0087F01307875923A00700D8C323A40700BC
:10B4EC008280411106C6EFF0BFE809C52821B240A1
:10B4FC00410182800145E5BF411122C426C24AC0E8
:10B50C0006C6AA842E893284EFF09FE609E94165CC
:10B51C00CA857D15EFF0DFE5C54701C506A120A161
:10B52C008147B2402244924402493E8541018280C7
:10B53C0039E38948354763911605011106CE22CCB3
:10B54C0026CA1832102293C7F7FF2207598EF18FA3
:10B55C0032C68DE7C4452A84A685EFF09FF83246A3
:10B56C000147630FA60022856244F240A685D244AF
:10B57C0005616FF07FF82D473A858280130700082C
:10B58C00F2406244D2443A850561828083C805004A
:10B59C0009486395080303A845008347180003482E
:10B5AC000800A207B3E70701C2070D68C18713089B
:10B5BC0028906395070189476FF09FF705458280B6
:10B5CC00011122CC37340020130404F3182006CECA
:10B5DC0026CA4AC84EC69307F00F630FF702AA8912
:10B5EC002945B2842E899750FB1FE78040C40DC5B6
:10B5FC009307100B1EA12302050023113501231301
:10B60C00250106A5AA8508206244F240D24442498D
:10B61C00B24905616F705FC7F2406244D24442493F
:10B62C00B249056182804111B737002026C2AE8431
:10B63C0083A507FD22C406C62A84EFF09FEA098978
:10B64C0009C922852244B240A685924441016FF07B
:10B65C00EF96B2402244924405454101828041114B
:10B66C0022C426C24AC006C6AA8413044500130984
:10B67C00850B1E209DC3084409C59750FB1FE7800E
:10B68C00A0A82285314681459750FB1FE78080D0CA
:10B69C003104231A04FEE31E24FDB2402244FD575C
:10B6AC009EA00249924441018280B737002003C614
:10B6BC005740B737002003A7C7FD81476315F60035
:10B6CC00814636858280BA861307870B835587F4AB
:10B6DC00E389A5FE850793F7F70FCDB7B7370020A1
:10B6EC0083A747FE81CBDA236314A70088478280A7
:10B6FC009C43CDBF01458280411106C6EFF01FFE71
:10B70C0009C50845B240410182800145E5BF0111E0
:10B71C0026CA9384450022CC4EC606CE4AC852C4D3
:10B72C0056C25AC0268781490144814681473D450E
:10B73C00122345CABDEE42233E23B286A297C2070E
:10B74C00C18385093107E395A9FE35C42E8991651E
:10B75C009385457022859750FB1FE780E08D2A8BDF
:10B76C0039C9814A014A8C4495C1D22033054B0119
:10B77C009750FB1FE78060BBDE2088443E9A420A4C
:10B78C00135A0A019750FB1FE780009863890A003F
:10B79C003146814526859750FB1FE780A0BF850A5F
:10B7AC00B104E3E23AFD232669012314890005451F
:10B7BC0021A0630DD6000145F2406244D2444249B7
:10B7CC00B249224A924A024B056182803223E31429
:10B7DC00F6FE52233294B2974204C2074180C183D1
:10B7EC008DB70545E37A35FD8DB7B737002083A7B4
:10B7FC0087FD99E30145828098473A276315A70096
:10B80C001385470082809C43EDB7411106C6EFF0CB
:10B81C00DFFD09C50A21B240410182800145E5BF27
:10B82C00411106C6EFF07FFC09C52821B240410149
:10B83C0082804145E5BF411122C42A842E8506C66B
:10B84C00EFF01FFEAA8505462285EF30406B954729
:10B85C006305F500BD476313F5002145B240224452
:10B86C00410182804111B737002022C406C603A4CF
:10B87C0087FD8146938787FD21C0184432271840E5
:10B88C006317A60285CA98C22E8581C921469305E5
:10B89C0044009750FB1FE78040A922859750FB1F5F
:10B8AC00E78080860145B240224441018280A28615
:10B8BC003A84D9B798C3C9BF0545F5B737370020C7
:10B8CC00832747FE0146130747FEA9C703D8470045
:10B8DC009443631CA802011106CE22CC26CA0DCAC1
:10B8EC0014C2AA843E852E849750FB1FE780C0812A
:10B8FC002C002685EFF01FF701E519C0B2471CC0DC
:10B90C00F2406244D244056182803E86B68775BFA0
:10B91C0014C3C1BF05458280411122C42A84090584
:10B92C0006C6EFE00FE9FD573CB0B240224441019E
:10B93C008280411122C4416406C626C29307E4FFEB
:10B94C006301F502AA849DE19750FB1FE780800CF0
:10B95C0009E91305F4FF9750FB1FE780A00B11C1F9
:10B96C0006A1B240224492444101828085476392F1
:10B97C00F5049750FB1FE780E0092A847DD1FD5721
:10B98C001EA13C201307F00F6382E7021307E00FA0
:10B99C006389E70028300147F9465146A685EFE058
:10B9AC008FD32285EFF05FF7FD573CA023020400F4
:10B9BC004DBF8947E397F5FA8545EF30407455F153
:10B9CC0026859750FB1FE780E0042A845DF951BF60
:10B9DC001D71A6CACEC686CEA2CCCAC8D2C4D6C247
:10B9EC00DAC05EDEAE84AC21F947AA896397F50410
:10B9FC009750FB1FE78000022A8411ED0144228539
:10BA0C00F6406644D6444649B649264A964A064B01
:10BA1C00F25B256182803C210547890793F7F70F7C
:10BA2C00E37EF7FC28310147F9460146CE85EFE06D
:10BA3C008FCA2285EFF05FEED1B703AB0400B707D6
:10BA4C000001938707F037071200B377FB00130749
:10BA5C000710B28A0149638BE7022EC69750FB1F71
:10BA6C00E78040FB2A89B24515C1502105C29317C6
:10BA7C008601E187E3C407F84E85EFE02FCE8347BC
:10BA8C00490093E707F82302F9008DBF373A0020ED
:10BA9C000347EAF39307F00F130AEAF31944E300A0
:10BAAC00F7F6E147E3EDB7F493D71500FD171397BD
:10BABC003700B7E706009387075ABA9703A8070021
:10BACC00E30F08F283AB4700E38B0BF2420B135BE3
:10BADC000B0163050B00C947E393F5F2D6209044A4
:10BAEC008C308820380802982A8411F92C084E854D
:10BAFC00829B2A8431C19C30E39307F0BC20230A3B
:10BB0C00A10039472308F1006396E70262471C3312
:10BB1C001823A207D98F0C084E85FC81EF809FE378
:10BB2C00E30E05EC14080546D9454E85EFE04FE1D0
:10BB3C002A84F1B5BC84C5B7B4209147E380F6ECF8
:10BB4C0003450A0038080146CE85EFE0CFB82A84B9
:10BB5C00E31705EAAC202808EFE00FB019C12380E9
:10BB6C000A009840B7070001938707F07D8FB7074D
:10BB7C00120093870710E303F7E8E30109E8BC2000
:10BB8C002302F900ADBD011106CE2EC69750FB1F46
:10BB9C00E78040E811C95C21B24513871700639513
:10BBAC00E50093F707F85CA1F240056182803971DA
:10BBBC0052D42E8A4ED69305E101AA89528522DCF5
:10BBCC004AD856D206DE26DA328936C63AC4BE8A3E
:10BBDC009750FB1FE780C0E6054435C1AA84A887AF
:10BBEC003944EFF0BFAF21CD0328450063090804A9
:10BBFC002247B246D6874A86A6854E8502982A8465
:10BC0C001DED9307E00F638CFA02982089476318A7
:10BC1C00F702D8401C331823A207D98FC2070D672F
:10BC2C00C18713072790639CE700834719000346DD
:10BC3C000900D285A2075D8E4E85EFF07F98228594
:10BC4C00F2506254D2544259B259225A925A21613A
:10BC5C008280797122D422214ECEAA89228556CA9D
:10BC6C0006D626D24AD052CC5AC85EC662C4AE8A18
:10BC7C00EFF0BFA301E92285EF908FD9594431E54C
:10BC8C000144A1A003C789008547AA840144631716
:10BC9C00F702AA8513858900EFF07FA729C9FA203E
:10BCAC009624D044CE2003D52900E147EFF03FF095
:10BCBC00D9472A846318F50223A604002685EFF0E1
:10BCCC001F9A41C0D947E30DF4FA2285B250225491
:10BCDC0092540259F249624AD24A424BB24B224C1C
:10BCEC004561828061DDDE202390FA00C1BF13899B
:10BCFC004400014AB94B594C3D4B83550900DDDDDD
:10BD0C00E14763067A010357C90011C3D9470357AA
:10BD1C002900835649000326890003D52900EFF03A
:10BD2C001FE92A846319850123240900050A3109B6
:10BD3C00E3156AFD61B77DD9835709002390FA009A
:10BD4C00F5B703D529000DBF011170879307E00FDC
:10BD5C001306E1000147894606CEEFF05FE5F2409D
:10BD6C0005618280797122D42A840A2526D2AE8478
:10BD7C009305210106D64AD09750FB1FE78040CC93
:10BD8C0079C51C252AC693F707029DC7A881EFF039
:10BD9C00BF96AA87B24511E91E2439459EA0B25020
:10BDAC00225492540259456182802A204946829736
:10BDBC0001C51E249EA0E5B7035924004A85EFF067
:10BDCC00DF8E01ED41657D15EFF03F8E09E51E24F8
:10BDDC0025459EA0E9B7231025011307450081478F
:10BDEC00BD46122339EE3147B387E70213098400AD
:10BDFC003146CA8591073E959740FB1FE780E0527C
:10BE0C003146CA8548089740FB1FE78000525224F0
:10BE1C002A2041478146DD45EFE0EFCC2ACE09E5EB
:10BE2C001E2445459EA0A5BF0C4852249740FB1FDD
:10BE3C00E780A04F2A204C08EF904FB92DD15945DF
:10BE4C00B9BF85073107E39ED7F825459DB7054552
:10BE5C008DB7797122D42A840A2526D2AE84930513
:10BE6C00E1014AD006D632899750FB1FE78040BDCE
:10BE7C002DC91C2593F7070295EF18389307200559
:10BE8C0011E35C20362450440E242A200147EFF0A5
:10BE9C001FD2AA8729E11C3891E72A20EF900FAF17
:10BEAC00D94711E18147B2502254925402593E8530
:10BEBC00456182802AC6A887EFF01F84AA8705C532
:10BECC00B2452A2049468297AA8745D91A249AA0B6
:10BEDC00183869FBC9BF5947E31AE5FE230009006E
:10BEEC00D1B78547E5B7B947D5B7397122DC4AD800
:10BEFC004ED652D406DE26DAAA892E8A32C6368966
:10BF0C009750FB1FE78000B109440DC53C21130776
:10BF1C00E00FAA845D44638FE7001307F00F5944C8
:10BF2C00639AE700324605E2D2854E85EF906FB2F8
:10BF3C002A841DCD2285F2506254D2544259B259F2
:10BF4C00225A2161828003550A009305E101231FC7
:10BF5C0001009750FB1FE780A0AEA887EFF05F8C25
:10BF6C00AA8505464E85EF2090792A8455DDD9B7F0
:10BF7C009307F00FE300F9FC37B504009386240017
:10BF8C007946A6851305053AEFE0EF81A3812401DC
:10BF9C0055B73971B737002026DA83A487FD52D400
:10BFAC005AD05ECE62CC06DE22DC4AD84ED656D2B1
:10BFBC0066CA2A8BAE8B328C368A99E08149A9A04D
:10BFCC00804483DC44000149835AA4006314990122
:10BFDC008440E5B73E24A28963F86701050942094C
:10BFEC00135909014104DDB7E3EAFBFE630B0A00B8
:10BFFC000C204840D28662863AC6EF802FEB32473F
:10C00C0071DD19C323105701F25062544E85D2547E
:10C01C004259B259225A925A025BF24B624CD24CA0
:10C02C00216182809A21B621854763E5E60439C3F4
:10C03C004111D42126C237F506009384550022C441
:10C04C0026862E84130505C8894506C6EF800FE6A3
:10C05C00C14719C954202E200A2001472686EFF02B
:10C06C005FF3814711E1A947B240224492443E85D7
:10C07C00410182803E8582802E860A22AE21854730
:10C08C0063E1A50219CD542241110147150606C6DC
:10C09C00EFF03FF0814711E1A947B2403E854101E5
:10C0AC0082803E8582802E860A22AE21854763E1FE
:10C0BC00A50219CD542241110147150606C6EFF011
:10C0CC005FED814711E1A947B2403E854101828075
:10C0DC003E85828039714ED6BE2183D9050006DE9D
:10C0EC0022DC26DA4AD852D456D25AD05ECE62CC52
:10C0FC0066CA6AC863EA3715854763880912416BBB
:10C10C00AE8A2A8A2314010002C6014401497D1B10
:10C11C00894B054CC94C054D83D52A0001478146F6
:10C12C0001464E8523130100EFF0BFE6AA84630B92
:10C13C00050E09EC13072002930661005A869545FB
:10C14C005285EFE04F9A2A846302051038849C20B4
:10C15C0041CB18856305A70741476385E7022C008F
:10C16C005285EF80BFD309CD34001546D945528591
:10C17C00EFD01FFD11C532459740FB1FE780C0F87B
:10C18C00814765A0BE244146130524001CA0BE2493
:10C19C00A1831CB0CC409740FB1FE78000194904D9
:10C1AC003C848507C207C1837C8463FD2707BE24BA
:10C1BC00638A67078509C20993D90901B1BFE39066
:10C1CC0077FBBE240946130524001CA0BE24A183C2
:10C1DC001CB0CC409740FB1FE78020151104C9B759
:10C1EC0022C603596100B82413052400638F77011C
:10C1FC00335999032305710118A0BE244146A1832C
:10C20C001CB0CC401379F90F79B72305810118A024
:10C21C00BE24135929001379F90FA1831CB00946C8
:10C22C00CC404DBF3C8485FFA947F2506254D25498
:10C23C004259B259225A925A025BF24B624CD24C7E
:10C24C00424D3E85216182808547C5B7C547F1BF08
:10C25C00B737002003C727FF854763F4E7060111B2
:10C26C0022CC26CA4AC806CE2A843289AE8497408C
:10C27C00FB1FE780207A19C538219307E00F5D4535
:10C28C006308F700631C0900A6852285EF801FF95F
:10C29C00F2406244D2444249056182808A2093056F
:10C2AC00E100231701009740FB1FE7806079288786
:10C2BC00EFF00FD7AA8505462285EF20504469D5AB
:10C2CC00C1BF5945828013F7050201C7B2856FF0D3
:10C2DC008FD6411126C24AC006C622C413F9850066
:10C2EC00AA8463170900139785016187635B0702B2
:10C2FC0032853684EFF0CFD2AA8505466313090048
:10C30C0001462685EF20B03F01E90145B2402244A9
:10C31C0092440249410182801C34EDDB1C24F5F768
:10C32C00F5B793F72500F5F30D45CDB77971AE86CA
:10C33C0022D42A848A229305E10106D636C6974078
:10C34C00FB1FE780E06F19C90C25B246B087228528
:10C35C00EFF07FF7B2502254456182800545DDBF76
:10C36C0013F7050201C7B2856FF0EFCC411122C45F
:10C37C0026C206C693F485002A8491E4139785019E
:10C38C006187635007023285EFF08FC9AA85054695
:10C39C0091E0014622852244B240924441016F2033
:10C3AC00103693F72500014591E30D45B240224428
:10C3BC009244410182807971AE8622D42A848A22E9
:10C3CC009305E10136C606D69740FB1FE780406710
:10C3DC00B24611C90C25B0872285EFF07FF8B25018
:10C3EC002254456182800545DDBF797126D2AA842D
:10C3FC002A25C16722D44AD04ECE06D62317010077
:10C40C00FD173284B6890149630CF50005059420AB
:10C41C00D04042051307E1004181EFF09FB72A8914
:10C42C009420D04037F506008945130505C8EF80E8
:10C43C00EFA715C5A2242285EFF02FBD09C57D14E9
:10C44C002A94420441806384090023908900B250ED
:10C45C0022544A8592540259F249456182809420B3
:10C46C00D04037F5060089451305C5C8EF800FA4E9
:10C47C0071F19420D04037F5060089451305C5C5E8
:10C48C00EF80CFA211C9E30809FA3C87E39587FA3C
:10C49C000354A9007D1475B7A22475B7397122DC39
:10C4AC0026DA4AD84ED652D456D25AD062CC06DEB0
:10C4BC005ECEBE899C252A8AAE84C18B328C368492
:10C4CC003A89C28A468B9DE783CB04008947638BEC
:10C4DC00FB046285EFF08FA01DC1832805006380EB
:10C4EC0008025A88D6874E87CA862286A685528528
:10C4FC00829839A03285EFF02FA0AA8711ED39452B
:10C50C00F2506254D2544259B259225A925A025B96
:10C51C00F24B624C216182802946A6855285829716
:10C52C0045D5F9BFD8401C331823A207D98FC207B1
:10C53C000D67C187930607906383D71E63CCF606FD
:10C54C0093062780638ED70A63C0F6021307078011
:10C55C00E3C1E7F82D45E39509FADC449023CC437D
:10C56C002310C9002285B9A213073780E393E7F69D
:10C57C002D45E39709F885472310F900DC448145E4
:10C58C009C231CA0AA240505420541819740FB1F52
:10C59C00E780004B835709006310051091072310A7
:10C5AC00F90011468145130514009740FB1FE780E5
:10C5BC0060DEF1A8930627906386D71463C1D71069
:10C5CC0093063790638DD71413074790E393E7F0E6
:10C5DC002D45E39709F2DC441D472310E90098230D
:10C5EC0018A0983318B0BA2338A0BA23218338B0D6
:10C5FC00D82358A0FA2358B0FE23A1837CA041A8CD
:10C60C002D45E39F09EEDC446C0083C91700982389
:10C61C00A209B3E9E90011472310E9009C234E85D8
:10C62C001CA0DC449C331CB09740FB1FE7804041AE
:10C63C00AA8425C13086C1659306E100FD158329C6
:10C64C00C500EFF09FDA09ED9420D04037F50600D5
:10C65C0089451305C5C8EF806F8519E1FD577C87A7
:10C66C0003C7090089476310F70283A549000946EF
:10C67C00130544009740FB1FE78020CB835709002C
:10C68C0089072310F9003C873CA0A1833CB00145ED
:10C69C0085BD23173101C5BF18218907BA9723100F
:10C6AC00F9003E251CB03E25A1833CA010214C4135
:10C6BC00130534009740FB1FE78020C7C9BFC8444F
:10C6CC009740FB1FE780E0CF93170501C1832A87B2
:10C6DC001D45E3E737E36399F90023100900CC44C7
:10C6EC0003560900CE95BDBD4207B3863A0141837E
:10C6FC0063C7E600B38737412310F900CDB7231089
:10C70C005901F1BF2D45E39D09DECC445285EFE084
:10C71C005FDD2310790108A0218108B08DBF2D4564
:10C72C00E39009DEDC44231079019C231CA0DC443B
:10C73C009C331CB0A9BF1D71CAC82A892A21A2CC5E
:10C74C00CEC6D2C4D6C2DAC05EDE62DC66DA6ED683
:10C75C0086CEA6CA6AD8AE8AEF806F89130CF5FF15
:10C76C0093170C01B73B0020C1832A8A814913849B
:10C77C004B1A3EC6373B0020B73C0020C16D835797
:10C78C00C90063F5F9001E2063CC8701035529000D
:10C79C0093854B1AEF807F942A8D15CD594D25A882
:10C7AC0083278900139719009305E101BA97843305
:10C7BC009C23A204DD8C26859740FB1FE780402834
:10C7CC00AA8515E923909A004840054D09C5974064
:10C7DC00FB1FE7806093F64066446A85D644464961
:10C7EC00B649264A964A064BF25B625CD25C425DC5
:10C7FC00B25D2561828032488348490083A64CFD96
:10C80C00B0870355290081471307ABFCEFF01FC914
:10C81C002A8D13884CFD09C523909A0048407DB79A
:10C82C005C4085E703552900514781461386FDFF7F
:10C83C00BD45EFD05FABB737002048C0138847FD2C
:10C84C0009E523909A00454D79B71E200357ABFCA0
:10C85C009304ABFC3E976346470113C7F7FF52970F
:10C86C009AA048409220832508003E958509974060
:10C87C00FB1FE78080AB1E209A20C20993D90901C7
:10C88C00BA971EA0EDBD397122DC2A842A2106DE5E
:10C89C0026DA4AD84ED652D45AD05ECE62CC66CA6C
:10C8AC002E8B56D26AC8EF709FF42A8A54242E24F9
:10C8BC000A2478001306D400130CBAFF651AEFF0A3
:10C8CC004FED420A37390020AA898144135A0A01D4
:10C8DC00B73B0020B73C00201309491A63820904B6
:10C8EC0063D08405938A4CFD8348440083A60A00D8
:10C8FC0030862A20528881471387ABFCCE85138D56
:10C90C00ABFCEFF0BFB91DC1814A30862E244E8599
:10C91C009306E100EFF07FADAA8963990A065DFDED
:10C92C00F1E41E2429452310FB0035A883570D0084
:10C93C001228E31BF6FC83A50A0048489740FB1F0E
:10C94C00E780A0AF71D18327490095EF2A2041667B
:10C95C00454781467D169D45EFD0FF981DE11E246D
:10C96C0045452310FB00F2506254D2544259B2593F
:10C97C00225A925A025BF24B624CD24C424D2161CC
:10C98C0082802322A90083DAA90041B783274900BA
:10C99C00A6972380570193871400139707018327C9
:10C9AC004900418393DA8A00BA9723805701138791
:10C9BC002400832649009387340042079104418365
:10C9CC00C207C204C183C180369711C9348714A32E
:10C9DC0003274900BA973887218398A301B7FD56DE
:10C9EC0014A303274900BA9794A31DBF2A20B73577
:10C9FC00002089802392951A9385451AEF808FD554
:10CA0C003DD159458DB7411122C406C693F7050196
:10CA1C002A84328585C3EFE0BFE0AA8505462285CE
:10CA2C00EF20E04D95476305F500BD47631DF5020A
:10CA3C00214515A893F7450099CBEFE07FDE05461D
:10CA4C00AA8522852244B24041016F20404B93F7C6
:10CA5C00050489C7EFE0DFDC0146DDB713F51500EF
:10CA6C00133515000605B2402244410182807971CC
:10CA7C004AD04ECE52CC06D622D426D22A8AAE89A1
:10CA8C00014983D749006364F900014581A083A75C
:10CA9C00090013141900930414003387970018230A
:10CAAC00A297882322079305E100598D9740FB1F1D
:10CABC00E78000F905E583A7090005453E94182099
:10CACC0098A383A70900BE94982098B3B25022541F
:10CADC0092540259F249624A456182800C25308792
:10CAEC005285EFF05FF201CD83A709003E94182028
:10CAFC0098A383A70900BE94982098B3C1BF0509D9
:10CB0C00420913590901B5BF011122CC2A848A218B
:10CB1C009305E10006CE9740FB1FE78060F211C938
:10CB2C000C2530872285EFF01FEEF2406244056140
:10CB3C0082800545DDBF1D71CAC82A892A2186CE8F
:10CB4C00A2CCA6CAD2C4D6C2DAC05EDE62DC66DA79
:10CB5C002E8ACEC66AD86ED6EF707FC92AC6834697
:10CB6C00C9008355A9000355890078081306D9001C
:10CB7C00EFF02FC2B247B7340020416B938AA7FF66
:10CB8C00C20AAA8B014493DA0A01373C0020B73C55
:10CB9C0000209384441A7D1B63820B18B08683C5D6
:10CBAC008B0003552900EFF01FE6AA8D63130516C1
:10CBBC008348490083A64CFDB0860355290056884E
:10CBCC0081471307ACFCDE85EFF05F8DAA8D9309CE
:10CBDC00ACFC138D4CFD631E051215CC03D709005C
:10CBEC00BE2011076397E7003247A2976D1763C702
:10CBFC00E706B73500209387451ABA230355290059
:10CC0C009385451A3354E40282A3EF80CFD0AA8DCA
:10CC1C0015C1D94D05A003552900494781465A86AF
:10CC2C00C545EFD04FECC8C015E583D7AB00C54D5B
:10CC3C002310FA00F64066446E85D6444649B64940
:10CC4C00264A964A064BF25B625CD25C425DB25D50
:10CC5C002561828083D709009107BEA0DC4003D7F1
:10CC6C00AB009306E101A29798A3930714001397C6
:10CC7C000701DC4041835E85BA9703D7AB00218363
:10CC8C0098A3B0868355A900EFF02FF61307240064
:10CC9C00D44093073400420711044183C207420475
:10CCAC00AA8BC1834180369715EDFD5614A3D8404D
:10CCBC0083250D00BA9794A3C84003D6090022958A
:10CCCC009730FB1FE780606683D709003E944204CF
:10CCDC00418005F0835789002310FA00E39C0DF482
:10CCEC00A94D89BFB48783250D0014A3D840BA97EA
:10CCFC00B887218398A3C84003D6090022959730A2
:10CD0C00FB1FE780806283D709003E944204418078
:10CD1C0061B583D7AB002310FA0065BF814D55BFB9
:10CD2C005D71A6C2CAC0AA84035985002A21A2C477
:10CD3C004EDE52DC5AD85ED662D466D286C656DA3D
:10CD4C006AD06ECE2E8BEF709FAA930BD5FF711508
:10CD5C00131A0501B73900200144135A0A01373C54
:10CD6C000020B73C00209389491A635B7413D424C8
:10CD7C00AE241307E1001386D4004A85EFF06FA1AF
:10CD8C002A8D630F05100359A5000C253087AA20A6
:10CD9C00EFF07FC7631B051083C8440083A64CFDCE
:10CDAC003087AA20528881471307ACFCEA85EFF044
:10CDBC00EFEE930DACFC13884CFD65E905C883D7E9
:10CDCC000D0003D7290089076308F706B735002043
:10CDDC001387451A3E23AA209385451A3354F4022F
:10CDEC0002A3EF80EF9F0DC559451DA0AA204166F7
:10CDFC004D4781467D16A545EFD0EFCEB7370020C5
:10CE0C0023A2A900138847FD1DE123102B014545E2
:10CE1C00B640264496440649F259625AD25A425BAD
:10CE2C00B25B225C925C025DF24D6161828083D7C1
:10CE3C000D0089072391F90083D70D00A29763D1C8
:10CE4C00770783A749000357AD00930A2400A297E4
:10CE5C0098A305049317040103A44900C183C20AD3
:10CE6C003E948357AD008325080093DA0A01A18311
:10CE7C001CA003A5490003D60D0056959730FB1F47
:10CE8C00E780A04A03D40D00C167FD1756944204F5
:10CE9C004180E30CF9EC0509420913590901F1B57C
:10CEAC0029450DF423102B01A5B76DDC05B71E2108
:10CEBC0081E789473E858280411126C2444122C4C4
:10CECC0006C64AC09420D0402A8437F5060089450E
:10CEDC00130505C8EF708FFD11C93C202547E517D8
:10CEEC0093F7F70F6376F702E14721A89420D0401F
:10CEFC0037F5060089451305C5C8EF702FFB71FD8A
:10CF0C008947B2402244924402493E8541018280C5
:10CF1C00373900208356C9F385471309C9F3F5D275
:10CF2C001A203697C166E3CEE6FC91659385257091
:10CF3C0031459730FB1FE7802010AA84CD4771D173
:10CF4C00314681459730FB1FE780C0441E20835536
:10CF5C00090001460147B386E500C206C182636B36
:10CF6C00F702AE97C207C18319C22310F90023A0A0
:10CF7C0004002146A285138544009730FB1FE780EF
:10CF8C00C03AB7370020938787FD984309EF84C3D5
:10CF9C00814785BF50401315470005072A9636A6D2
:10CFAC00054655BF3E871C43F5FF04C399BF0111CD
:10CFBC0006CE22CC26CA4AC809E98944F24062440A
:10CFCC0026854249D244056182802AC62A842800DB
:10CFDC0036896C845085EFF09FEDAA8465F1E30FE0
:10CFEC0009FC3E24F9DB91659385557031459730EA
:10CFFC00FB1FE780600405C53E2423200500232485
:10D00C0025015EA1B7370020938747FE984301E7BF
:10D01C0088C36DB73E871C43F5FF08C345B7CD44A5
:10D02C0071BFB73700209387C7FC98230DE30547E2
:10D03C0098A3058909CDB736002037350020938693
:10D04C0086F041469145130585EC6FF05FF601457E
:10D05C008280B73700202388A7F28280C167FD1732
:10D06C006315F5002E856FE02FB6411106C6EFE073
:10D07C002FB009C5FD571EA123010500B240410187
:10D08C00828001114AC806CE22CC26CA85472A893D
:10D09C006392F5044A85EFE04FE131E9C16437F65C
:10D0AC0006009385F4FF1307E1008946130606C6B4
:10D0BC000545EFE01FEE2A84FD1405C44C444A8557
:10D0CC00EFF0DFF9308722858146A685EFF0EFB1CE
:10D0DC002A84E5B789476396F5008545EF20200241
:10D0EC0055D9F2406244D244424905618280EFE056
:10D0FC000FD76DB7011126CAB73400209384C43FF3
:10D10C0022CC8834373400201304C4FDB7370020F8
:10D11C003737002006CE4AC84EC62320040023A071
:10D12C0007FE232807FC59C1138907FE9307200C1F
:10D13C003305F502916593851570930907FD190563
:10D14C00420541819730FB1FE78000EF9034930735
:10D15C00200C81453306F60208C019069730FB1FD8
:10D16C00E78040231C40983481459386870B7D557E
:10D17C0063E8E5069306800BB306D7020146FD551E
:10D18C000507B6972320F900BE868EA2ACB2ACA2DE
:10D19C002382060005069906E369E6FEF95696A376
:10D1AC0099463307D702BA9723A0F90037C5040074
:10D1BC001305C59DEFD0EF8C37C50400130525B9B9
:10D1CC00EF70CFD537C504001305E593EF10306A27
:10D1DC00F2406244D2444249B24901450561828021
:10D1EC002394A6F41386C6F4231006002324060009
:10D1FC003106E31BD6FE85059386860B95BF411140
:10D20C0006C622C42A84EFC08FA7EFE00F9EB73763
:10D21C000020A38787F2B737002003A507FDEFE0B6
:10D22C00AF9AB7370020238F87F22244B24037D50C
:10D23C0004001305E50841016F1070639397050115
:10D24C00C18763D10730B737002003C5F7F2797176
:10D25C0022D45AC806D626D24AD04ECE52CC56CA62
:10D26C002E8B9730FB1FE780E0012A8429C51821FB
:10D27C009307000B631EF702B73400208547938495
:10D28C0044FDDC849C4023150100B9E3EF0080755C
:10D29C009165938535709730FB1FE780E0D988C086
:10D2AC0005E99C8491C74C2013058400EFD0AFD9BD
:10D2BC002285EF509FF8B250225421653345AB00C4
:10D2CC0092540259F249624AD24A424B45618280D9
:10D2DC00373A00206146814513054A1A9730FB1FE7
:10D2EC00E780400B03494400894793044A1AD289CA
:10D2FC00930A4A1A631AF904F5258AA02A20930581
:10D30C004A1AEF701FB63A209E20162401ED63E3F3
:10D31C00F6001EA40E243A85EFC05FF72285EFC0FD
:10D32C003FCC41B763E3F6001EA41E24D945938677
:10D33C00491A0D463A852390FA00EFC07FE08D45DF
:10D34C0071DD1385491A65A899476319F90293058C
:10D35C00A1002285EFF02FD3AA8469D1D947639E0F
:10D36C00F40C05092A201379F90FD9459386491A2B
:10D37C004A86EFC0FFDCCA8555D1E1B7A1476318D7
:10D38C00F9009305A1002285EFF09F99F1B7A94709
:10D39C00631AF9060A246C009730FB1FE780406A79
:10D3AC002A89630905122A2041669306E100554734
:10D3BC007D16AD45EFC03FF3C8C0AA8625CD834886
:10D3CC0044000358E10030862A20814713074A1A8B
:10D3DC00CA85EFF0AF8CAA84631F050C2A20930535
:10D3EC004A1AEF709FC51DD92A2093064A1A2D465A
:10D3FC00D945EFC0FFD41DD1AD4513054A1AEFD066
:10D40C008FC429BFB147631BF90C0A246C009730F9
:10D41C00FB1FE780E062AA8455CD2A204166930663
:10D42C00E10059477D16B545EFC0FFEB23A2AA00DA
:10D43C00AA8631E11E24C5447C851830D147E30F00
:10D44C00F7EC5C202A209385491A2380FA003C854E
:10D45C0023829A002391FA00EF70CFCFE30005EC02
:10D46C002A209386491A0546D945EFC07FCDE3079C
:10D47C0005EA8545F9B5834844000358E1003E248C
:10D48C0030862A20A68513074A1AEFF02F81AA842A
:10D49C001DE12A2093054A1AEF707FBFE30005E8CF
:10D4AC002A20D94593064A1A3546EFC07FC9B5459F
:10D4BC00E30605E679B5D9476393F400814403A5E7
:10D4CC004A009730FB1FE78020C4E38904E41E2444
:10D4DC007C85A5B71E2485447C8585B7B947631820
:10D4EC00F9009305A1002285EFF0EFA4B5B5C14773
:10D4FC006318F9009305A1002285EFF0CFE3A9BDD5
:10D50C00C947631AF900130691009305A1002285FF
:10D51C00EFE03F9491B5D947631DF9009305A10045
:10D52C002285EFE03F84AA84E31A05E2A3040100FC
:10D53C00F5B3E147E314F9DE9305A1002285EFE092
:10D54C004FF119BD01458280F9CE011152C42E8ACA
:10D55C00854522CC4EC656C206CE26CA4AC8AA8AD1
:10D56C00B6893284EF10B039D1471DC5B7370020CA
:10D57C003737002083C707FF834617FF814419E024
:10D58C00B684BE8637370020032787FE9397440066
:10D59C00BA9763EDD400D547F2406244D244424975
:10D5AC00B249224A924A3E85056182803E89C10772
:10D5BC0003D727FF09C7850493F4F40FD9BF31CCE7
:10D5CC009565938525C0130500029730FB1FE780F6
:10D5DC00A0A62326A90061D11306000281459384DD
:10D5EC0004049730FB1FE780E0DA23119900230035
:10D5FC000900231359010DC4373700201C340326AE
:10D60C0007362304F900118C8327C900118411807B
:10D61C00C0AF23A02901814741B723260900C1BF10
:10D62C0023044901FDB785473E858280B73700202A
:10D63C0083C507FFB737002003A787FE8147639593
:10D64C00F5008146368582803223BA8619C2E30BF7
:10D65C00A6FE850793F7F70F4107D5B7B73700201C
:10D66C0003C607FFB737002003A787FE8147631562
:10D67C00F6008146368582802E23BA8681C54C23DE
:10D68C00E38AA5FE850793F7F70F4107CDB7B737A8
:10D69C00002083C537FFB737002003A70736814723
:10D6AC006395F5008146368582801223BA8619C2AD
:10D6BC00E30BA6FE850793F7F70F4107D5B7B737EE
:10D6CC00002003C817FFB737002083A787FE014748
:10D6DC006315E800814636858280B223BE8609CA6E
:10D6EC00F2236317A600D04701C63222E305B6FE2B
:10D6FC0005071377F70FC107E1BF411122C440455D
:10D70C0026C206C6AA8415C0484409C59730FB1F1B
:10D71C00E780809F484809C59730FB1FE780C09E73
:10D72C0022859730FB1FE780209E26854146814548
:10D73C009730FB1FE78000C6B2402244FD579CB4D3
:10D74C00924441018280011122CC2A842A2106CEE6
:10D75C002EC6EF102068324622858145EF00F05628
:10D76C0022856244F24005616FF03FF905C53A210C
:10D77C00411122C406C62A8411CBDD45EF00F057B7
:10D78C0022852244B24041016FF03FF7B24022445F
:10D79C00410182808280411126C2B1469304C5FFAB
:10D7AC00B386D402B73700201387073706C622C4C6
:10D7BC00369736276397B602484305C51384073757
:10D7CC009307F00F6305F6001C21639CC70097308C
:10D7DC00FB1FE7806093B147B387F402A29723A2A3
:10D7EC000700B2402244924441018280411122C47C
:10D7FC002E8426C24946AA848145228506C69730C6
:10D80C00FB1FE78020B995CCDC2C13974700B7376A
:10D81C00002083A70736BA979A231AA0BA23FE23AF
:10D82C003AA0373700200357E7FE5AA09A207AA077
:10D83C00BA201AA4DA203AA4FA205AA49A241EA8D0
:10D84C007AA4B2402244924441018280B73700202E
:10D85C0083C507FFB737002003A80736B73700206A
:10D86C0003A687FE014781476394E5003E858280CD
:10D87C00142299CA544689CAD42E9206C2966315AC
:10D88C00D500850793F7F70F05071377F70F4106B8
:10D89C00E1BF130600643386C50293069500AA8582
:10D8AC0037D50400130585776F60CF84411122C4EE
:10D8BC0006C62A840835EF60EF9DFD571CB4B240B4
:10D8CC00224441018280011122CC4AC84EC652C466
:10D8DC0056C25AC006CE26CA2A89AE890144373AA6
:10D8EC000020B73A00201D4B83471AFF6365F404F0
:10D8FC0063990902B7390020373A0020930AF00FD8
:10D90C0083C709FF6364F4061144A144228505040E
:10D91C0042041306F00FCA854180EFF0DFE7E317EE
:10D92C0094FEF2406244D2444249B249224A924A9D
:10D93C00024B0561828083A78AFE93144400BE9437
:10D94C009C208DC3FE20639F270163956901AA204B
:10D95C00EF10404826854E868145EF00103726850E
:10D96C00EFF0BFD905041374F40FBDBF83278AFEF3
:10D97C0093144400BE949C208DC39C34638F570138
:10D98C00FE20639C27012685EFF05FF22685D145AA
:10D99C00EF00B0362685EFF05FD605041374F40F54
:10D9AC0085B741677917630BE502411122C406C69E
:10D9BC0085472A846399F50022852244B24081452B
:10D9CC0041016FF05FF089476396F5008545EF10D4
:10D9DC0000737DD1B24022444101828082809D45FA
:10D9EC006FF07FEEB737002003D5E7FE8280B737A4
:10D9FC00002003C7C7FE011106CE68876C868547D9
:10DA0C006318F70070009305E1000545EF50501FB7
:10DA1C00F24005618280A947631DF6029C31982172
:10DA2C00A207D98F1EA1BC31B821A207D98F3EA164
:10DA3C00DC31D821A207D98F5EA1FC31F821A207D5
:10DA4C00D98F7EA19C359825A207D98F1EA501459B
:10DA5C008280054582809147631EF6009C31982197
:10DA6C00A207D98F1EA1BC31B821A207D98F3EA124
:10DA7C0001458280054582809387C5FF93960701F7
:10DA8C00C1820D47636ED7003147B387E702373742
:10DA9C00002013070737BA97A8A38EA301458280ED
:10DAAC00094582809306402037370020AA8763F40B
:10DABC00A60093074020F1172317F7FEB737002075
:10DACC002389B7FEB7370020238AB7FE8280190559
:10DADC00956542054111938535C0418106C6972055
:10DAEC00FB1FE780605501C9B240E955410117237E
:10DAFC00FB1F6700A36EB24041018280B737002044
:10DB0C00238907FEB737002079710547238607FE66
:10DB1C00B73700202386E7364ECEB7370020B7390B
:10DB2C00002022D426D24AD037340020B73400202B
:10DB3C00A38A07FE37390020B7370020938939FFB5
:10DB4C0006D652CC2AC6230804FEA38804FE2397CB
:10DB5C0007FE232409FE23800900EF1040303245D4
:10DB6C00B7370020130600032382A7363735002071
:10DB7C001305053781459730FB1FE780A081373AA5
:10DB8C00002003450A3A130404FF938414FF13097D
:10DB9C0089FE05CD9565938545C012059720FB1F21
:10DBAC00E7808049373700202320A73619CD03465C
:10DBBC000A3A93070A3A9C332380C900814512061E
:10DBCC009CA09720FB1FE780E07CB737002003C5A3
:10DBDC0047409C209565938555C03E951375F50F70
:10DBEC0008A012059720FB1FE78000452320A90001
:10DBFC0051C11020814512069720FB1FE7808079C8
:10DC0C00032709001420814725077D56639EF604DF
:10DC1C00EF104045B1473305F5029565938565C016
:10DC2C00420541819720FB1FE7800041B737002058
:10DC3C0023A4A7362A8401CDEF10C0423146330607
:10DC4C00C502814522859720FB1FE780A0742254D2
:10DC5C00B25092540259F249624A37E50400130556
:10DC6C00E59A45616F10A040850710A393F7F70F55
:10DC7C00410769BF230004002380040051BF4111F8
:10DC8C009397050126C206C622C44AC0C187AE843A
:10DC9C0063DE070837390020034549369720FB1F00
:10DCAC00E780405E2A8429C9182193070009631272
:10DCBC00F7041831CD476319F706B736002003482F
:10DCCC00250003C5B62437370020834727FF1306EA
:10DCDC00640081458146130727FFAA886316D80282
:10DCEC0091C11CA31C2391C7034549368545EF50B0
:10DCFC00DF8D2285EF506FD42165258DB2402244F3
:10DD0C0092440249410182800C22AE9793F5F70FA1
:10DD1C0093F7F80F63F4A50093F7F50F850693F6C8
:10DD2C00F60F090685455DBF092BE1B793F7150082
:10DD3C000145E9D7EF00305209CDB737002083C732
:10DD4C0027FF81CBB737002003C547368545EF50F9
:10DD5C00DF8713C514005DB785462A8763FFC602AB
:10DD6C009C319021A207D18F1EA16399D700BC31A1
:10DD7C00B421A207D58F3EA1014582808946014579
:10DD8C00639ED700BC31B421A207D58F3EA3DC31F2
:10DD9C00D421A207D58F5EA382800545828091474E
:10DDAC00631EF6009C319821A207D98F1EA1BC31AD
:10DDBC00B821A207D98F3EA10145828005458280FA
:10DDCC009147631EF6009C319821A207D98F1EA1A2
:10DDDC00BC31B821A207D98F3EA1014582800545EF
:10DDEC008280A1476318F6029C319821A207D98F33
:10DDFC001EA1BC31B821A207D98F3EA1DC31D8219C
:10DE0C00A207D98F5EA1FC31F821A207D98F7EA180
:10DE1C00014582800545828089476319F6009C3153
:10DE2C009821A207D98F1EA10145828005458280C9
:10DE3C003E2279714ECE06D622D426D24AD0130772
:10DE4C00F007AE896371F70209473AC47C8630004B
:10DE5C0093F5F50FEF00F076B2502254925402591C
:10DE6C00F249456182805A22D9462A89328463F765
:10DE7C00E6007E2263F4F6006379F70023140100B8
:10DE8C00300093F5F90F4A85F1B70A2202C4EFF07E
:10DE9C001F80AA8435C5EFF07F9B9C246369F50035
:10DEAC001146A246CE854A85EF00706875B73400DE
:10DEBC0026869305F00F4A85EFF00FE975F1A2471E
:10DECC001A24DC479AA33A20BAA35A20DAA37A2060
:10DEDC00FAA3DA209AA7DC4495C793F4F90F2286AB
:10DEEC00A6854A858297C167FD172A86E31BF5FA3A
:10DEFC0022459947F9451CA144A1EFF09F99A9BF70
:10DF0C00094645B7014671BFA947631DF6029C310E
:10DF1C009821A207D98F1EA1BC31B821A207D98F95
:10DF2C003EA1DC31D821A207D98F5EA1FC31F821AA
:10DF3C00A207D98F7EA19C359825A207D98F1EA543
:10DF4C0001458280054582809C211CA19C311CB11D
:10DF5C00BC31B821A207D98F3EA1828023220500B3
:10DF6C00D82189476304F70005458280F6210D47C7
:10DF7C00E37CD7FE9C45011106CE22CC26CA4AC8AA
:10DF8C004EC684339023A204D18C138644006311B3
:10DF9C00D604A033BC23AE8922045D8C9307C4FF46
:10DFAC00C207C1832A896361F70203A58900231183
:10DFBC00990023108900F1559720FB1FE780002260
:10DFCC002322A900014531A02285EFF02FE671FD37
:10DFDC000545F2406244D2444249B249056182800F
:10DFEC00397122DC2E841C204AD806DE26DA4ED665
:10DFFC0019472A89B2856392E70630202800EFF092
:10E00C001FDAAA8405E92884EFF04FE2AA890C30C4
:10E01C0015C937F704002E86130727D234009D4507
:10E02C004A85EF00702F4E850946814579294E852A
:10E03C00EFF0AFECF250625426854259D254B259EB
:10E04C002161828089477C803C840A867C813C8566
:10E05C007C824A85EF00F056F1BF49476398E7028E
:10E06C0032202800EFF0FFD7AA8469F5373500205D
:10E07C00130505375E2599E381446DBF18301420D4
:10E08C0068253C000146CA85CD2C6DB75147639E6F
:10E09C00E70032202800EFF01F98AA8441FD0C30D5
:10E0AC0030004A85EFF0DFD871B75947639BE7041E
:10E0BC0032202800EFF03F9AAA842DFD2C844A854B
:10E0CC00EFF0EFDF05C9584534851E23B697C2071C
:10E0DC00C1831EA3D5D35C47C5D3B737002083C7F4
:10E0EC0027FFD9DBB737002003C547368545EF50EE
:10E0FC00CFCD89B789473EC03C840A860C307C82E0
:10E10C0089BF0C300A8623100100EF00904BADB78D
:10E11C005D71A6C256DA86C6A2C4CAC04EDE52DCF7
:10E12C00AA8A8831AE8432C6EFF04FD3B24501EDE6
:10E13C008144B6402644268506499644F259625AD3
:10E14C00D25A61618280230205002311050083C924
:10E15C00040085472A846399F900B0202808EFF061
:10E16C00BFBFAA8405491DA09D476391F9041821DE
:10E17C008D47E31FF7FAB02028080549EFF05FC47C
:10E18C00AA8409E505468145228581262285EFF082
:10E19C00EFF108243C080147CE862686D685F12A65
:10E1AC00E30909F82285EFF04FD561B7CD47639BA2
:10E1BC00F90018219147E31DF7F6B0202808EFF07D
:10E1CC00BFC545B7D547E395F9F6034A050089471E
:10E1DC00E310FAF6B02028080549EFF0FFD2AA8424
:10E1EC0055F583570102A1EBB8841306F0035C4488
:10E1FC00930607FCC206C182636AD600B085D94675
:10E20C0063F6C600B486D94563EDD5002A20BAA3BF
:10E21C000549EF00303C03560102D2852285A92C1A
:10E22C00B5B7AC87BAA3D2A38EA3F6A385471CA01F
:10E23C00014A0149CDB7014AF9BF7971AA8522D4A7
:10E24C0026D22221AA84280806D6EFF03FD1F24527
:10E25C0099E53DE185452285EFF06FF975A0BC8409
:10E26C0015476395E706B8858D4763F7E7046800A3
:10E27C00EFF09FCD3887DD4763FBE7008C86B7074F
:10E28C0017008507100822853EC8EF0090333C87A5
:10E29C00B88591076305F7002285EFF04FF41C86D3
:10E2AC0072466C00858B1106228591CFEFF05FE6EC
:10E2BC0001C52285EFF0AFF2884449DD9720FB1FA2
:10E2CC00E78080E441BFEFF0BFD1DDB71147638930
:10E2DC00E7001387A7FF42074183854663EBE602FD
:10E2EC003147F117B387E702373700201307073799
:10E2FC00BA979A2371D3A8233008A28505204DFD27
:10E30C00B8849147E318F7F4B25022549254456103
:10E31C0082802C082285FD2445F1FDB701114AC8E5
:10E32C002A89314526CA06CE22CC2EC6B284972025
:10E33C00FB1FE780C0EF21C1B2459307000A1EA165
:10E34C002EA12A84214611058DC0A6859720FB1F7E
:10E35C00E780A0FDA2854A85EF401FF30145F240FE
:10E36C006244D24442490561828081459720FB1F5B
:10E37C00E7804002C5B70545DDB7797126D2AA847E
:10E38C001305000206D622D42ECE32CC36CA3AC899
:10E39C003EC69720FB1FE78080E929C56246F245FF
:10E3AC004247D246B2472A84130520FA08A010B07F
:10E3BC002EA058A054B013058400614691CFBE85A1
:10E3CC009720FB1FE78060F6A2852254B250268569
:10E3DC00925445616F405FEB81459720FB1FE780AE
:10E3EC0060FBDDB7B250225492544561828058458F
:10E3FC00797122D406D62A84AE862DC73E23FC859D
:10E40C00930720066397F504B737002003D6E7FE81
:10E41C007E236373F600B28713F6F70F2E2B1C2B9B
:10E42C008D8F93F7F70F81E5890793F7F70FB29765
:10E43C00FD17B3C7C702FC863E206E200824FC845F
:10E44C0001473C080146EFF05FF3B250225445619E
:10E45C008280582FB737002083A707361207BA9748
:10E46C00FE23D1BF2EC61946814528089720FB1FD5
:10E47C00E78040F2B246C9B7797122D406D626D2CB
:10E48C002A8499CD81470147930600062E866E207B
:10E49C000824EFF09FEEB2502254925445618280D2
:10E4AC00B284280059469720FB1FE780A0EE6484B5
:10E4BC0099E43E2048446C007C85EFF02FB33C007F
:10E4CC000147930600060146D9B7797106D68147F4
:10E4DC0091E93E21584570867C843C0001C73E235F
:10E4EC007C853C002E866E2108250147930600068C
:10E4FC00EFF0BFE8B25045618280411122C406C6DC
:10E50C001C2111472A846392E7022E866E2108256E
:10E51C0081470147CD46EFF05FE649466E20224425
:10E52C00B240154541016FF00FA713F7B70F89469D
:10E53C006317D7000146EFF03FF45146C5B70D47BE
:10E54C006398E7002244B240014641016FF0FFF7A7
:10E55C00B2402244410182809A21B146B737002053
:10E56C0071173307D70293870737BA97D84301EB54
:10E57C00D841AAA70145D8C3BA219AA78280594588
:10E58C008280797122D4404526D24AD006D6AA84FC
:10E59C002E8931C4484419C59720FB1FE780C0B6AB
:10E5AC00232604001E20EE2088247C853E20014773
:10E5BC00930640067C861E244A867C871C483EC8EF
:10E5CC00BE207C843C00EFF05FDBA30E24012328EB
:10E5DC000400B250225492540259456182802800A2
:10E5EC00314681459720FB1FE780C0DABE20EE2024
:10E5FC0088247C8401473C00930640064A86EFF051
:10E60C00DFD7C1BF797152CC2A8A8A2126D206D68D
:10E61C0022D44AD04ECE56CAAE84EFF02F8119E1E7
:10E62C00854795A84045AA8965DC7E21E39A47FF7A
:10E63C001E2463890710542CB73A002003A70A360E
:10E64C009206FD173697C2077A23C1831EA4631660
:10E65C00F70093053006EFF09FD95C48A5EFC84052
:10E66C00034915001C2122093369F900BE20130748
:10E67C002900631CF702F9559720FB1FE78000B6B1
:10E68C00C8C02391240103C589002686D285EFF0EA
:10E69C00FFC8814721E1B250225492540259F249E9
:10E6AC00624AD24A3E85456182809565938515C044
:10E6BC004A859720FB1FE780209848C8C840231C38
:10E6CC002401F9559720FB1FE78040B1BE20C8C03C
:10E6DC00F917BEA0484825CDB220362C1E2C330885
:10E6EC00D60063C80707582C83A70A36954512072E
:10E6FC00BA97BE2363C90705CC4036959720FB1FFC
:10E70C00E780A0C23A2CBE20BA97C2071A2CC1834C
:10E71C003EACE397E7F003D7290003C5890030002E
:10E72C0078845848D2857C853AC6EFF03FBF11C536
:10E73C0048489720FB1FE780209D232A0400232CA8
:10E74C000400F9BD99454E85EFE0FFFFD1BDA5450D
:10E75C00DDBF9145CDBFBA2171CBB737002083D631
:10E76C00E7FEED4763E5E60C011122CC2E8426CAA8
:10E77C00AA844840914506CE9720FB1FE78000A64F
:10E78C003E20AA861CA13E20A1831CB11E203CA1C8
:10E79C001E20A1833CB13220C167F9171106420635
:10E7AC0041826394F4042AC4314532C69720FB1F7E
:10E7BC00E780E0A7AA85CD471DC1930700F91CA1EE
:10E7CC003246F957A2463EA189475CA1B7370020D3
:10E7DC0072A114C503C54736EF401FAB8147F24009
:10E7EC006244D2443E850561828081452685EF4096
:10E7FC00B055AA8711E9B736002003C726FF65D3A9
:10E80C007D172389E6FEE1BF09476304E5021D4736
:10E81C006303E50249476302E5027D47E311E5FC2A
:10E82C00B736002003C726FF8147D1BFED473E8591
:10E83C008280D1476DB791475DB789474DB70111BC
:10E84C004AC831471309C5FF3307E902B73700201F
:10E85C0026CA9384073706CE22CCBA94D84029C74F
:10E86C0013840737B737002083C627FF854795C623
:10E87C0068849E24AA242C003AC67C85EFF0BFED58
:10E88C0011C5C8409720FB1FE7800088B147B3072C
:10E89C00F902A29723A207008547F2406244D244B2
:10E8AC0042493E85056182808147C5BF797126D278
:10E8BC004445373700204AD0FE200359E7FE52CC9E
:10E8CC0006D622D44ECE56CA2A8A63F327013E8935
:10E8DC00BA284209135909019E2835CF998F4A84C9
:10E8EC0063D5270113940701418089452285EFF0F8
:10E8FC000F9EAA89CD4A31C5BE202AC660857C846C
:10E90C00BE2899EB9E28930925001CA19E28A18363
:10E91C001CB1637424058228BE28CC4422864E8503
:10E92C00BE959720FB1FE78040A003556A002C0082
:10E93C00EFF07FE2AA8A15C54E859710FB1FE78082
:10E94C00A07CB2502254568592540259F249624A24
:10E95C00D24A45618280890759B7791442044180B3
:10E96C0065BFBA289E203A94FD17C20742049A2824
:10E97C00C18341809EA0A2A86376E400F9F3FD5701
:10E98C00DCBCC1B781455285EFF0BFBF5DBF79716B
:10E99C004AD03739002052CC034A59FF22D456CAE8
:10E9AC005AC85EC662C406D626D24ECE5284B73A38
:10E9BC000020054B930BF00F373C002083A78AFEF9
:10E9CC0093144400BE9483C90400639B6907DC4420
:10E9DC00A5CBD84735C79A2329CBB737002083C797
:10E9EC0027FF99CF2685EFF07FECAA8515E9B7377D
:10E9FC00002083C717FF05046351F402A30A89FEA4
:10EA0C00B25022544E8592540259F249624AD24A6B
:10EA1C00424BB24B224C45618280A30A09FECDB712
:10EA2C002685EFF01FB68149E1BFDC3F639A770181
:10EA3C00930520062685EFF09F9BDC44A38E0700F0
:10EA4C0083471CFF05041374F40F6363F400014443
:10EA5C00E31644F7C9BF4111154506C6EFF03FDE7A
:10EA6C0009C50545B240410182801945EFF03FDDF3
:10EA7C006DF91145EFF0BFDC6DF51D45EFF03FDC96
:10EA8C006DF1B737002083C717FFE9DFB2404101B2
:10EA9C006FF0FFEF9E210D47F117C207C18363632F
:10EAAC00F706DC41A5C3411122C42E84854526C23C
:10EABC0006C6AA84A92529C92685B92BC167F917C9
:10EACC00638FF40009ED3E2099CB16201947639310
:10EADC00E604373700200357E7FE63FDE702B7373C
:10EAEC00002083C727FFA285268599C72244B24000
:10EAFC00924441016FF03FC62244B240924441011E
:10EB0C006FF09FA5094582805145B2402244924442
:10EB1C00410182806D45D5BF397126DA4ED6AA8463
:10EB2C00AE895D4589454AD806DE22DC328936C677
:10EB3C003AC4EFE0DFF935C122472A84014511C7F9
:10EB4C00B24613054400B6850297935785002300FF
:10EB5C003401A30024013CB09547FC84B737002056
:10EB6C0083C727FF28A01105E88522CE2C0826850F
:10EB7C0095C3EFF05FBEAA8411C522859710FB1FC9
:10EB8C00E7808058F250625426854259D254B259CB
:10EB9C0021618280EFF05F9CF9BFCD44E5B77971BC
:10EBAC0026D24AD052CC56CA06D6BA8A22D44ECED7
:10EBBC0019472E89B284368A6395E5062A220944C0
:10EBCC00EFE0DFA62AC635C55C4583596500BE2338
:10EBDC009EA0B247B736002015472380570103C6C5
:10EBEC00C636BAA3130716001377F70F2386E6363B
:10EBFC00D0A301E705472386E63651476317E900A2
:10EC0C001547BAA0DC479A249AA75287A686CA85CC
:10EC1C004E85EFF07FF02A84324515C4EFE0FFAD4E
:10EC2C0009A842867400BE85AA89EFE0FF912A8468
:10EC3C004DD12285B250225492540259F249624A63
:10EC4C00D24A45618280F945EFE0BFC4DDB79E2111
:10EC5C001CA19E21A1831CB1BE213CA1BE21A1837C
:10EC6C003CB1114582809E211CA19E21A1831CB127
:10EC7C00BE213CA1BE21A1833CB1DE215CA1DE21E1
:10EC8C00A1835CB1FE217CA1FE21A1837CB1214535
:10EC9C0082809E211CA19E21A1831CB109458280EA
:10ECAC009E211CA19E21A1831CB1BE213CA1BE2191
:10ECBC00A1833CB1DE215CA1DE21A1835CB1FE21EC
:10ECCC007CA1FE21A1837CB19E251CA59E25A18340
:10ECDC001CB5294582809A218546AA8718A19A21BC
:10ECEC00218318B19A216319D700BA2138A1BA210E
:10ECFC00218338B1114582800945631DA700BA21D3
:10ED0C001945B8A3BA212183B8B3DA21D8A3DA21E3
:10ED1C002183D8B382809E211CA19E21A1831CB18A
:10ED2C00BE213CA1BE21A1833CB1114582807971E9
:10ED3C0026D24AD04ECEB2842A89AE892946814544
:10ED4C00480022D406D636849710FB1FE7808064D7
:10ED5C0064868DE43E207C82B737002083D7E7FEA3
:10ED6C007C845C4481CFD42F3737002003270736AF
:10ED7C0092069E2736973A237C85788337F70400D2
:10ED8C004A851307C7CA540013F6F90FD545EFF09F
:10ED9C00BFD82A8911C195E085471CA02302040025
:10EDAC00014681452285EFF02FEDB25022544A8561
:10EDBC0092540259F249456182802285EFE0FF931B
:10EDCC00EDB737F70400B286130727CE2E8685459C
:10EDDC006FF09FD401116887B7F60400416570008D
:10EDEC0001489307F00F0D479386A6C599457D15ED
:10EDFC0006CEEFF0DFDAF24005618280B7F6040050
:10EE0C00B28701482E861147938626C7C9456FF0F5
:10EE1C001FD937F70400B2861307E7C92E86CD45F4
:10EE2C006FF09FCF011122CC373400201304843AA9
:10EE3C0026CA4AC84EC606CE2A89AE899304040354
:10EE4C001C4081C7CE854A8582971104E31A94FE33
:10EE5C00F2406244D2444249B24905618280B737DC
:10EE6C00002003C51725411122C4373400209377A5
:10EE7C0035001304C43F09811CB4AA9706C626C2E8
:10EE8C001CA4ADCB1305C0033385A702A56585056E
:10EE9C00B73400209710FB1FE780001A102493074B
:10EEAC00C00381453306F60223A2A43A9710FB1F38
:10EEBC00E780404E83A7443A1424014789077D56C6
:10EECC006341D7022244B2409244373500201306E6
:10EEDC00000381451305853A41011713FB1F670099
:10EEEC00634B92A32381070023A507020507938791
:10EEFC00C703F9B7B2402244924441018280011108
:10EF0C0022CC2EC632C406CE2A849720FB1FE78063
:10EF1C00E0B72246B24511E9C167F9176303F40063
:10EF2C005145F24062440561828054555C218DC28A
:10EF3C0013F7270141456314A70015457DF2C18BDA
:10EF4C003D45E5D3BC2E0145E3FDB7FC3145D1BFB2
:10EF5C00C18B0145F9F71545E9B7797126D24AD02D
:10EF6C00B7340020416922D44ECE52CC56CA5AC86E
:10EF7C0006D6AA8901449384C43F373A0020930AE9
:10EF8C00C0037D19054B9C246364F400014525A83E
:10EF9C00B307540303274A3ABA97BA2363162701D7
:10EFAC0005041374F40FC5B7C8333000938567009C
:10EFBC00EFD041061946CE8528009710FB1FE7803D
:10EFCC00C047E31F65FDB250225492540259F249D6
:10EFDC00624AD24A424B45618280B737002083C5D2
:10EFEC004740C166B737002003A7473AFD16814753
:10EFFC006395F500014632858280035827003A86D6
:10F00C006306D80003480700E307A8FE850793F7BB
:10F01C00F70F1307C703E9BF411106C69720FB1F63
:10F02C00E780C0A609C54A29B2404101828001454A
:10F03C00E5BFB737002083C64740B737002003A78A
:10F04C00473A0145814711076393F60082801023EC
:10F05C0001C605051375F50F850793F7F70F130711
:10F06C00C703DDB7B737002003C547408280373769
:10F07C0000209306873A81471307873A31468C4222
:10F08C0091E58A07BA9788C3014582808507910666
:10F09C00E397C7FE4D458280411106C622C49720D6
:10F0AC00FB1FE780A09E0DCD2A842A218545EFF019
:10F0BC007FD7485409C59710FB1FE780E0042285D1
:10F0CC001306C00381459710FB1FE780A02CFD574A
:10F0DC003EA0230204000145B2402244410182803B
:10F0EC000945DDBF411106C69720FB1FE780009A3A
:10F0FC0009C54825B240410182800145E5BFC16781
:10F10C00F9176305F502411122C406C62E84972017
:10F11C00FB1FE780A097AA87014589C7C823698C84
:10F12C0033358000B2402244410182800545828003
:10F13C00011106CE2EC69720FB1FE7802095854730
:10F14C0001C95A29B24585476304B7004EA98147C6
:10F15C00F2403E850561828029CD01114AC84EC618
:10F16C0037390020C16922CC26CA52C456C206CEF9
:10F17C000144AA841309C93F373A0020930AC003FB
:10F18C00FD1983478900634BF400F2406244D2447A
:10F19C004249B249224A924A05618280330554039E
:10F1AC0083274A3A3E953E216383370182940504B6
:10F1BC00C9BF8280B737002003C64740B73700204D
:10F1CC0083A7473AC166014589070147FD1691455A
:10F1DC006313E600828003D807006309D80003C8D4
:10F1EC00A7006315B80005051375F50F0507137710
:10F1FC00F70F9387C703E9BFB737002003C6474013
:10F20C00B737002083A6473A014781479106631020
:10F21C00E602858393C7F7FFC207C1830545636286
:10F22C00E50285473395A7004205418182808C22F7
:10F23C0099C1CE36CD8F05071377F70F9386C6038A
:10F24C00F9B793F61700F1FE050585831375F50FD5
:10F25C00F9B7797156CAAA8A2E8526D24AD04ECED3
:10F26C0052CC5AC85EC662C406D622D4AE84328B47
:10F27C00368CBA8B3E8AC28946899720FB1FE78061
:10F28C00E0803DED41657D159720FB1FE7800080F8
:10F29C002A84554531C81946DE8513056400A3023E
:10F2AC0084019710FB1FE78040088357010326A0B9
:10F2BC00230264013EA883574103230054012326F3
:10F2CC0004025EA8230644012317340123182401E9
:10F2DC00EFF09FF20AB8232A04022685232C04029D
:10F2EC008145EFF03FB40145B2502254925402597B
:10F2FC00F249624AD24A424BB24B224C456182805F
:10F30C004545DDB7B737002083C64740B7370020E7
:10F31C0003A7473A81476395F60041657D158280C6
:10F32C003A861307C703835547FF6394A5002A2227
:10F33C008280850793F7F70FF9BFB737002003C812
:10F34C004740B737002083A6473A416601477D16F0
:10F35C00954811436314E80001458280BE2236852E
:10F36C00638EC702CC5A9DC9BC31AC2189CD938523
:10F37C0097FD93F5F50FE372B3FE9387D7FA93F7E6
:10F38C00D70F89EF82809385F7FD93F5F50FE3F6A0
:10F39C00B8FC9387D7FA93F7D70FE1D30507137708
:10F3AC00F70F9386C6037DB7B737002083C5474058
:10F3BC004166B737002003A7473A7D168147254899
:10F3CC006394F5000145828036233A85638BC60031
:10F3DC00545B81CAB4329386E6FD93F6F60FE37460
:10F3EC00D8FE850793F7F70F1307C703D1BF011199
:10F3FC0022CC2A84494506CEEF601FC31DC12AC604
:10F40C0022859710FB1FE780606801CD6244B737F7
:10F41C00002032460E39F24003C5F73F05616F40BC
:10F42C00AFB8F24062440561828039714ED652D435
:10F43C00AE892A8A93053005414526DA4AD856D238
:10F44C0006DE22DC32C63689BA8A9710FB1FE780AB
:10F45C00A0BECD4429C92A8489446381090432465B
:10F46C008145F08241469710FB1FE780A0F256863B
:10F47C00CE8522859710FB1FE78020EB2146630E7B
:10F48C000902CA8528089710FB1FE78000EAA286AC
:10F49C0050082C085285EF30707AAA842285971078
:10F4AC00FB1FE78060C6F250625426854259D25445
:10F4BC00B259225A925A21618280814528089710AC
:10F4CC00FB1FE78020EDE1B7411122C4405926C251
:10F4DC0006C6AA8429CC085409C59710FB1FE780DF
:10F4EC00A0C2285809C59710FB1FE780E0C16858D7
:10F4FC0009C59710FB1FE78020C1285C09C5971030
:10F50C00FB1FE78060C0685C09C59710FB1FE78094
:10F51C00A0BF0325040809C59710FB1FE780C0BED8
:10F52C0022859710FB1FE78020BE23AA04022244E9
:10F53C00B73700208E38B240924403C5F73F4101E3
:10F54C006F408FCE411126C206C622C4AE849710DE
:10F55C00FB1FE780A05329C14C592A8495CD83A861
:10F56C00C50703A88507FC59B859F4219221AC2191
:10F57C002685EF607FB32285EFF01FF5EFF0DFE219
:10F58C0001CD2244B7370020B240924403C5F73F67
:10F59C00854541016F406F83B24022449244410142
:10F5AC008280011122CC06CE2A842EC69710FB1F16
:10F5BC00E780C04D5C5989CF9E23B245639A870082
:10F5CC0085476397F5006244F24005616FF0DFEF09
:10F5DC00F240624405618280411106C622C426C2F3
:10F5EC00EFF0BFD529C14059AA8415CC3C209DC74A
:10F5FC00B737002083A7C73D89C7DC4399C3228551
:10F60C00829738309307F002631FF7002244AA2038
:10F61C00B2409244814541016FF0DFF2B7370020D0
:10F62C0083A7873DD1BFB2402244924441018280DE
:10F63C00411126C24AC006C622C4AA842E8997103C
:10F64C00FB1FE780A04405CD405955C41E20639490
:10F65C00970A3C30130710026395E7083C20ADCFA6
:10F66C007C5403270408DE2B15E313F7170019CF7E
:10F67C0018545A23058B19CB930720023CB0B24087
:10F68C0022449244024905454101828013F7270028
:10F69C0001CB18545A23098B01C793074002F9BFB9
:10F6AC00918B81CB1C54DE23918B81C79307600215
:10F6BC00F1B7B737002083A7C73DF1D3DC43E1D3C3
:10F6CC002285829738309307F0028145E319F7FAC7
:10F6DC002685EFF03FE765B7B737002083A7873D56
:10F6EC00E9BF1307A0026398E7006304090013093C
:10F6FC002003CA85F1BF631C090026859710FB1FE8
:10F70C00E780C03809C55C2193E707015CA1A68599
:10F71C004A85EF604FABA5B7797126D29947EC8536
:10F72C00AA842E858D4522D406D632C636C4FC84D6
:10F73C00EFE0EFB92ACE4D441DC13246A246AA8550
:10F74C00328582962A8419E52C082685EFF08FB431
:10F75C002A8411C572459710FB1FE780E09A268515
:10F76C00EFF0FFC82285B25022549254456182803A
:10F77C004111B716050022C42E862E849386A6FD51
:10F78C00894506C626C24AC02A89EFF0FFF80C202C
:10F79C00AA844A85EFF01FDBB24022442685024939
:10F7AC00924441018280B737002083A7873D85CBE7
:10F7BC009C4395C71D71A2CC86CE984110082A8413
:10F7CC003AC8D84185453ACA829711C548862A203D
:10F7DC006C00EFF0FFF9F640664425618280828070
:10F7EC00AE8711CD785501CF142394A1143394B165
:10F7FC00342BB4A1142F584BB4B1D8C182804146DC
:10F80C0081453E851713FB1F6700C3B8B73700202F
:10F81C0083A7C73D91C703A387006303030002833B
:10F82C0009458280373700200327875E1DC7584360
:10F83C00AA8705450DC703A50708411106C69306FF
:10F84C0005021306050C930505061305050402971E
:10F85C00B2401375F50F410182800545828082808C
:10F86C004DC9357122CD2A840A2126CB4AC94EC7EF
:10F87C0056C306CF52C55AC1DEDEB68AB2892E896E
:10F88C009710FB1FE7808020AA8431C50C182285B5
:10F89C00EFF01FF53C20138A6400A9CBEF501FED4D
:10F8AC002A8B014583CB5400EF505FEAAA840C10DD
:10F8BC000818EF10605508542C10EF108055D288A2
:10F8CC00268A56C05E88D2875A8714103010CE858F
:10F8DC004A85EF20207DFA406A44DA444A49BA4905
:10F8EC002A4A9A4A0A4BF65B0D618280EF501FE858
:10F8FC00AA8B014503CB5400EF505FE52ACE085488
:10F90C000C10EF1060502C100818EF108050F248BB
:10F91C004DBF8280C14719C91455C14781CA78555A
:10F92C0011C7BC32BD4663F3F6001C2F3E858280A6
:10F93C00894779C9F1C9411106C622C426C21C31B6
:10F94C002E849CA13C219CB13C31BCA15C21BCB15E
:10F95C005C31858B93968700DE2193F7F7EFD58F7B
:10F96C00DEA1543193F7F7DFA20693F60620DD8E65
:10F97C00D6A1583193F6F6BF220713770740558F5F
:10F98C00DAA15C31FD769386F67F8D87858B758F3A
:10F99C00AE07D98FDEA17421F99B858ADD8ED6A1A5
:10F9AC0078219377270013F7D6FF5D8FDAA17C219E
:10F9BC0093F647009377B7FFD58FDEA17821DD9BB7
:10F9CC004D45218BD98FDEA1EF600FE6AA845145FE
:10F9DC00EF608FE5383093F4F40FC94763609702FA
:10F9EC001375F50F636CE50014201147E14763674D
:10F9FC00D700143005476363D7008147B2402244D7
:10FA0C0092443E85410182803E85828015C1AA8741
:10FA1C0009458DC141112E8541469385170006C6B7
:10FA2C009710FB1FE7806090B24001454101828036
:10FA3C0009458280828089470DC585C5411106C65E
:10FA4C001831AE87194698A1930525001385170028
:10FA5C009710FB1FE780608DB24081473E854101C6
:10FA6C0082803E85828015C1AA8709458DC14111CE
:10FA7C002E8541469385170006C69710FB1FE7801D
:10FA8C00C08AB24001454101828009458280828052
:10FA9C00894705C99DC5411106C638211431AE8769
:10FAAC002207558F9AA1214693053500138527000F
:10FABC009710FB1FE7806087B24081473E8541016C
:10FACC0082803E85828015C1AA8709458DC141116E
:10FADC002E8541469385170006C69710FB1FE780BD
:10FAEC00C084B240014541018280094582808280F8
:10FAFC00894709C981C91831BD46E14763E4E6006D
:10FB0C0098A181473E85828015C1AA8709458DC180
:10FB1C0041112E8541469385170006C69710FB1F91
:10FB2C00E780A080B2400145410182800945828076
:10FB3C00828015C1AA8709458DC141112E85414688
:10FB4C009385170006C69700FB1FE780007EB24026
:10FB5C000145410182800945828082801DC1AA87AE
:10FB6C00094595C141112E85130600049385170094
:10FB7C0006C69700FB1FE780407BB2400145410160
:10FB8C00828009458280828015C1AA8709458DC172
:10FB9C0041112E8541469385170006C69700FB1F21
:10FBAC00E780A078B24001454101828009458280FE
:10FBBC0082801D71A2CC2A84084586CEA6CA230653
:10FBCC000100042135479387F4FF93F7F70F636423
:10FBDC00F70C37E706008A0713070760BA979C43B0
:10FBEC0082870C08EFF0DFD4C9476310F502994700
:10FBFC005C862A206C00EFF0BFB7F6406644D64412
:10FC0C00256182800C08EFF01FEC31C51C86F5F3E2
:10FC1C002A20EFF0CFFDD5B70C08EFF0FFEEF5B7CB
:10FC2C000C08EFF0FFECD5B70C08EFF03FDEF1BF9E
:10FC3C000C08EFF0FFE5D1BF0C08EFF0DFE2F1B7F5
:10FC4C000C08EFF05FDFD1B70C08EFF09FEE75BF3B
:10FC5C001C312308F1002A209710FB1FE78000E3DA
:10FC6C00A14705C15825631AF702B737002003A72F
:10FC7C00C73D9D4719C7184309C71008A6850297A9
:10FC8C00AA875C8661B70C08EFF05FEDBDBF0C086E
:10FC9C00EFF09FEF9DBF9D47A1BFB737002003A793
:10FCAC00873DC1BF011122CC06CE26CA4AC84EC61A
:10FCBC001821930720092A846313F7121C31394742
:10FCCC006393E70A56210967610781476391E61040
:10FCDC00B739002003A5C93ECE84630A050E0C4437
:10FCEC0003C90500631E09001C2185052146A9CF07
:10FCFC0029059700FB1FE780406383A7C43EB5C36B
:10FD0C0049459700FB1FE78080522A840DC5930755
:10FD1C0010FC1CA1A300250183A5C43E0905414686
:10FD2C0089059700FB1FE780406083A7C43EA2852E
:10FD3C008833EF306FD503A5C43E9700FB1FE780D7
:10FD4C00A03C23A6043E31A809059700FB1FE780C1
:10FD5C00C05DEF30606E05494DF183A7C93E23802D
:10FD6C0027018547ADA01307E0036398E708382106
:10FD7C009547631CF7024A21EFF0CFB69147E31287
:10FD8C00F5FEB737002083A7873DE1DF03A387008B
:10FD9C00E30903FC72244A20930564006244F24098
:10FDAC00D2444249B24905610283A147631CF70062
:10FDBC006C204A206244F240D2444249B249056167
:10FDCC006FF01F87930600038147E303D7FEF240D1
:10FDDC006244D2444249B2493E8505618280930611
:10FDEC00000A8147E315D7FEEFF0BFDC084435D994
:10FDFC009700FB1FE7804031ADB78147C9BF0111A8
:10FE0C0026CA06CE22CC89440DCD85CDAA842E845B
:10FE1C0068008D45EF500FE71C872685228693F7E7
:10FE2C00F70393E707046C005C87EF20A01EAA84FD
:10FE3C0009E90D466C00130534009700FB1FE780A1
:10FE4C00C04EF24062442685D244056182805D71C9
:10FE5C004EDE86C6A2C4A6C2CAC052DC56DA5AD836
:10FE6C005ED6894945CD5DCA138B4500420B135BA9
:10FE7C000B01AE8A2A8A930530055A85B284970005
:10FE8C00FB1FE780601B2A84CD4949C9EF50FF8FC7
:10FE9C002A895686D285935A8900135A0901937B75
:10FEAC00F90F1305440093FAFA0F137AFA0F13594A
:10FEBC0089019700FB1FE780C05CA301740123013B
:10FECC005401A300440123002401EF507F8BAA8529
:10FEDC00414608089700FB1FE780A05A21473400D1
:10FEEC005A86A2850808EF206039AA891DE12146AF
:10FEFC002C0023807401A380540123814401A3812D
:10FF0C002401138544009700FB1FE7808057EF50B6
:10FF1C009F8822859700FB1FE780001FB640264470
:10FF2C004E8596440649F259625AD25A425BB25BEC
:10FF3C006161828001114AC82A892E8506CE22CCA5
:10FF4C0026CA2EC69710FB1FE78040B45DCD4059E2
:10FF5C005DCC5C300947B24593F6B70F6387E6007A
:10FF6C0011471305E00F639DE7061E2009456399B1
:10FF7C00B706930484004146CA8526859700FB1F6B
:10FF8C00E780A03A4146CA85130584019700FB1F00
:10FF9C00E780A039383085469307F7FE93F7F70FC3
:10FFAC0063E6F6041306C4033285C14532C6EF502E
:10FFBC006FCD32469306C402A6852285EFF05F8A88
:10FFCC003C2089CB22856244F240D24442490561EF
:10FFDC006F1020083830C947E306F7FE3CB00145E6
:10FFEC00F2406244D2444249056182809307100575
:04FFFC000145E317C1
:020000025000AC
:10000000F7FE3C20E5D722856244F240D2444249C3
:1000100005616F10000B0945D1BF4945C1BF39715A
:1000200052D42A8A328526DA4ED606DE22DC4AD817
:10003000AE8932C69710FB1FE78000A6C94451C1A4
:100040004059C9443DCC1E203246639CC7065C30F3
:10005000A18BB1CB373900208327895E9304E00F51
:10006000ADC39C47B9CF9304840126854146D28510
:100070009700FB1FE780202C8327895E83250408D7
:1000800026869C4793850504180881462E8582970D
:10009000AA844146CE8508089700FB1FE780A03A56
:1000A00093F4F40F11E1894438309307B005631AD3
:1000B000F7002285EF00D07D3C2089CF9307C00553
:1000C0003CB0F250625426854259D254B259225A59
:1000D000216182809307E005E5B739C9011126CA7D
:1000E00006CE22CCAA8409459DCD0D4628002E843B
:1000F0008D059700FB1FE78000241C8570002C00F5
:1001000093F7F70393E7070426855C85EF1050719A
:1001100019E90D46A28568009700FB1FE780A03211
:100120007D153335A000F2406244D24405618280DF
:1001300009458280011152C42A8A32854EC656C2B0
:100140005AC006CE22CC26CA4AC82E8BB28AB6899D
:100150009710FB1FE780409409ED8944F240624408
:1001600026854249D244B249224A924A024B05614D
:1001700082805C592A89C544F5F34D45EF509FEBC9
:100180001374F50F5145EF50FFEAE38809FC83C76C
:100190008901E3E487FC1375F50FE360F5FC930533
:1001A0003005130540089700FB1FE780A0E9232ACC
:1001B000A9022A84CD445DD11306400881459700E9
:1001C000FB1FE780E01DA30104002301440123027B
:1001D0006401231054012326340723240402A302BC
:1001E00004008144E30C0AF62285EF009061AA84A2
:1001F00035D54A85EFF00FAE95B7397122DC06DEB2
:1002000026DA4AD84ED652D456D25AD05ECE62CCD6
:1002100066CA0944630D0610630B0710AA8B3A895E
:10022000368BB28A2E8C9710FB1FE780E0862A8AD5
:100230005144630E050E9305300541459700FB1FA1
:10024000E78040E0AA894D447DC18344190083477B
:100250002900A204C207BE9483470900BE948347C5
:100260003900E207BE9483278A0263E697007D5730
:1002700009446399E70A63070C0083474A00054471
:10028000898BCDC3930C4B00214681450A85C20C56
:100290009700FB1FE780C01093DC0C01930530052D
:1002A00066859700FB1FE780E0D92A8C4D443DC945
:1002B0005A86D68511059700FB1FE780401D114621
:1002C000CA8562859700FB1FE780601C4146930545
:1002D0008A014E859700FB1FE780601B21478A86B5
:1002E0006686E2854E85EF10307A2A841DE5214628
:1002F0008A8528009700FB1FE78060192146930537
:10030000490028009700FB1FE780E0138547631E24
:10031000F502A6855E85EF60AF8862859700FB1FBA
:10032000E78040DF4E859700FB1FE780A0DE228537
:10033000F2506254D2544259B259225A925A025B34
:10034000F24B624CD24C216182800544F9B779713D
:100350009397050122D406D626D24AD04ECEC18725
:100360002E8463D50704B73400209384C43FA8309B
:100370009700FB1FE780C0F12AC609CDEFF05F931D
:10038000B24511E5A8209307F00F631EF5002E85F6
:10039000EF207FEB2165218DB250225492540259F7
:1003A000F24945618280EF20FFEEEDB793F715002B
:1003B00091C7EFF02FA313451400F9BFA1E1014548
:1003C000E1BF850493F4F40FEFE09FCAE3F9A4FEC4
:1003D000339599001319050113590901B3772401C5
:1003E000EDD34A85EFE0DFF2C167FD176305F50045
:1003F000DD45EFF0EF953345240179BF854485490C
:10040000E1B7B737002023A6073EB737002023AE59
:10041000073C37170500B73700201307A79B23AC0D
:10042000073CB737002023A8E73E3707050093872E
:10043000073F13078770D8C337F7040013076743D4
:1004400098C737270500B73700201307078423A074
:10045000E73E371705009387073E1307E73ED8C3EB
:10046000371705001307E76898C78280B737002061
:1004700083C70740A18B89C7B73700209387073F01
:1004800037370020232EF73C01458280B737002004
:1004900083C70740918B89C7B73700209387073EF2
:1004A00037370020232CF73C01458280011106CE0E
:1004B0002AC6EFF01FF53245B73700209945A38FC4
:1004C000A73EEFD02FDCF24037F504001305E55AC4
:1004D00005616FE09FBA1C5581C7A1473E858280A8
:1004E000011122CC26CA2A84AE8413050004930588
:1004F000300506CE9700FB1FE780C0B408D475C155
:1005000013060004A6859700FB1FE780C0E278541D
:100510003C2B93F68700F5CA1454B422A18AF5C681
:1005200083270408DDEF93053005130500109700BD
:10053000FB1FE78020B12320A4088D4745C5A302F7
:10054000040078549C30143391EB91EABC20918BD9
:10055000C5E33C2B918BC9EF854701A881C6214794
:1005600058B089C75C3093E707015CB06C54BC2974
:10057000858B99CB1C540547BC238D8B6396E70074
:100580007C2093E717007CA08327040889C77C2080
:1005900093E787007CA05C300547639EE70A9304DD
:1005A00084004146814526859700FB1FE78040DF98
:1005B00041468145130584019700FB1FE78040DE1B
:1005C0001306C4033285C14532C6EF407FEC832752
:1005D00004083246B9CF2285EF00B02E93070005FC
:1005E00025C5A147F2406244D2443E850561828020
:1005F0009C2014231547B387E70237E7060013074B
:100600004765BA97B6979C238DB7943089C6143343
:1006100099C2E14799BFB420D58F918B95DF9C207B
:1006200014231547B387E70237E7060013078763EC
:10063000C9BF22859306C402A685EFF02FA32285A9
:10064000EF00F02159FDC1470A203CB08145EF5031
:100650005FBF814741BF13F7870135CFC18B93043B
:1006600084004146B1C7890526859700FB1FE780B6
:1006700080CC41468145130584019700FB1FE7802C
:1006800020D27C201306C403328593E747007CA068
:10069000C14532C6EF40DFDF83270408324685C3F9
:1006A0002285EF0010229307200505FD3CB055B7C9
:1006B000814526859700FB1FE78080CE5DBF9306AE
:1006C000C402A6852285EFF06F9A2285EF003019CB
:1006D000CD4769DD39B7094785456388E70093F75A
:1006E000D70F11476396E70089450A20EF507FB581
:1006F0007C2093E747007CA08327040881C79307E9
:1007000010056DB7C5475DB73C21638B0722797132
:1007100022D406D626D24AD03C31130750052A846B
:10072000639DE706034975001306C503C14593574A
:100730003900AA973285842732C6EF407FD5B73774
:10074000002083A7875EA1C79C47B1C30325040887
:1007500093767900B3D6D4403246858A9305050452
:10076000180893E606081305050882971375F50F18
:1007700019ED41460C081305C4029700FB1FE780E2
:1007800080BB2285EF00B00D930760053CB0B250EE
:1007900022549254025945618280130710026392D9
:1007A000E7021C5503270508DE2361E313F7071052
:1007B0004DCF78555A2B1377071045CB930770020E
:1007C0003CB03C30130770026397E70C3C5885E35C
:1007D0009305300571459700FB1FE780A08628D858
:1007E00019C5714681459700FB1FE78060BB2458FF
:1007F000B1C4BC2C89E72285EFF08F92A8AC2858B1
:10080000814541469700FB1FE78080B928583D4746
:100810002C2D9387F5FF93F7F70F6364F700EF40F4
:100820003FC7EF203FC13C58A1458AAB1385270144
:10083000EF401FC62C580A20EF00B031930780020A
:100840000A203CB09700FB1FE7800025414609C500
:100850007E2513D617003E96B737002003C5F73F15
:1008600006068545EF201FF51DB713F7072009CBB6
:1008700078545A2B1377072001C79307900289B742
:1008800093F707409DDF7C54DE2B93F7074095DB01
:100890009307B00235B7130780026397E7023C580D
:1008A00099C78E2B0A2013862701EF00F02F1C54C6
:1008B000DE2313F7072029CF78545A2B137707200C
:1008C00021CB93079002ADBF13079002639BE70013
:1008D000EF403FEBAA850A20EF00102C9307A002FF
:1008E00085B71307A0026390E704EF40FFE8AA85ED
:1008F000854701456384F500814505452EC6EF40D7
:10090000BFE52A86B2450A20EF00B0251C54DE233D
:1009100093F707409DC37C54DE2B93F7074091CF9C
:100920009307B00231BF1307B0026398E700EF40AE
:10093000FFE5AA850A20EF00902A9307F002B9B5D7
:100940008280411122C4405926C206C67C54AA8422
:10095000DE2B13F7071011C718545A23137707100B
:100960000DE313F7072011C718545A2313770720F4
:1009700009EB93F707408DCB1C54DE2393F7074018
:1009800085C7930710023CB02285EFF0FFD73830BF
:100990009307F002631EF7002244AA20B24092445B
:1009A000814541016FE0DFBA9307F0023CB0EDB73B
:1009B000B2402244924441018280397122DC405984
:1009C00026DA4AD84ED606DEAA89AE843289630278
:1009D000043A2A211E206384A700A14421A03C20C0
:1009E00091EB9D44F250625426854259D254B2593B
:1009F000216182809387E5FF93F7F70F2D47E3622C
:100A0000F7FE37E706008A0713070767BA979C4384
:100A10008287B2852285EFF01FACAA84E1B74146F8
:100A2000CA851305C4049700FB1FE780C090228588
:100A30008525AA8411C1A1443C3013074005639663
:100A4000E700930790053CB071BF130760056395FD
:100A5000E7009307A005C5BFD147F5B79309C405C3
:100A60004E854146CA859700FB1FE780C08C032551
:100A7000040845C53C30130790056398E7002285BC
:100A80004D259307E0053CB079A01307A0056390BE
:100A9000E7087C3013D73700229714279D8BB3D6F5
:100AA000F640B737002083A7875E858A93E606F86D
:100AB00093F6F60F9DD39C478DD393050508180830
:100AC0004E861305050482979374F50FE39704F09F
:100AD00041460C081305C4049700FB1FE780A0964D
:100AE0007C304D47850793F7F70F7CB06377F700AD
:100AF0002285052D9307E005B9B7B737002003C558
:100B0000F73F8545EF203FAD930750052DBF1307F5
:100B1000C005E386E7F68144F1B5130984004E86EB
:100B2000CA8522851408EFE07FD441469305C404AA
:100B300008089700FB1FE7800091E30505EA8A8615
:100B40001306C403CE854A85EF10A06A05E122850D
:100B5000EFE01FDDB73700202A8783A7873F0A20F1
:100B6000814601468A858297AA8411C1A1449307D0
:100B70002002D1BD0C22EFE0BF9D71BF383093073A
:100B80002002E310F7E67C5889EB930530057145A8
:100B900097F0FA1FE780004B68D86858E30305E434
:100BA0004146CA8597F0FA1FE780E07864582285AD
:100BB000EFE01FD7A8AC93073002F1B538309307A8
:100BC0003002E310F7E21E226858214693052900FF
:100BD0001EA9490597F0FA1FE780E0757C54DE2BCB
:100BE00013F727002DC718545A23098B2DC39307D9
:100BF000400251BD383093074002E314F7DE3C5CFD
:100C000081EB85455D4597F0FA1FE780A04328DC1E
:100C1000285CE30205F0834709004146CA857CA9A8
:100C200097F0FA1FE780207193075002A9BD383072
:100C300093075002E317F7DA285C19469305190069
:100C4000410597F0FA1FE780006F7C54DE2B918BF3
:100C500095CF1C54DE23918B95CB9307600225B56D
:100C60007C5C89EB93053005514597F0FA1FE780CE
:100C7000603D68DC685CE30205D64146CA8597F0B2
:100C8000FA1FE780406B7C5C7D5798CB4E85EFF078
:100C90005FCB51B50325040813060004CA8513056C
:100CA000050497F0FA1FE78000692285EFE05FB83E
:100CB0003C30130700056395E70093074005E1B357
:100CC00013071005639CE700B737002003C5F73F03
:100CD0008545EF205F909307500575B313072005F6
:100CE000E39BE7E2B737002083A7875EE38707CE61
:100CF0009C47E38407CE83250408930484001808E6
:100D000093850508814626862E8582970A2010083D
:100D1000A685EF50EFDB9307B005B5B338309307E6
:100D2000E005E310F7CC8325040841464A8597F097
:100D3000FA1FE7804071AD44E30605CA03250408A5
:100D40004146CA8597F0FA1FE780E05E2285EFE012
:100D50003FBDB73700202A8783A7873F2C580A203A
:100D6000814601468297AA8411C1A14493071002CB
:100D7000D9B9AD47E391F5DA14222E2113066500A7
:100D80000821EF40FFD541BB894759C2D1C108A214
:100D90009C211CB29C313CA2BC213CB2BC31A302C0
:100DA00006005CA2DE21A183858B5CB2DA21137779
:100DB000072001C793E727005CB2DE2193F70740C5
:100DC00089C75C3293E747005CB2DE211397470185
:100DD000635607005C3293E787005CB2230306008A
:100DE000DC21858B7CA2DA21098B01C793E72700E0
:100DF0007CA2DE21918B89C77C2293E747007CA2ED
:100E0000DA218147218B09C778221367870078A2EE
:100E10003E8582802E86AA8505456FF0FFF62E86D8
:100E2000AA8509456FF05FF6894785C51DC1411147
:100E300006C6AE870D47AA8598A3138517004146BD
:100E400097F0FA1FE780204FB24081473E8541016D
:100E500082803E858280894785C51DC1411106C6B5
:100E6000AE871147AA8598A313851700414697F0CE
:100E7000FA1FE780404CB24081473E8541018280A5
:100E80003E858280894785C51DC1411106C6AE8752
:100E90001947AA8598A313851700414697F0FA1FB2
:100EA000E7806049B24081473E85410182803E85AE
:100EB0008280894795C90DC9411106C61D4798A171
:100EC0001A21AE87214698B11A212183B8A1930532
:100ED00025001385370097F0FA1FE780C045B24020
:100EE00081473E85410182803E858280894785C554
:100EF0001DC1411106C6AE872147AA8598A3138557
:100F00001700414697F0FA1FE780E042B240814760
:100F10003E85410182803E85828089479DC515C5F9
:100F2000411106C6254798A11821AE87194698B1E8
:100F3000930515001385270097F0FA1FE780A03F5F
:100F4000B24081473E85410182803E85828089474B
:100F500085C51DC1411106C6AE872947AA8598A33C
:100F600013851700414697F0FA1FE780C03CB24056
:100F700081473E85410182803E85828089478DC5BB
:100F800005C5411106C6AE873147AA8598A31385CA
:100F900017001306000497F0FA1FE780C039B2402B
:100FA00081473E85410182803E858280894785C593
:100FB0001DC1411106C6AE873547AA8598A3138582
:100FC0001700414697F0FA1FE780E036B2408147AC
:100FD0003E85410182803E858280894799C511C541
:100FE00095479CA11C219CB181473E858280894701
:100FF00099C511C5AD479CA11C219CB181473E8577
:1010000082800DC55D718A8586C6A2C42A84EFE000
:10101000EFFD0A20B71605000A86938646E19D4536
:10102000EFE04FF0B6402644616182800545828042
:101030000DC55D718A8586C6A2C42A84EFE00FFBC8
:101040000A20B71605000A869386E6E19D45EFE083
:101050006FEDB640264461618280054582805D71F6
:10106000A2C49305C5022A8441460A8586C697F024
:10107000FA1FE780402C0A20B71605000A869386DF
:1010800086E2C545EFE00FEAB64026446161828002
:101090005D71A2C49305C5032A8441460A8586C6AC
:1010A00097F0FA1FE78020290A20B71605000A8664
:1010B000938666E5C545EFE0EFE6B64026446161FC
:1010C0008280B737002083A7875EA9CB9C435D71E0
:1010D000A2C486C62A841305E00F8DCF0325040819
:1010E0009305050C1305050882978325040813064C
:1010F00000040A859385050897F0FA1FE780A0236E
:101100000A20B71605009386C6F70A8693051004D1
:10111000EFE04FE1B6402644616182801305E00FA5
:101120008280317122DD2A840A2126DB06DF4AD93A
:101130004ED752D556D35AD15ECF62CD9700FB1F02
:10114000E78080953C58AA8489EB9305300571456A
:1011500097F0FA1FE78000EF28D82858CD4705C937
:101160007146814597F0FA1FE78080230329040721
:101170002285EFE0EFFA230DA9003C20373900204B
:10118000638107128327895E85E39307E00FFA5096
:101190006A54DA544A59BA592A5A9A5A0A5BFA4B8B
:1011A0006A4C3E852961828083AB0701E38F0BFC8B
:1011B000032B0408EF404FDC2A8C0145EF40CFD9C8
:1011C000DC303858130B0B029309C403130AC4050F
:1011D000938A64003AC0B337F0002A879308010469
:1011E0005688B33680015286CE855A85829B1C5420
:1011F000B8232307E1029833A306E1029C232306C8
:10120000F1028327895ED1D303AB4701E30F0BF6CD
:10121000DC30B337F0003ECEEF400FD6AA8B01454D
:10122000EF408FD303270408F2472AC03AC2B338ED
:10123000700156887810930684004E86D285880007
:10124000029B7C54B82B2305E1029833A304E102EE
:101250009C232304F1028327895E03A94701EF4001
:10126000AFD12A8B0145EF402FCF83C854009C0893
:101270002A883EC2B3381001B33760013810930694
:1012800084015286CE8556C0880002990A20B7167E
:1012900005009386C6FA9008C545EFE0AFC8AA8757
:1012A000FDB5D4308327895E032B0408B336D00004
:1012B00083AB070136CEEF402FCC2A8C0145EF409F
:1012C000AFC93C58F246130B0B02130AC40593092D
:1012D000C403938A64002A88930801044E86D28549
:1012E0003EC05687B33780015A85829B1C54130B2E
:1012F0000103B8232307E1029833A306E1029C23EC
:101300002306F1028327895E83AB4701DC30B337C4
:10131000F0003ECEEF404FC62A8C0145EF40CFC3D0
:10132000F2472AC0B33880015688781093068400AB
:101330004E86D2855AC28800829B83250408414686
:101340005A8597F0FA1FE7800010AD47E31B05EEC2
:101350003DBDB71605002E86938646E8C5456FE06D
:101360006FBC5D71B287A2C44C802A84BE85130510
:101370001100194686C697F0FA1FE780C0FBB71622
:1013800005000A8622859386A6F1A145EFE08FB974
:10139000B640264461618280B71605002E8693868A
:1013A000C6EEC5456FE00FB85D71B287A2C46C8010
:1013B0002A84BE8513052100214686C697F0FA1FB0
:1013C000E78060F7B71605000A862285938626EB2C
:1013D000AD45EFE02FB5B640264461618280B71677
:1013E00005002E869386E6F4C5456FE0AFB37971AC
:1013F00022D406D626D23C31130730052A846381D5
:10140000E708130750056392E7089307A0053CB16E
:101410007C31C14513D737002A9714279D8B1305BC
:10142000C503B3D6F640858A93E606F893F6F60F21
:1014300036C6EF40EF85B246B737002083A7875EF8
:101440009DCB9C478DCB0325040818081306C403C5
:10145000930505041305050882971375F50F01ED33
:101460001305C40241460C0897F0FA1FE780A0EC70
:101470002285EFF0DFBEB250225492544561828043
:10148000930790053CB1814645BF13071002639155
:10149000E7027C5503270508DE2B61EF13F71700E1
:1014A00069CB18555A23058B69C7930720023CB0B6
:1014B0003C30130720026394E70E3C5889EB9305F8
:1014C0003005714597F0FA1FE780C0B728D8245837
:1014D000ADCC2285EFE0CFC4A8AC28588145414669
:1014E00097F0FA1FE780C0EB28583D472C2D9387D3
:1014F000F5FF93F7F70F636DF702B737002083C747
:10150000375FD9CB41468145080897F0FA1FE7803D
:1015100020E9B735002019469385052B080897F078
:10152000FA1FE78040E130580C082E85EF20E14497
:10153000EF105FF03C58A1458AAB13852701EF30CF
:101540003FF52C580A20EFF0DFE0930730020A2025
:101550003CB097F0FA1FE7802054414611C1722534
:10156000B737002003C5F73F06068545EF208FA457
:1015700019B713F7270001CB18545A23098B01C759
:10158000930740022DB7918B85D71C54DE23918B96
:1015900085D39307600221BFEF309FEF51BF130740
:1015A00030026396E7023C5899C78E2B0A201386B7
:1015B0002701EFF07FDF7C54DE2B13F7270021CBD0
:1015C00018545A23098B21C79307400249B71307C0
:1015D0004002639BE700EF40CF9AAA850A20EFF014
:1015E000BFDB93075002A5B713075002639DE702C4
:1015F000EF408F9815E5814505452EC6EF40CF9504
:101600002A86B2450A20EFF0DFD57C54DE2B918B81
:101610008DC71C54DE23918B8DC39307600205BFD9
:1016200085450145D9BF130760026398E700EF4085
:10163000EF95AA850A20EFF09FDA7C54032704086F
:10164000DE2B09EF13F7071011CB18545A23137729
:10165000071009C7930770023CB031BD13F707208C
:1016600009CB18545A231377072001C79307900218
:10167000E5B793F7074089CB1C54DE2393F7074067
:1016800081C79307B002C9BF9307F002F1B7397160
:1016900022DC26DA4ED652D406DE4AD8AE89328A09
:1016A000AA8497F0FA1FE780203F405941468145C0
:1016B0000A8597F0FA1FE780A0CE35C403590400CD
:1016C00063139906383093071002631FF7028327CC
:1016D000040899CF2C58A1C94A85EF10B057054589
:1016E000F2506254D2544259B259225A2161828036
:1016F0008A861306C4059305C40313058400EF000E
:10170000502F15E18A85C9BF2C5891CD9E29639C25
:1017100047012146C9054E8597F0FA1FE780A0D200
:1017200019C12C5855BF268597F0FA1FE780C0369F
:101730002A84054555D44C54B1C59E296394470568
:101740002146C9054E8597F0FA1FE780C0CF85472F
:10175000631AF502B737002083C777F489C74C5462
:10176000BC3D639AA70CBD452685EF103049B737BD
:10177000002083A707270145A5D71D4589458297E6
:101780000145B9BFB737002003C7475FB73900200D
:101790009389C923058B3E8929C3B7370020583068
:1017A00083C7C75E631BF702B735002019469385D0
:1017B000D55E1305640097F0FA1FE780C0C885471F
:1017C000631DF50083A7490381C791451D45829795
:1017D000BD452685EF10904219B7373700200347E3
:1017E000375F83A7490331CB0347495F098B09CB97
:1017F00081C795451D4582972685EF10F045C5B5F3
:1018000081C78D451D45829741468145080897F05F
:10181000FA1FE780E0B8B735002019469385052BFD
:10182000080897F0FA1FE78000B10C082E850A8699
:10183000EF20A1148A8526854DB58545C5FF6DBF6E
:10184000797122D440594AD04ECE52CC06D626D2F7
:10185000AA892E8A3289630A04622A211E20638C97
:10186000A700A144B2502254268502599254F2494D
:10187000624A45618280242099C09D44E5B79387E0
:10188000F5FF93F7F70F3147E369F7FE37E70600F7
:101890008A071307076ABA979C4382871C54F1F39F
:1018A000930530051305000497E0FA1FE78080795F
:1018B00008D445D903470900914763F4E7008D44F4
:1018C00055B7034719008547E3EBE7FE130600040D
:1018D000CA8597F0FA1FE78000A60C547054A30243
:1018E0000400D4415C4A858AFD8E5E2AF99BD58F1F
:1018F0005EAAD841544AF59B0583058B8582F98EF3
:101900008606DD8E56AADC41584AED9A8983858B7E
:1019100009837D8F0A07558F5AAAD4415C4A5D9B83
:101920008D82858A8D83F58F8E07D98F5EAAD841E7
:10193000544A93F7F7EF2183058BA182F98EA20613
:10194000DD8E56AADC41584AA583858B25837D8F81
:101950009317970013F7F6DF5D8F5AAAD4415C4ABC
:10196000A982858AA983F58F9396A7009377F7BFFD
:10197000D58F5EAAD441584AAD82858A2D83758F52
:10198000FD769386F67F2E07F58FD98F5EAA3C2AC7
:1019900003250408A18BFDC3BC21A18BE5C3E31281
:1019A00005EC930530051305001097E0FA1FE7805A
:1019B00060692320A40801D57C54A30204000347D6
:1019C0001900943399E641C75C3093E707015CB096
:1019D00021A0A1475CB06DFB2285EFF06FE56C5450
:1019E000BC29858B89CB1C54BC238D8B89C77C205B
:1019F00093E717007CA08327040889C77C2093E71E
:101A000087007CA05C300547639BE70A414681451F
:101A10001305840097F0FA1FE780809841468145BE
:101A20001305840197F0FA1FE7808097C1451305DD
:101A3000C403EF30FFA5032704089307000511E353
:101A4000C1470A203CB08145EF40AFFF21BDB82B14
:101A5000118B19E703472900118B19E3854785BFCF
:101A60009C23154783460900B387E70237E7060042
:101A700013074765BA97B6979C2391BF19C597E09E
:101A8000FA1FE7802069232004087C54983311C78B
:101A90000347190019C3E1471DBFB82B118B09E794
:101AA00003472900118B5DDB9C2315478346090002
:101AB000B387E70237E706001307876365BF13F7AD
:101AC000870139CBC18B13058400414695CF890529
:101AD00097F0FA1FE780208641468145130584016F
:101AE00097F0FA1FE780C08B7C20C1451305C40323
:101AF00093E747007CA0EF30BF998327040899CB78
:101B0000930720053CB0B9BB814597F0FA1FE780E9
:101B10002089D9B7CD47FDB7094789456386E700D6
:101B200011476397E70085450A20EF408FF121A018
:101B30001947E38AE7FE7C2093E747007CA08327D0
:101B4000040881C79307100575BFC54765BF4146A7
:101B5000CA851305C40497E0FA1FE780C07D3C30B6
:101B600013076005639CE700B737002003C5F73F04
:101B70008545EF105FA69307500569B74547638316
:101B8000E7029306C4021306C4039305840022856A
:101B9000EFD0DFCD2285EFF08FCCAA8411C1A14414
:101BA000D1478DB7C947B9BF9309C4054E85414692
:101BB000CA8597E0FA1FE78000780325040869C505
:101BC0003C30130790056398E7002285EFF04FCC77
:101BD0009307E00505BF1307A0056399E706B7372C
:101BE000002083A7875EE38A07C803A88700E3066F
:101BF00008C87C30930505084E8613D73700229716
